:020000040801F1
:10C00000B08E0020B9C20108D9790208DB79020894
:10C01000ED790208EF790208F179020800000000CA
:10C02000000000000000000000000000CBC201087A
:10C03000F379020800000000CFC20108A14D0208F8
:10C04000D3C2010843560208D3C201085F46020862
:10C05000D3C20108D3C201081144020831440208C6
:10C060005344020873440208954402080B3E020838
:10C070004D3E02088F3E0208DB3E0208F13F0208F7
:10C080004140020891400208D3C20108D3C201080E
:10C09000D3C20108D3C20108D3C20108B5440208C3
:10C0A000D3C20108D3C20108D3C20108D3C2010818
:10C0B000A94F0208CB4F0208ED4F0208D3C2010876
:10C0C000D3C20108D3C20108D3C20108D3C20108F8
:10C0D000D3C20108CB3802083B390208AB39020849
:10C0E000F744020897460208D3C20108D3C20108E8
:10C0F000D3C20108D3C20108D3C20108D3C20108C8
:10C10000D3C20108D3C201080F500208D3C20108EC
:10C110001B3A02088F3A02083150020853500208B5
:10C12000E14002082F4102087F410208CB4102088A
:10C1300000F002F800F0B0F80AA090E8000C824489
:10C140008344AAF10107DA4501D100F0A5F8AFF266
:10C15000090EBAE80F0013F0010F18BFFB1A43F0E5
:10C160000103184770170100901701000A444FF0AF
:10C17000000C10F8013B13F0070408BF10F8014B46
:10C180001D1108BF10F8015B641E05D010F8016B8B
:10C19000641E01F8016BF9D113F0080F1EBF10F8EF
:10C1A000014BAD1C0C1B09D16D1E58BF01F801CB12
:10C1B000FAD505E014F8016B01F8016B6D1EF9D595
:10C1C0009142D6D3704700000023002400250026AA
:10C1D000103A28BF78C1FBD8520728BF30C148BFEA
:10C1E0000B6070476E290BF0B98770290CF09F80A7
:10C1F00066290FF0CA8465290FF0C78467290FF0FC
:10C20000C48461290FF0C38403681B0A28BF41F06E
:10C21000800169290BF0668764290BF06387752913
:10C220000BF060876F290CF02C8078290CF06B8064
:10C23000E9290CF02786E4290CF02486F5290CF076
:10C240002186EF290CF02980F8290CF06A80036818
:10C25000DB0928BF41F0800163290CF0DE857329DA
:10C260000CF0E385E3290CF00186F3290CF0068637
:10C27000002070471FB50CF0C1FE04000020002113
:10C280000EF0AEFD401C6060002000210EF0BEFDEF
:10C29000E0601FBD10B510BD0DF09CF91146FFF711
:10C2A000E9FF00F02EFC0DF0C8F903B4FFF7F2FF30
:10C2B00003BC07F0DAF80000094880470948004746
:10C2C000FEE7FEE7FEE7FEE7FEE7FEE7FEE7FEE746
:10C2D000FEE7FEE704480549054A064B70470000A3
:10C2E000FF7A020831C10108B05E0020B08E002044
:10C2F000B06E0020B06E002010B508F0F9FEF548D1
:10C300000078C0074CD0F44806F07AFB032804D02C
:10C31000BDE81040F1A006F0DFBCEF49F3A03231D8
:10C3200006F0DAFCEC49F5A006F0D6FCF648EA4C3B
:10C330004178E1B994F832103039092917D894F8C6
:10C3400035103039092912D894F8371030390929B5
:10C350000DD821783039092909D8E17830390929EF
:10C3600005D861793039092901D801214170DA49AC
:10C37000E27D0B31E5A006F0AFFCD74994F825200B
:10C380001831E5A006F0A8FCD349E6A0263106F056
:10C39000A3FCD149BDE810402C31E5A006F09CBCBF
:10C3A00010BD38B508F0A4FE4FF4007006F056FC3E
:10C3B0000446002000906A462146E14806F0B8FD98
:10C3C000B0B920460CF00DF9217828290CD194F849
:10C3D0002510262908D1221812F8051C242903D17A
:10C3E00012F8031C292907D02146D6A006F074FCB8
:10C3F000204606F06DFC38BD6278412A15D0632ACC
:10C4000008D02146D7A006F067FCDEA1522002F03A
:10C410009AFCEDE782B22146E14806F03AFD002899
:10C42000E6D0E0A006F0B2FCE2E72146E2A006F08A
:10C4300053FCDDE738B508F05BFE4FF4007006F002
:10C440000DFC0446002000906A462146D44806F0C0
:10C450006FFD20B9BDF80010204601F0AAFC20466F
:10C4600006F036FC38BD10B508F042FEBDE81040BD
:10C4700001F080BD38B508F03BFE964C20784007AF
:10C4800029D54FF4806006F0E9FB054600200090B6
:10C490006A462946D04806F04BFDC8B9BDF80020D1
:10C4A0002946CE4805F027FE032811D0BDF800200C
:10C4B0002946CA4805F01FFE032809D0207820F03D
:10C4C00004002070C6A006F061FCC5A004F0A1FE27
:10C4D000284606F0FDFB38BD7CB508F009FE4FF498
:10C4E000806006F0BBFB06460020019001AA3146A1
:10C4F000C04806F01DFD002851D1BFA1304606F00E
:10C5000055FE0546002D46DB4FF4007006F0A6FBF5
:10C5100004464FF480700090711900230A222046CF
:10C5200006F075FD20460CF05CF8217828290CD126
:10C5300094F82510262908D1211811F8052C242A51
:10C5400003D111F8031C292907D02146AEA006F01B
:10C55000C3FB204606F0BCFB21E06178412915D0E1
:10C56000432908D02146AFA006F0B6FBB5A1522062
:10C5700002F0E9FBEDE782B22146894806F089FC2A
:10C580000028E6D087A006F001FCE2E72146B4A02F
:10C5900006F0A2FBDDE73146B9A006F0F7FB304616
:10C5A00006F096FB7CBD70B508F0A2FD4948007806
:10C5B00040072DD5B948044605F0FDFAB748401F9D
:10C5C000054604F0DFFF2B462246B5A1482002F0C5
:10C5D000BAFB102006F042FB06462B46B7A21021FC
:10C5E00030460BF001FD304602F09AFA1021304639
:10C5F0000CF0ECF82346B3A2102130460BF0F4FC0B
:10C60000304602F054FA3046BDE8704006F060BB98
:10C6100070BD38B508F06CFD4FF4807006F01EFB5D
:10C620000446002000906A462146A84806F080FC97
:10C6300090B9BDF80010204605F0D9FD254A78B123
:10C64000022823D0032828D0042814D0A0A006F064
:10C650009DFB9FA004F0DDFD204606F039FB38BDB0
:10C66000107820F0040010709EA006F08FFB9DA0B3
:10C6700004F0CFFDF0E7107820F0010010709EA0CC
:10C6800006F084FB9CA004F0C4FDE5E79EA006F044
:10C690007DFB9DA004F0BDFDDEE7A0A006F076FBCB
:10C6A0009EA004F0B6FDD7E704F022B838B508F034
:10C6B0001FFD4FF4806006F0D1FA04460020009080
:10C6C0006A462146994806F033FC08B921462FE115
:10C6D00031E10000350000202C280020BBF1C8A16A
:10C6E000475053CAFDBEDDCAA7B0DC00555443C84D
:10C6F000D5C6DAA3BA2573B6C8000000555443CA9C
:10C70000B1BCE4A3BA25730000000020CEB3B6C8C4
:10C71000A3BA257325630000BEADB6C8A3BA2573BE
:10C7200025630000CBD9B6C8A3BA2573BDDA0000D3
:10C73000BDC7B7BDCFF2A3BA2573B6C800000000CD
:10C7400040110020555342CAD5B5BDCFC2D0D02725
:10C75000B7C727B7A8CAFDBEDDD6A13A2573202EDC
:10C7600000000000555342CAD5B5BDCFC2D0D0CECF
:10C77000B4D6AAC0E0D0CDCAFDBEDDD6A13A25739D
:10C78000202E0000555342CAD5B5BDCFC2D0D0CE61
:10C79000B4D6AAC0E0D0CDCAFDBEDDD6A10000004F
:10C7A0003C0800207355736572636D64517565753F
:10C7B00065D2E7B3F6A3A100555342C9CFCEBBBBA8
:10C7C000FAC8B7C8CFCAD5B5BDCAFDBEDDD6A13A35
:10C7D0002573202E000000003A0D0020F2010020F9
:10C7E0005463702053656E644461746120457272B5
:10C7F00021000000202000202B51495552433A20AF
:10C800002272656376220000544350CAD5B5BDCF6D
:10C81000C2D0D027B7C727B7A8CAFDBEDDD6A13A78
:10C8200025732000544350CAD5B5BDCFC2D0D0CE59
:10C83000B4D6AAC0E0D0CDCAFDBEDDD6A13A2573DC
:10C8400020000000544350CAD5B5BDCFC2D0D0CED1
:10C85000B4D6AAC0E0D0CDCAFDBEDDD6A10000008E
:10C8600054637020736572766572C8B7C8CFCAD535
:10C87000B5BDCAFDBEDDD6A13A257320000000007B
:10C8800054435020CFC2D0D0CAFDBEDDBDE2CEF6AB
:10C89000CAA7B0DC3A25732000000000821D0020EA
:10C8A0004353513A25732C204543323020566F6C48
:10C8B000746167653A25736D5600000025736D56E7
:10C8C000000000004353512573000000262400207F
:10C8D00054637020756E6B6E6F776E207572632077
:10C8E0002E000000546370207365727665722063B9
:10C8F0006C6F736564202E00546370205044502088
:10C900006465616374202E0054637020696E636FE8
:10C910006D696E672066756C6C202E005463702004
:10C92000696E636F6D696E67202E00004C190020E0
:10C93000D7A006F0D1F9204606F0CAF938BD38B5BF
:10C9400008F0D6FB4FF4806006F088F9044600201A
:10C9500000906A462146D34806F0EAFA18B9214603
:10C96000D1A006F0B9F9204606F0B2F938BD2DE99C
:10C97000F04108F0BDFBD14ED14C4FF000053078AE
:10C98000C10708D0810706D5410704D5000702D5A5
:10C990002570BDE8F0812078401CC0B220700228CC
:10C9A00004D9C8A004F035FC0BF04AF83078C00771
:10C9B0000CD1CAA002F057F804F083FE03286AD015
:10C9C000C8A004F026FCCBA006F086F93078C10799
:10C9D0001DD080071BD4CAA002F045F81E2006F027
:10C9E0003DF907461E21384605F0FDF803285CD0C6
:10C9F000384604F00EFC307820F00100307004F06E
:10CA000081FE384606F068F9384606F061F930785C
:10CA1000C10714D0810712D5400710D4BAA002F084
:10CA200022F802F076F9032844D0307820F0040090
:10CA30003070B9A006F050F9BAA004F0EAFB3078E3
:10CA4000C10711D081070FD500070DD405F0A7FD50
:10CA500003283BD0307820F008003070B5A006F0F5
:10CA60003BF9B8A004F0D5FBBAA006F035F9307850
:10CA7000C1078ED081078CD541078AD5000788D59C
:10CA8000B84805F098F8B748401F04F07BFD02F065
:10CA900065F825707DE702F0CDFA307840F00100AE
:10CAA0003070B1A006F018F990E7307840F002003D
:10CAB0003070A6E7307840F004003070ADA14C2013
:10CAC00002F041F9B1A006F007F9B8E7307840F07C
:10CAD00008003070B0A001F0C6FF02F0F5F907467B
:10CAE000AFA14C2002F02FF9032F04D0B1A004F025
:10CAF00090FB0AF0A5FFB9A006F0EEF800F0E8FA06
:10CB0000B2E708B54FF4E0314FF0006008F0D5FD12
:10CB100008F0EEFA4FF4407008F09AFDB34800F0C8
:10CB200091FBB34800F01AFCB24800F0F0FAB248AA
:10CB300003F060FE08F0DCFA00F070FA01F09DFAF4
:10CB4000AE4C4FF47A7501230A222946207808F06A
:10CB5000B6F9AB49207808F097F908F0C9FAAFF2B6
:10CB6000F110009000236A100221A6A00BF08AF9B0
:10CB7000534C60600BF09EF9AFF23D200090012312
:10CB800064220221A1A00BF07DF9A0600BF092F9C4
:10CB9000AFF2E74002230090642219469EA00BF0FA
:10CBA00071F9E0600BF086F9AFF2035000900323B7
:10CBB000642202219BA00BF065F920610BF07AF949
:10CBC000AFF2B150009004233222022197A00BF063
:10CBD00059F960610BF06EF9AFF2356000900523F2
:10CBE000AA00022194A00BF04DF9A0610BF062F9AC
:10CBF000AFF21B70009006230A22022192A00BF0D4
:10CC000041F9E0610BF056F9AFF2977000900723FD
:10CC10000A2202218FA00BF035F920620BF04AF9AD
:10CC2000AFF2BD7000900823322201218CA00BF0DE
:10CC300029F960620BF03EF9AFF607000090092376
:10CC40003222012189A00BF01DF9A0620BF032F90C
:10CC5000AFF6B10000900A231422012186A00BF048
:10CC600011F9E0620BF026F9AFF6731000900B2378
:10CC70002A46022182A00BF005F920630BF01AF975
:10CC80008249834801F0D4FF01F0EBFFFEE77047D3
:10CC9000527334383520726563646174613A257368
:10CCA000202E000046150020527332333220726568
:10CCB00063646174613A2573202E00003500002002
:10CCC00000000020CFB5CDB3CDF8C2E7B1C0C0A3FE
:10CCD000A3ACD6D8C6F4CFB5CDB32100CED5CAD635
:10CCE000D6D03A00C4A3BFE9B0B2D7B0D2ECB3A358
:10CCF00021000000CED5CAD6CAA7B0DC00000000D3
:10CD0000C8EBCDF8D6D03A00C1ACBDD3544350B730
:10CD1000FECEF1C6F73A0000544350C1ACBDD3CAB1
:10CD2000A7B0DC00544350C1ACBDD3CAA7B0DC21CE
:10CD30000000000048545450B3F5CABCBBAFCAA7AA
:10CD4000B0DC000048545450B3F5CABCBBAFCAA70E
:10CD5000B0DC2100CACDB7C545433230D7CAD4B400
:10CD600021000000821D0020CED5CAD6B3C9B9A6C5
:10CD70002100000044657669636520746370206358
:10CD80006F6E6E657463656421000000544350C18A
:10CD9000ACBDD3B3C9B9A600D7A2B2E1D6D03A0090
:10CDA00044657669636520526567697374657221AD
:10CDB0000000000048747470B3F5CABCBBAF4F4BA1
:10CDC000A3ACD7A2B2E1C7EBC7F3CAA7B0DCA3AC50
:10CDD000D6D8C6F4CFB5CDB321000000D3B2BCFE87
:10CDE000D7A2B2E1B3C9B9A621000000420C0020CD
:10CDF00048000020FF0700202465030034000020C5
:10CE0000D1D001084E65745461736B005273323394
:10CE1000325461736B0000005273343835546173BF
:10CE20006B0000004C65645461736B005463705573
:10CE300072635461736B000054637048656172746F
:10CE40005461736B00000000546370446F776E543C
:10CE500061736B0054637055705461736B00000014
:10CE60004D656E755461736B0000000055636D6411
:10CE70005461736B000000005573625461736B0062
:10CE8000476E73735461736B00000000057F0208E6
:10CE9000C17E020800B585B01322A34968460BF095
:10CEA00016FC9DF80900401C8DF809009FA0008821
:10CEB000ADF80B00684607F0C5FE9B4804F0A9F9E1
:10CEC0009BA004F0A6F90AF0BBFD05B000BD70B54B
:10CED00005460C467B2008F095FD012804D122462A
:10CEE00098A128460BF0BBFC7C2008F08BFD0128A4
:10CEF00004D1224696A128460BF0B1FC7D2008F013
:10CF000081FD012804D1224694A128460BF0A7FCFC
:10CF10007E2008F077FD012804D1224693A12846FF
:10CF20000BF09DFC7C2008F06DFD88B97D2008F099
:10CF300069FD68B97E2008F065FD48B97A2008F0DF
:10CF400061FD012804D122468CA128460BF087FC04
:10CF5000BDE8704008F07DBE10B504460B2204F118
:10CF600019000BF07CFC002084F8250010BD10B5E2
:10CF700004460B2204F125000BF071FC002084F81C
:10CF8000310010BD30B5A1B07F480BF00BF87F48E1
:10CF90000BF008F87E4C7F48211DFFF7E8FF7D4B22
:10CFA0000B22253300217CA00AF0FCFF79481930C0
:10CFB000054607F0EBFA29467648FFF7CDFF2946EC
:10CFC0007AA00AF0EFFFA1787CA030390AF0EAFFDE
:10CFD0000121704807F0E3FA6E4A18217CA00AF09C
:10CFE000E1FF6C480B2131300446FFF770FF224609
:10CFF0000B217CA00AF0D6FF63480AF0D3FF802102
:10D0000001A80BF005FC23467BA2802101A80AF0B1
:10D01000EBFF01A804F0FDF821B030BD10B507F01A
:10D02000C0FE04F0D3F8002006F020F90D2007F030
:10D0300077FCFFF7A7FFAFF2A311022007F0D6FAA3
:10D0400000F070FF03F04FFB03F0B3FB08F0F6F9BC
:10D0500003F038FE4FF4E134204603F0FBFB20469A
:10D0600003F02AFCBDE8104008F0C3BA2DE9F041F6
:10D07000654D4FF48078404605F0F0FD0746634E5D
:10D080007068C0F30F240BE042463946284608F08A
:10D0900031F83A465EA14C2001F055FE05F5807549
:10D0A000641EA4B2F0D2414638460BF08FFB3279B1
:10D0B0003946284608F01EF83A4655A14C2001F0A2
:10D0C00042FE384605F004FEBDE8F04104F036B8F3
:10D0D00010B5524C207807F061FF5148007870B9C4
:10D0E0002C481022104913380BF020FA60B100F0E0
:10D0F0009DFF284814220C4913380BF0B0FB207810
:10D10000BDE8104007F03BBF01F0B6FCF7E7002197
:10D1100040F8191F41608160C160016141611938A7
:10D1200019210BF053BB0000245D002030310000BA
:10D130005274635F416C725F43616C6C6261636BDC
:10D1400021000000D6D8C9CFB5E7C6F4B6AF0000BD
:10D15000C8EDB8B4CEBBC6F4B6AF0000B6C0C1A22D
:10D16000BFB4C3C5B9B7C6F4B6AF0000B4B0BFDA38
:10D17000BFB4C3C5B9B7C6F4B6AF0000D3B2B8B434
:10D18000CEBBC6F4B6AF000054D3020898D3020851
:10D19000420C0020FF0700200D0A426F6F74B0E6BA
:10D1A000B1BE203A20252A2E2A7300000D0A4150D4
:10D1B0005020B0E6B1BE203A202573000D0A52750A
:10D1C0006E4170704E756D3A2041505025640000DC
:10D1D0000D0AC9E8B1B8B1E0BAC5203A20252E2A17
:10D1E000730000000D0AD6D8C6F4D4ADD2F2203AAE
:10D1F00020252E2A73000000D6D8C6F4D4ADD2F272
:10D200003A25732E0000000000F80708541D002086
:10D21000B1BEB5D86C6F673A2573000034000020AA
:10D220004C000020F8220146F94808F006B810B575
:10D23000F8210BF0CBFABDE81040F822F549F4488C
:10D2400007F058BF7CB50446F34805F019FE2046A8
:10D25000FFF7EDFF5B202070302060703120A07060
:10D26000E070207CFF2809D104F110004021054620
:10D270000BF0ACFAE9A128460BF084F994F85000C1
:10D28000FF2809D104F15000402105460BF09EFA19
:10D29000E4A128460BF076F994F89000FF2809D114
:10D2A00004F19000402105460BF090FADEA12846DB
:10D2B0000BF068F994F8D000FF2809D104F1D000F0
:10D2C000102105460BF082FADBA128460BF05AF933
:10D2D00094F8E000FF2816D0A8B1CE49DA48E03132
:10D2E00001F0FAFC94F8F000FF2817D0B0B1C9495A
:10D2F000D548F03101F0FDFC5D2084F8F7002046B0
:10D30000BDE87C408EE704F1E000102105460BF0FB
:10D310005DFAC9A128460BF035F9E3E70020C4F80F
:10D32000F000A4F8F400009001900A22694641F64A
:10D33000583005F0C4FE694604F1F0000BF022F904
:10D34000DAE701460322C14807F077BF00220280D6
:10D35000827001460322BD4807F0CCBE10B50446DA
:10D360002046FFF7F3FF2046BDE81040E9E72DE92E
:10D37000F04105460F46032640F2492005F06EFCB9
:10D3800004463B464FF40077B1A2394604F126002B
:10D390000AF02AFE002801DDB8420BDD40F29E2291
:10D3A000ACA1B1A005F0F2FC204605F091FC0220F2
:10D3B000BDE8F08128222270642190FBF1F2303226
:10D3C000A27090FBF1F201FB12020A2192FBF1F232
:10D3D0003032E27090FBF1F201FB1200303020712C
:10D3E000A84908786071401CC0B20870392801D97A
:10D3F000302008700422A4A1A01D0BF030FA0121F6
:10D4000004F10A0007F0CBF83B2184F82210B5F8AC
:10D410002310A4F82310262184F8251068784328C7
:10D4200014D072216170032299A120460BF06CF890
:10D4300020460BF0D6F8401C82B22146002006F0B0
:10D4400054F9204605F044FC3046B1E752216170A2
:10D4500003228FA120460BF057F820460BF0C1F8AD
:10D4600082B221468B4805F014FD0028E9D04FF424
:10D470002E7278A188A005F089FCE2E7532070475E
:10D480002DE9F04707463C46A0782179303800EB7B
:10D49000C00202EB001001EB8001E0786FF02F0278
:10D4A000303800EB800002EB40000D18DFF860A17F
:10D4B000F8225849504607F01DFE4FF4807630465A
:10D4C00005F0CCFB8046534B7BA2F03399463146A6
:10D4D00040460AF089FD064694F82300312804D11D
:10D4E000611991F82610242902D030281DD021E09E
:10D4F000102148460BF06AF92A4604F126014846F5
:10D500000BF0ADF9F8224349504607F096FEC6F5F8
:10D51000807108EB06004B466CA20AF065FD5324AF
:10D5200041463846FFF723FF05E0601990F82600D2
:10D53000242806D04924404605F0CAFB2046BDE811
:10D54000F087532441463846FFF711FFF3E72DE9F2
:10D55000F04707463C46A0782179303800EBC002FE
:10D5600002EB001001EB8001E0786FF02F02303801
:10D5700000EB800002EB40000D18DFF894A0F822C9
:10D580002449504607F0B6FD4FF48076304605F04A
:10D5900065FB80461F4B52A2E03399463146404618
:10D5A0000AF022FD064694F82300312804D16119BF
:10D5B00091F82610242902D030281DD021E0102116
:10D5C00048460BF003F92A4604F1260148460BF0C1
:10D5D00046F9F8220F49504607F02FFEC6F5807134
:10D5E00008EB06004B4643A20AF0FEFC53244146DA
:10D5F0003846FFF7BCFE05E0601990F826002428A5
:10D6000005D04924404605F063FB204697E77BE0C0
:10D6100000880108420C00203C0800202F41424DA8
:10D620000000000041424D0053686F7033343437BE
:10D6300039343734390000003132312E352E323151
:10D64000372E323532000000F20100200090010830
:10D650002573000055534552434D445C7573657204
:10D66000636D642E6300000025732C25643A757089
:10D6700044617461427566207370696C6C6F766585
:10D6800072A3A100380000204D41433A0000000081
:10D69000245829003A0D002025732C25643A735430
:10D6A0006370305175657565207370696C6C6F7649
:10D6B0006572A3A1000000002A4745542A20546344
:10D6C00070506F72743A5B25735D21002A53455484
:10D6D0002A20546370506F72743A5B25735D210089
:10D6E0002A4745542A2054637049503A5B25735D9C
:10D6F000210000002A5345542A2054637049503AAF
:10D700005B25735D21000000532441463846FFF736
:10D710002EFE77E72DE9F04707463C46A0782179B1
:10D72000303800EBC00202EB001001EB8001E07822
:10D730006FF02F02303800EB800002EB40000D1834
:10D74000DFF8F4A3F822FB49504607F0D3FC4FF46E
:10D750008076304605F082FA8046F64BF7A2D03349
:10D760009946314640460AF03FFC064694F82300AD
:10D77000312804D1611991F82610242902D03028CB
:10D780001DD021E0102148460BF020F82A4604F174
:10D79000260148460BF063F8F822E649504607F0A8
:10D7A0004CFDC6F5807108EB06004B46E8A20AF076
:10D7B0001BFC532441463846FFF7D9FD05E06019AC
:10D7C00090F82600242805D04924404605F080FA28
:10D7D0002046B4E6532441463846FFF7C8FDF4E737
:10D7E0002DE9F04707463C46A0782179303800EB18
:10D7F000C00202EB001001EB8001E0786FF02F0215
:10D80000303800EB800002EB40000D18DFF828A351
:10D81000F822C849504607F06DFC4FF48076304638
:10D8200005F01CFA8046C34BCEA290339946314690
:10D8300040460AF0D9FB064694F82300312804D16B
:10D84000611991F82610242902D030281DD021E03A
:10D85000402148460AF0BAFF2A4604F1260148460C
:10D860000AF0FDFFF822B349504607F0E6FCC6F582
:10D87000807108EB06004B46C0A20AF0B5FB5324AA
:10D8800041463846FFF773FD05E0601990F8260021
:10D89000242805D04924404605F01AFA20464EE6D1
:10D8A000532441463846FFF762FDF4E72DE9F0477F
:10D8B00007463C46A0782179303800EBC00202EBE5
:10D8C000001001EB8001E0786FF02F02303800EBA0
:10D8D000800002EB40000D18DFF85CA2F8229549A9
:10D8E000504607F007FC4FF48076304605F0B6F955
:10D8F0008046904BA7A250339946314640460AF0E5
:10D9000073FB064694F82300312804D1611991F87D
:10D910002610242902D030281DD021E0402148467D
:10D920000AF054FF2A4604F1260148460AF097FF00
:10D93000F8228049504607F080FCC6F5807108EB5C
:10D9400006004B4699A20AF04FFB53244146384645
:10D95000FFF70DFD05E0601990F82600242805D09A
:10D960004924404605F0B4F92046E8E553244146F1
:10D970003846FFF7FCFCF4E72DE9F04707463C4644
:10D98000A0782179303800EBC00202EB001001EBE7
:10D990008001E0786FF02F02303800EB800002EB5E
:10D9A00040000D18DFF890A1F8226249504607F0B8
:10D9B000A1FB4FF48076304605F050F980465D4B70
:10D9C00080A210339946314640460AF00DFB0646C8
:10D9D00094F82300312804D1611991F826102429E4
:10D9E00002D030281DD021E0402148460AF0EEFE4A
:10D9F0002A4604F1260148460AF031FFF8224D4933
:10DA0000504607F01AFCC6F5807108EB06004B463D
:10DA100072A20AF0E9FA532441463846FFF7A7FC00
:10DA200005E0601990F82600242805D049244046D6
:10DA300005F04EF9204682E5532441463846FFF76B
:10DA400096FCF4E72DE9F84307463C46DFF8E890FA
:10DA5000F8223849484607F04DFB4FF480752846B8
:10DA600005F0FCF806466348804606F08FFDCDF8C9
:10DA70000080DFF8C08060A2294698F80230304666
:10DA80000AF0B2FA054694F82300312804D167A1C0
:10DA9000A01C05F08BFB20B194F82300302821D086
:10DAA00025E094F82600302807D0312805D0322808
:10DAB00003D0332801D050241AE088F80200F8225D
:10DAC0001C49484607F0B9FB98F80230C5F580714B
:10DAD000701957A20AF088FA532431463846FFF7E6
:10DAE00046FC05E051A1A01C05F060FB30B14924C3
:10DAF000304605F0EDF82046BDE8F8835324314662
:10DB00003846FFF734FCF3E72DE9F04707463C467B
:10DB1000DFF82490F8220749484607F0EBFA4FF463
:10DB20008075284605F09AF80646DFF8088098F8D0
:10DB300001308FE0420C0020008801082A4745543C
:10DB40002A2046747049503A5B25735D210000001D
:10DB50002A5345542A2046747049503A5B25735D18
:10DB6000210000002A4745542A20467470506173F2
:10DB700073776F72643A5B25735D21002A534554B5
:10DB80002A2046747050617373776F72643A5B2514
:10DB9000735D21002A4745542A20467470557365E9
:10DBA000726E616D653A5B25735D21002A534554A1
:10DBB0002A20467470557365726E616D653A5B25F7
:10DBC000735D21002A4745542A20467470466F6CC5
:10DBD0006465723A5B25735D210000002A53455449
:10DBE0002A20467470466F6C6465723A5B25735DDB
:10DBF00021000000180800202A4745542A205275A9
:10DC00006E4170704E756D3A5B41505025635D20DA
:10DC1000212020202A4745542A20417070566572E1
:10DC200073696F6E3A5B25735D20210030303100DF
:10DC30002A5345542A2052756E4170704E756D3AC4
:10DC40005B41505025635DD6D8C6F4BAF3C9FAD00B
:10DC5000A721000083A2294630460AF0C5F90546EF
:10DC600094F82300312805D1AFF24001A01C05F043
:10DC70009DFA20B194F8230030281DD022E094F8BA
:10DC80002600302803D0312801D050241BE088F82A
:10DC90000100F8227949484607F0CFFA98F8013098
:10DCA000C5F58071701976A20AF09EF953243146A9
:10DCB0003846FFF75CFB06E0AFF29001A01C05F0D0
:10DCC00075FA28B14924304605F002F8204636E4BA
:10DCD000532431463846FFF74AFBF4E7F0B58DB0E0
:10DCE0000446F82265496B4807F004FA6AA104F17A
:10DCF000260005F05BFA18B149240DB02046F0BDAE
:10DD00004FF40076304604F0A9FF07466448054604
:10DD100006F03CFC5948F030A0F12002A0F1E003ED
:10DD2000CDE90932A0F11001CDE90B105D4A603850
:10DD3000A2F10903CDE905329039CDE90710111F91
:10DD4000A0F18C029038C378CDE9022501930491AB
:10DD5000817800914378544A314638460AF044F9B4
:10DD600039462046FFF703FB5324384604F0B0FF42
:10DD7000C3E770B504464DA104F1260005F016FA7C
:10DD800010B15025284670BD53254AA12046FFF703
:10DD9000EEFA642007F049F800F0B2FF642007F0C3
:10DDA00044F803F0AFFC4CA003F033FA09F048FE4E
:10DDB000E8E710B5044694F824003038112835D22D
:10DDC000DFE800F0090D1115191D2125292D343426
:10DDD0003434343431002046FFF7CBFF27E02046AF
:10DDE000FFF77CFF23E02046FFF78EFE1FE0204672
:10DDF000FFF728FE1BE02046FFF7BEFD17E0204698
:10DE0000FFF754FD13E02046FFF7EAFC0FE0204641
:10DE1000FFF780FC0BE02046FFF799FB07E0204668
:10DE2000FFF72EFB03E0FFF729FB00E04E202E4911
:10DE3000502809D049280DD04E2811D149682046D4
:10DE4000BDE81040FFF793BA89682046BDE810404E
:10DE5000FFF78DBAC9682046BDE81040FFF787BAC2
:10DE600010BD00002A4745542A20496170466C6164
:10DE7000673A5B25635D212000000000420C002012
:10DE80002A5345542A20496170466C61673A5B25E4
:10DE9000635D2100008801084745545F49415000F7
:10DEA00018080020861D0020E8D30208434D445F77
:10DEB000525354002A5345542A20557365722063E7
:10DEC0006F6E74726F6C206465766963652072652D
:10DED0007374617274210000D6D8C6F4C3FCC1EE1D
:10DEE000C8EDD6D8C6F421003800002049490620E4
:10DEF00048707047474907204870704745490520DA
:10DF000048707047434909204870704741490320D1
:10DF1000487070473F490C20487070473D490B20BE
:10DF20004870704710B502F0F1FBAFF20F010C2002
:10DF300006F03DFAAFF223010B2006F038FAAFF2FB
:10DF40003301092006F033FAAFF247010D2006F045
:10DF50002EFAAFF25701072006F029FAAFF26B0153
:10DF60000F2006F024FAAFF27B01BDE81040062036
:10DF700006F01DBA27484278011D0D2A48D2DFE875
:10DF800002F0474747174727372F471F47070F001C
:10DF9000027802EB420201EB8202527802702EE01C
:10DFA000027802EB420201EB82029278027026E0D4
:10DFB000027802EB420201EB8202D27802701EE08C
:10DFC000027802EB420201EB82021279027016E043
:10DFD000027802EB420201EB8202527902700EE0FB
:10DFE000027802EB420201EB82029279027006E0B3
:10DFF000027802EB420201EB8202D2790270002227
:10E000004270007800EB400001EB80008068004720
:10E01000704700004C00002008B5F8A000230090D5
:10E0200003220C21184602F042FD08BD38B51E201F
:10E0300004F014FE04460522F64920460AF00FFCBF
:10E040000122002310211046009402F030FD1E2111
:10E0500020460AF0BBFBEF490A220B3920460AF0A2
:10E06000FEFB002302220C210120009402F01FFD80
:10E070002046BDE8384004F02BBE10B5FFF7D6FFB0
:10E08000BDE81040C8E708B5E3A0012300901A4698
:10E090001021002002F00BFDE2A0002300900222DC
:10E0A0001021184602F003FDE1A000230090032296
:10E0B0001021184602F0FBFC08BD08B5D6A00023CD
:10E0C000009001221021184602F0F1FCD5A000902A
:10E0D000012302221021002002F0E9FCD4A0002339
:10E0E000009003221021184602F0E1FC08BD08B59B
:10E0F000C9A00023009001221021184602F0D7FC8D
:10E10000C8A00023009002221021184602F0CFFC84
:10E11000C7A00090012303221021002002F0C7FCB9
:10E1200008BD08B5BFA000230090012210211846A9
:10E1300002F0BDFCBEA00023009002221021184670
:10E1400002F0B5FCBDA000900123032210210020A5
:10E1500002F0ADFC08BD08B5B5A000230090012277
:10E160001021184602F0A3FCB4A000230090022264
:10E170001021184602F09BFCB3A00090012303225B
:10E180001021002002F093FC08BD08B5B1A00123C6
:10E1900000901A461021002002F089FCB0A0002354
:10E1A000009002221021184602F081FCAFA000234B
:10E1B000009003221021184602F079FC08BD08B532
:10E1C000A4A00023009001221021184602F06FFC49
:10E1D000A3A00090012302221021002002F067FC7E
:10E1E000A2A00023009003221021184602F05FFC39
:10E1F00008BD08B597A00023009001221021184601
:10E2000002F055FC96A0002300900222102118462F
:10E2100002F04DFC95A00090012303221021002064
:10E2200002F045FC08BD08B58DA000230090012236
:10E230001021184602F03BFC8CA000230090022223
:10E240001021184602F033FC8BA00090012303221A
:10E250001021002002F02BFC08BD08B589A0012385
:10E2600000901A461021002002F021FC88A0002313
:10E27000009002221021184602F019FC87A000230A
:10E28000009003221021184602F011FC08BD08B5C9
:10E290007CA00023009001221021184602F007FC08
:10E2A0007BA00090012302221021002002F0FFFB3E
:10E2B0007AA00023009003221021184602F0F7FBF9
:10E2C00008BD08B576A0012300901A461021002051
:10E2D00002F0EDFB75A000230090022210211846E9
:10E2E00002F0E5FB6DA000230090032210211846E8
:10E2F00002F0DDFB08BD08B569A0002300900122F3
:10E300001021184602F0D3FB68A0009001230222DE
:10E310001021002002F0CBFB60A00023009003221C
:10E320001021184602F0C3FB08BD08B562A0012306
:10E3300000901A461021002002F0B9FB61A00023D2
:10E34000009002221021184602F0B1FB61A00023C8
:10E35000009003221021184602F0A9FB08BD08B561
:10E3600055A00023009001221021184602F09FFBC7
:10E3700054A00090012302221021002002F097FBFC
:10E3800054A00023009003221021184602F08FFBB6
:10E3900008BD08B548A000230090012210211846AE
:10E3A00002F085FB47A000230090022210211846AE
:10E3B00002F07DFB47A000900123032210210020E2
:10E3C00002F075FB08BD08B546A0012300901A466F
:10E3D0001021002002F06BFB44A0002300900222D9
:10E3E0001021184602F063FB42A000230090032294
:10E3F0001021184602F05BFB08BD00004D454E554C
:10E4000020202020202020202020202020424143A6
:10E410004B0000002F5D002046545020D0C5CFA2F5
:10E420000000000054435020D0C5CFA200000000DF
:10E43000C9E8B1B8C9FDBCB600000000C9E8B1B870
:10E44000D0C5CFA20000000047505320D0C5CFA2B6
:10E4500000000000B2E9D1AF465450D5CBBAC50098
:10E46000B2E9D1AF465450C3DCC2EB00B2E9D1AF40
:10E470004654502020495000B2E9D1AF465450C212
:10E48000B7BEB600B2E9D1AF544350202049500086
:10E49000B2E9D1AF544350B6CBBFDA002000000040
:10E4A000B2E9D1AFB5B1C7B041505000C1A2BCB4C0
:10E4B000C9FDBCB641505000B2E9D1AF4D4143490E
:10E4C00044000000B2E9D1AF41505020B0E6B1BEE7
:10E4D00000000000B2E9D1AF424F4F54B0E6B1BEE8
:10E4E00000000000BEADCEB3B6C80000BDC7B7BDCA
:10E4F000CFF20000CBD9B6C8D6B5000008B5AFF250
:10E500001C000023009001221021184602F0CFFACF
:10E51000AFF228000090012302221021002002F017
:10E52000C6FAAFF2300000230090032210211846F3
:10E5300002F0BDFA60E708B5AFF258000023009082
:10E5400001221021184602F0B2FAAFF26000002357
:10E55000009002221021184602F0A9FAAFF26C00D6
:10E560000090012303221021002002F0A0FA43E7CB
:10E5700008B5F9A0012300901A461021002002F0EE
:10E5800096FAF8480023009002221021184602F063
:10E590008EFAAFF2F80000230090032210211846F3
:10E5A00002F085FA28E708B5EFA0012300901A468B
:10E5B0001021002002F07BFAEA480023403000904E
:10E5C00002221021184602F072FAE64840380AF09A
:10E5D00008F8102809D9E3480023303800900322B6
:10E5E0001021184602F063FA06E7AFF2501000233C
:10E5F000009003221021184602F059FAFCE608B5F3
:10E60000DCA0012300901A461021002002F04FFAEE
:10E61000D44800238030009002221021184602F0D6
:10E6200046FAD048403809F0DCFF102809D9CD4817
:10E6300000233038009003221021184602F037FAE8
:10E64000DAE6AFF2A810002300900322102118464A
:10E6500002F02DFAD0E638B5C8A0012300901A4682
:10E660001021002002F023FABE4C0023403C02227D
:10E6700010211846009402F01AFA204609F0B1FF62
:10E68000102809D904F11000002300900322102162
:10E69000184602F00CFA38BDAFF2002000230090BB
:10E6A00003221021184602F002FA38BD08B5B6A0C0
:10E6B000012300901A461021002002F0F8F9A94821
:10E6C00000239030009002221021184602F0EFF94A
:10E6D000A448403809F085FF102809D9A148002333
:10E6E0003038009003221021184602F0E0F983E64A
:10E6F000AFF258200023009003221021184602F0A8
:10E70000D6F979E608B5A2A0012300901A46102197
:10E71000002002F0CCF993480023A03000900222A0
:10E720001021184602F0C3F98E48403809F059FF0D
:10E73000102809D98B48002330380090032210217B
:10E74000184602F0B4F957E6AFF2B020002300906B
:10E7500003221021184602F0AAF94DE638B58FA021
:10E76000012300901A461021002002F0A0F9102089
:10E7700004F074FA04467B488CA250381021837848
:10E78000204609F031FC0023022210211846009493
:10E7900002F08DF9AFF2FC2000230090032210213B
:10E7A000184602F084F92046BDE8384004F090BADB
:10E7B00010B56C49312050394870F822804806F075
:10E7C0003CFD80A004F088FA022006F02EFBBDE894
:10E7D000104009F035B938B57FA0012300901A46E2
:10E7E0001021002002F063F9192004F037FA0446E2
:10E7F0000121204605F0D3FE002302220C211846F9
:10E80000009402F054F904F1150000230090032253
:10E810000C21184602F04BF92046BDE8384004F0C0
:10E8200057BA38B56EA0012300901A461021002077
:10E8300002F03DF90C2004F011FA0446204605F0E0
:10E84000A5FE0023022210211846009402F02FF9A1
:10E85000AFF2B8300023009003221021184602F0D6
:10E8600026F92046BDE8384004F032BA08B55FA06A
:10E87000012300901A461021002002F018F93948AF
:10E8800000234C38009002221021184602F00FF9A4
:10E89000AFF2F8300023009003221021184602F056
:10E8A00006F9A9E53EB554A0012300901A461021AF
:10E8B000002002F0FCF8524C207E08B9E07AD8B172
:10E8C00094F825004E494FA21831CDE900210023CC
:10E8D000029003221021184602F0E9F8E07D484931
:10E8E00048A20B31CDE90021002302900222102121
:10E8F000184602F0DCF83EBD44A00023009002223E
:10E900001021184602F0D3F8AFF2704000230090B7
:10E9100003221021184602F0CAF83EBD1CB53FA0E4
:10E92000012300901A461021002002F0C0F834485C
:10E930003CA12C30CDE90010002302221021184602
:10E9400002F0B5F8AFF2AC40002300900322102192
:10E95000184602F0ACF81CBD465450D5CBBAC53AA7
:10E9600000000000920C0020465450C3DCC2EB3A79
:10E97000000000004654502049503A00465450C20E
:10E98000B7BEB63A000000005443502049503A0048
:10E99000544350B6CBBFDA3A00000000B5B1C7B05F
:10E9A000D4CBD0D0415050BAC53A000052756E4118
:10E9B00070704E756D3A5B25635DA1A30000000089
:10E9C00000880108C9FDBCB6C9E8B1B8A3ACBCB4A5
:10E9D000BDABD6D8C6F400004D414349443A0000CF
:10E9E00041505020B0E6B1BEBAC53A00424F4F5434
:10E9F000B0E6B1BEBAC53A00BEADCEB3B6C83A00B5
:10EA00002C2800202573256300000000475053D0B8
:10EA1000C5BAC5C8F52E2E2E00000000BDC7B7BD73
:10EA2000CFF23A00257320B6C80000001CB570A0D4
:10EA3000012300901A461021002002F038F86E4899
:10EA40006EA1CDE90010002302221021184602F029
:10EA50002EF8AFF2B8500023009003221021184680
:10EA600002F025F877E708B5002300901A46102138
:10EA7000184602F01CF8BFE438B5624C2078C10794
:10EA80004FF010000AD000905FA30022022138202E
:10EA900001F0E2FF2068401C206038BDAFF2046343
:10EAA000009000220221382001F0D6FFF2E71CB5C9
:10EAB000044610200022009054A31146104601F095
:10EAC000CBFF554809F002FD00211C2808DB534804
:10EAD0001023CDE900102022084602F0B1FA16E01A
:10EAE00017280ADA4D4810238030CDE900100021A4
:10EAF0002022084602F0A4FA09E0484810234030DA
:10EB0000CDE9001000212022084602F099FA0C20DD
:10EB100000220090234611461A2001F09DFF1AE7BB
:10EB20001CB5044610210022009138A31146402054
:10EB300001F092FF39490022C031CDE900211023B4
:10EB400020220021402002F07BFA0C2100220091BB
:10EB5000234611465A2001F07FFFFCE610B5102035
:10EB600004F07CF804462C4B2DA25B1F102120469C
:10EB700009F03AFA2046FFF7D3FF1021204609F0AA
:10EB800025FE254B28A21021204609F02DFA20460B
:10EB9000FFF78DFF2046BDE8104004F099B870479C
:10EBA00008B50023009001221021184601F07FFFD4
:10EBB000BDE80840022001F06FBF08B500230090B7
:10EBC00002221021012001F072FF15E438B50C4635
:10EBD0000023009001221021184601F068FF002355
:10EBE000022210211846009401F061FF38BD000098
:10EBF000CBD9B6C8D6B53A0052280020257320BD1F
:10EC0000DA000000E80100203A0000002020202067
:10EC10002020202000000000821D002082BC02086D
:10EC200025736D560000000043535125730000000A
:10EC300070B505460C4600230F220A21032006F07A
:10EC40003EF92946032006F01FF900230E220A216F
:10EC5000022006F034F92146BDE87040022006F09B
:10EC600013B910B5032006F08AF9BDE81040022060
:10EC700006F085B910B5032006F090F9BDE8104004
:10EC8000022006F08BB913480168491C0160016835
:10EC9000491C00D10160704710B500230C2264218B
:10ECA000052006F00CF9AFF22101BDE81040052067
:10ECB00006F0EAB810B5052006F061F90549002014
:10ECC000086010BD10B5052006F068F9014800681D
:10ECD00010BD0000EC01002070B504460D46102167
:10ECE000601C09F073FD2946601CBDE8704009F006
:10ECF00049BC10B50446084609F0E8FB608210BD27
:10ED000010B5002003F0DEF9BDE81040012002F04C
:10ED100078BE10B503F000F903280CD1434803F086
:10ED2000D5F904464149032C06D04A8A491C40A023
:10ED300004F02CF8204610BD4A8A491C43A003F079
:10ED4000CBFF204610BD0FB4F8B50646032540F2B0
:10ED5000492003F083FF044608AB00934FF400778B
:10ED6000394604F12600079A09F002F9002801DD6E
:10ED7000B8420BDD82223CA140A004F007F82046F7
:10ED800003F0A6FF0220F8BC5DF814FB28222270D5
:10ED90006670642290FBF2F13031A17090FBF2F1C9
:10EDA00002FB11010A2291FBF2F13031E17090FB7C
:10EDB000F2F102FB1100303020711C49891E0878E5
:10EDC0006071401CC0B20870392801D93020087029
:10EDD000042231A1A01D09F042FD012104F10A0025
:10EDE00005F0DDFB3B2184F822103022022104F1E2
:10EDF000230009F0E3FC262184F82510032228A132
:10EE0000204609F081FB204609F0EBFB82B2214647
:10EE1000244804F03EF820B1A12213A122A003F05F
:10EE2000B5FF204603F054FF2846ACE7F20100206E
:10EE300054435020536572766572C1ACBDD3CAA7E6
:10EE4000B0DC3A25733A256420A3A1005443502036
:10EE5000536572766572C1ACBDD3B3C9B9A63A2504
:10EE6000733A256420A3A100555345525F54435083
:10EE70005C757365725F7463702E630025732C2557
:10EE8000643A757044617461427566207370696C90
:10EE90006C6F766572A3A1004D41433A00000000FB
:10EEA000245829003A0D002025732C25643A735408
:10EEB0006370305175657565207370696C6C6F7621
:10EEC0006572A3A100000000F0B585B001213748AC
:10EED00005F065FB01F0EAFA0746344801F0D0FA84
:10EEE000024633A1384601F0B7F9384601F054F92B
:10EEF000044621462FA003F01DFF2146324803F0AF
:10EF000059FB0446032C0DD03048017821F008014C
:10EF100001702FA002F07DF9384600F0E1F805B04D
:10EF20002046F0BD03F093FB0446032CF4D17B2173
:10EF30002B4809F04BFB00F0ECFD064630000FD0EB
:10EF400028A101F054F9054615B1E86804280FD04E
:10EF5000022427A003F01AFF304600F0C1F8DBE7D7
:10EF600000F072F8014627A003F0B6FE0224F3E792
:10EF700013222848296909F072FC264805F0C2FDD1
:10EF800013222449684609F0A2FB9DF80900401CA1
:10EF90008DF8090020A00088ADF80B00684605F048
:10EFA00051FE1EA0296903F0C5FED5E7FF0700202A
:10EFB0006D616300D3B2BCFED7A2B2E14A534F4E9B
:10EFC000A3BA2573000000000802002035000020CD
:10EFD0004874747020706F7374206572722E000014
:10EFE000E01E002073797354696D653200000000E3
:10EFF0004E6F20226A736F6E5F74696D6522202EDA
:10F0000000000000636A736F6E206572723A2573A8
:10F0100000000000245D0020303100002573CEAADE
:10F02000BBF1C8A1B5BDB5C4B7FECEF1C6F7CAB134
:10F03000BCE42E0010B503F0D7FC03F0D8FC044666
:10F0400003F0D8FC204610BDFE480068704770B53C
:10F0500004460D46002C01D02DB10AE00DB101206F
:10F0600070BD002070BD012070BD207898B1641C77
:10F070006D1C207808F06FFF0646287808F06BFFBB
:10F080008642F2D0207808F066FF0446287808F01F
:10F0900062FF201A70BD002070BD70B50646304674
:10F0A00009F09FFA451C284603F0D8FD041E06D03F
:10F0B0002A463146204609F00AFB204670BD20460C
:10F0C00003F006FE002070BD10B5282003F0C6FD39
:10F0D00004461CB12821204609F09AFB204610BDA9
:10F0E00070B5044619E02568A089C00503D4A0685E
:10F0F00008B1FFF7F5FFA089C00503D4206908B166
:10F1000003F0E6FDA089800503D4206A08B103F06E
:10F11000DFFD204603F0DCFD2C46002CE3D170BD62
:10F120002DE9F34F85B08A4600242546C6490020C4
:10F13000CDE90201002637468346012001909AF866
:10F1400000002D2805D1C1490020CDE902010AF1B6
:10F15000010A9AF80000302801D10AF1010A9AF850
:10F1600000003138082817D89AF8000030380CF021
:10F1700010F9804689460022B54B204629460CF0FE
:10F180006FF942464B460BF057FE04460D461AF8FF
:10F19000010F30380928E7D99AF800002E2827D126
:10F1A0009AF80100302823D3392821D80AF1010A1E
:10F1B0009AF8000030380CF0ECF8804689460022BE
:10F1C000A34B204629460CF04BF942464B460BF028
:10F1D00033FE04460D4600229B4B304639460CF068
:10F1E00065FB06460F461AF8010F30380928DFD9AB
:10F1F0009AF80000652801D045281DD11AF8010FA2
:10F200002B2802D02D2803D010E00AF1010A0DE0CE
:10F210004FF0FF3001900AF1010A07E00BEB8B0180
:10F2200000EB410B0AF1010AABF1300B9AF8000038
:10F23000A0F130010929F1D901980BFB00F00CF085
:10F24000A8F832463B460BF0F7FD02460B4600207D
:10F250007F490BF0B3F806460F46DDE9020122466E
:10F260002B460CF0FDF832463B460CF0F9F804460C
:10F270000D460598C0E90645204629460CF02CF8B5
:10F280000599486105980321C16007B05046BDE863
:10F29000F08F401E40EA600040EAA00040EA2010E3
:10F2A00040EA202040EA2040401C704770B50446E8
:10F2B000002C08D0236833B1A268501861688142DD
:10F2C00003DB981870BD002070BDFFF7E2FF064613
:10F2D000304603F0C3FC054665B1D4E90012284668
:10F2E00009F0F5F9206803F0F3FC66602560A0687A
:10F2F000284470BD206803F0EBFC002060602060B3
:10F3000070BD10B50446002C08D0206830B1A1684B
:10F31000084409F066F9A168084410BD002010BD3A
:10F320002DE9F04707460E46DFF82881D7E9064564
:10F3300000221346204629460BF092FF12D12EB12F
:10F3400002213046FFF7B2FF814603E0022003F0BE
:10F3500085FC8146B9F1000F03D03FA00088A9F8D1
:10F3600000009CE078690CF014F822462B460CF063
:10F370009DFA21F00041002243460CF035F821D8D7
:10F38000364A374B204629460CF02EF81AD8002270
:10F39000344B204629460CF061F913D82EB11521C3
:10F3A0003046FFF783FF814603E0152003F056FC4B
:10F3B0008146B9F1000F72D02BA148467A6908F056
:10F3C000FDFD6CE02EB140213046FFF76FFF814616
:10F3D00003E0402003F042FC8146B9F1000F5ED00B
:10F3E000204629460AF0CEFD22462B460CF05EFA56
:10F3F00021F00041002243460BF0F6FF0ED825F025
:10F4000000412046194A1A4B0BF0EEFF06D2224665
:10F410002B4618A1484608F0D1FD40E0204625F0D3
:10F42000004106460F46154A154B0BF0DDFF06D38B
:10F43000304639460022134B0CF010F929D22246EF
:10F440002B4621E0180200200000F03F0000F0BF32
:10F45000000024400000B03C300000000000C0FF6D
:10F46000FFFFDF410000E0C12564000044F3C2E477
:10F47000E4E9634C252E3066000000008DEDB5A058
:10F48000F7C6B03E65CDCD41F6A1484608F096FDE1
:10F4900005E022462B46F4A1484608F08FFD484679
:10F4A000BDE8F0870178A1F13002092A01D81146A0
:10F4B0000AE0A1F14102052A01D8373904E0A1F19F
:10F4C0006102052A0AD857390A01401C0178A1F1C6
:10F4D0003003092B04D8303A11440EE00020704765
:10F4E000A1F14103052B02D8373A114405E0A1F1FF
:10F4F0006103052B0BD8573A11440A01401C0178CF
:10F50000A1F13003092B04D8303A11440EE0002059
:10F510007047A1F14103052B02D8373A114405E0A9
:10F52000A1F16103052B0AD8573A1144090140782B
:10F53000A0F13002092A04D830390844704700206D
:10F540007047A0F14102052A02D8373908447047B4
:10F55000A0F16102052A02D85739084470470020FB
:10F5600070472DE9F04780460D466C1C0020297835
:10F57000222907D0BD480560002091E7641C5C2A61
:10F5800000D1641C2278222A02D00AB1401CF5D195
:10F59000401C03F063FB0746380004D0681C3C465F
:10F5A0004FF480691AE000207AE75C2903D004F860
:10F5B000011B401C12E0461C3078722825D006DC66
:10F5C000622816D0662818D06E2804D119E0742855
:10F5D0001FD0752821D004F8010B701C0178222956
:10F5E00001D00029E1D100212170017822296AD0BF
:10F5F0006AE0082004F8010BEFE70C2004F8010B87
:10F60000EBE70A2004F8010BE7E70D2004F8010BF3
:10F61000E3E7092004F8010BDFE7701CFFF742FF66
:10F620000546361DA5F55C404845D6D3002DD4D0FF
:10F63000A5F55840484513D270785C28CDD1B078F4
:10F640007528CAD1F01CFFF72DFFB61DA0F55C414F
:10F650004945C2D2C5F3090161F39F2000F5803509
:10F660000421802D01D2012108E0B5F5006F01D2FF
:10F67000022103E0B5F5803F00D203216018012983
:10F680001AD0022911D0032908D0042919D105F074
:10F69000BF0242F0800200F8012DAD0905F0BF0263
:10F6A00042F0800200F8012DAD0905F0BF0242F0E2
:10F6B000800200F8012DAD096D4A525C2A4300F822
:10F6C000012D441889E7401CC8F810700421C8F8BF
:10F6D0000C10E5E62DE9F04705468A460024002196
:10F6E000A9460AE0421E1F2A11D322280FD05C2807
:10F6F0000DD00020014309F1010999F8000000280C
:10F70000F0D18046222721B125B32E4644E00120C6
:10F71000F0E7A9EB0506BAF1000F05D0F11C504641
:10F72000FFF7C4FD044603E0F01C03F097FA04461B
:10F7300074B1277004F101092946484608F022FFF8
:10F7400009F8067009EB060080F801802046A7E65C
:10F750000020A5E6BAF1000F05D003215046FFF7BF
:10F76000A5FD044603E0032003F078FA04462CB11B
:10F7700040A1204608F006FF204691E600208FE6D3
:10F7800049463DA008F0B6FE08B1641C03E0B9F19B
:10F79000200F00D2641D761C96F80090B9F1000F7E
:10F7A00001D0641CECD1BAF1000F05D0E11C504629
:10F7B000FFF77CFD064603E0E01C03F04FFA064627
:10F7C0002EB1304600F8017B4FF05C0925E00020A7
:10F7D00066E61F2907D9222905D05C2903D000F845
:10F7E000011B6D1C19E000F8019B044615F8012B64
:10F7F0000C2A25D006DC082A1ED0092A2CD00A2A79
:10F8000006D121E00D2A23D0222A12D05C2A0CD066
:10F810001BA1204608F0D2FB601D29780029D8D111
:10F82000077080F8018030463AE684F80090601C4A
:10F83000F3E72770601CF0E762202070601CECE7A3
:10F8400066202070601CE8E76E202070601CE4E7F2
:10F8500072202070601CE0E774202070601CDCE7E0
:10F86000006937E7256500002566000018020020C2
:10F8700082BD020822220000225C080C0A0D090049
:10F88000752530347800000000E0401C002804D0CA
:10F890000178002901D02029F7D970472DE9F041DE
:10F8A00007460878FE4E7B2803D031600020BDE873
:10F8B000F0810620F860481CFFF7E6FF054628782F
:10F8C0007D2818D0FFF700FC0446B860A8B1284690
:10F8D000FFF7DAFF01462046FFF743FEFFF7D4FFAC
:10F8E00068B1216921620027276101783A2908D08F
:10F8F00030600020DBE7681CD9E70020D7E7002054
:10F90000D5E7401CFFF7C0FF0146204600F086F80F
:10F91000FFF7BAFF0546280028D1C8E7FFF7D4FB58
:10F92000A8B1206044600446681CFFF7ADFF0146A3
:10F930002046FFF716FEFFF7A7FF50B121692162AD
:10F94000276101783A2906D030600020AFE7002017
:10F95000ADE70020ABE7401CFFF796FF01462046CD
:10F9600000F05CF8FFF790FF054645B128782C2899
:10F97000D4D028787D2804D03560002097E7002077
:10F9800095E7681C93E72DE9F04107460878C44ED7
:10F990005B2802D03160002089E70520F860481C10
:10F9A000FFF772FF044620785D2811D0FFF78CFB2B
:10F9B0000546B86070B12046FFF766FF014628464D
:10F9C00000F02CF8FFF760FF0446200004D016E09A
:10F9D000601C6CE700206AE7002068E7FFF774FB13
:10F9E000B0B1286045600546601CFFF74DFF014639
:10F9F000284600F013F8FFF747FF044654B120787B
:10FA00002C28EBD020785D2806D0346000204EE70B
:10FA100000204CE700204AE7601C48E770B5054627
:10FA20000C46002C20D004229EA1204608F0F8FDB0
:10FA3000E0B105229DA1204608F0F2FDD0B10422DC
:10FA40009CA1204608F0ECFDC0B1207822281AD0F5
:10FA50002D2803D0A0F13001092919D821462846C4
:10FA6000BDE87040FFF75CBB002070BD0220E8607D
:10FA7000201D70BD0020E860601D70BD0120E860A1
:10FA80006861201D70BD21462846BDE8704068E5CC
:10FA90005B2805D07B2808D081480460002070BD19
:10FAA00021462846BDE870406DE721462846BDE85E
:10FAB0007040F3E62DE9F04104460D469046FFF70D
:10FAC00003FB0646764F00203860BEB12046FFF7A4
:10FAD000DBFE01463046FFF7A1FF044684B1B8F1D2
:10FAE000000F12D02046FFF7CFFE0446207860B109
:10FAF0003046FFF7F5FA3C600020D8E60020D6E655
:10FB00003046FFF7EDFA0020D1E605B12C60304613
:10FB1000CDE600221146CDE72DE9F04F85B006462F
:10FB2000894615461C4600200490072002904FF09D
:10FB3000000BB06800270021019101E07F1C0068E4
:10FB40000028FBD137B1002C70D0A76895B34FF0D7
:10FB5000020A32E04CB115B109F1040100E00321C1
:10FB60002046FFF7A3FB024607E015B109F10400A8
:10FB700000E0032003F072F8024662B110467B21D8
:10FB800000F8011B85B10A2100F8011B002109239F
:10FB9000A9F1010906E0002005B0BDE8F08F00F8EA
:10FBA000013B491C4945FADB7D2101700021417070
:10FBB0001046F1E7FFE74FF0010A0AF10101204684
:10FBC000FFF774FB88B17B2100F8011B15B10A21F6
:10FBD00000F8011B4FF0000880F80080A068504436
:10FBE000A060B66809F101096CE00020D4E78DB18E
:10FBF00049462046FFF75AFB10B10021092204E0D4
:10FC00000020C9E700F8012B491C4945FADBA06830
:10FC10004844A0602146306AFFF75CFD2046FFF7AC
:10FC200070FBA0601DB14FF0020A02E06CE04FF0E3
:10FC3000010A51462046FFF739FBA8B13A2100F8E6
:10FC4000011B0DB109210170A0685044A06023463A
:10FC50002A464946304600F026FA2046FFF751FB77
:10FC6000A0601DB1012002E0002095E7002031686E
:10FC700009B1012100E0002100EB010A0AF10101B4
:10FC80002046FFF713FB18B3316811B12C2100F89F
:10FC9000011B15B10A2100F8011B80F800800DE05E
:10FCA000180200206E756C6C0000000066616C73B9
:10FCB000650000007472756500000000A068504483
:10FCC000A0603668002E92D125B109F1010102E051
:10FCD000002061E702212046FFF7E8FA28B15DB174
:10FCE00000270921A9F1010904E0002054E700F8E8
:10FCF000011B7F1C4F45FADB7D21017080F80180DC
:10FD0000206838440490D7E0BC00204602F0A6FFEB
:10FD100080465FEA080016D0204602F09FFF824628
:10FD20005FEA0A0011D02146404608F071FD2146E5
:10FD3000504608F06DFDB46809F101098DB30298D1
:10FD40004844029031E0002026E7404602F0C0FF20
:10FD5000002021E70021206AFFF7BCFC03904AF84D
:10FD60002B0000232A464946204600F09CF95946BC
:10FD70000BF1010B48F82100039999B190B108F0FB
:10FD800030FC0646039808F02CFC311815B109F137
:10FD9000020000E00020014402980844801C029008
:10FDA00002E002E0012001902468002CD2D10198E9
:10FDB00018B9029802F052FF0490049808B9012083
:10FDC00001900198B0B100240AE05AF8240008B16B
:10FDD00002F07EFF58F8240008B102F079FF641C9D
:10FDE000BC42F2DB504602F073FF404602F070FF67
:10FDF0000020D1E604997B200870049C641C15B196
:10FE00000A2004F8010B4FF0000B84F800B0002624
:10FE10003BE03DB10020092102E004F8011B401C39
:10FE20004845FADB5AF8260008F0DBFB00905AF848
:10FE300026102046009A08F04AFC009804443A2014
:10FE400004F8010B15B1092004F8010B58F826102D
:10FE5000204608F097FB58F8260008F0C2FB04443F
:10FE6000781E864202D02C2004F8010B15B10A201E
:10FE700004F8010B84F800B05AF8260002F028FFBD
:10FE800058F8260002F024FF761CBE42C1DB504623
:10FE900002F01EFF404602F01BFF4DB10020092179
:10FEA000A9F1010902E004F8011B401C4845FADBF6
:10FEB0007D20207084F801B004986DE62DE9FF4F95
:10FEC00081B0834690461F464FF000094FF0050A67
:10FED000DBF8080000260025002401E0761C0068FD
:10FEE0000028FBD17EB1002F5FD0BE6801213846CB
:10FEF000FFF7DCF9C8B15B210170B868401CB8603D
:10FF0000DBF808503DE02FB103213846FFF7CEF96A
:10FF1000044603E0032002F0A1FE04461CB1FCA14C
:10FF2000204608F02FFB204636E6002034E60299F2
:10FF30003B464246491C284600F0B5F83846FFF7D4
:10FF4000E0F9B8602868D8B1B8F1000F02D04FF0DE
:10FF5000020901E04FF0010909F101013846FFF7FC
:10FF6000A5F9F0B12C2100F8011BB8F1000F02D067
:10FF7000202100F8011B00210170B8684844B860D6
:10FF80002D680DB1002CD2D002213846FFF78EF932
:10FF900048B15D21017000214170386800EB06090D
:10FFA0007FE00020F8E50020F6E5B000009002F0C8
:10FFB00055FE0746380005D0009908F029FCDBF80B
:10FFC00008B01EE00020E7E5029900234246491CE4
:10FFD000584600F068F829466D1C47F8210068B1C2
:10FFE00008F0FFFA0146B8F1000F01D0012000E04F
:10FFF0000020084482440AF1020A00E00124DBF8F0
:020000040802F0
:1000000000B0BBF1000F01D0002CDDD01CB9504670
:1000100002F024FE8146B9F1000F00D1012474B131
:10002000002405E057F8240008B102F051FE641CDA
:10003000B442F7DB384602F04BFE0020ACE55B2013
:1000400089F800004C464FF0000A04F801AF002583
:100050001EE057F8250008F0C4FA834657F825102B
:100060005A46204608F033FB5C44701E85420AD095
:100070002C2004F8010BB8F1000F02D0202004F866
:10008000010B84F800A057F8250002F021FE6D1C3A
:10009000B542DEDB384602F01BFE5D20207084F89E
:1000A00001A0484678E570B50024002809D083B344
:1000B000057B072D6ED2DFE805F01320062D3237C1
:1000C0003B00002070BD05211846FFF7EFF80446FD
:1000D000002C5FD0AFF23441204608F053FA59E0CB
:1000E00006211846FFF7E2F80446002C52D0AFF282
:1000F0004441204608F046FA4CE005211846FFF737
:10010000D5F8044634B3AFF25441204608F03AFA29
:1001100040E011E01946FFF703F904463AE01946BA
:10012000FFF79EFB044635E0FFF7C8FE044631E0CA
:10013000FFF7F2FC04462DE0037B072B2AD2DFE811
:1001400003F00A1004161B202500AFF2A840FEF7AA
:10015000A4FF04461EE0AFF2AC40FEF79EFF04464B
:1001600018E0AFF2B040FEF798FF044612E000211D
:10017000FFF7D6F804460DE00021FFF771FB0446B7
:1001800008E00023FFF79AFE044603E00023FFF790
:10019000C3FC0446204670BD00230122194682E7B5
:1001A00000231A4619467EE7FEB505460C4616465C
:1001B000204602F053FD00900194002002906B460F
:1001C000324600212846FFF76EFFFEBD8168002001
:1001D00001E0401C09680029FBD17047806801E0FC
:1001E000491E0068002801D00029F9DC704770B56D
:1001F0000D46846800E024682CB12946206AFEF789
:1002000026FF0028F7D1204670BD01604860704786
:1002100070B50546FEF758FF044674B128222946FA
:10022000204608F099FA00202062E16841F48071CC
:10023000E16060602060204670BD002070BD024615
:100240009068002901D010B991607047104610B134
:100250000268002AFAD1D8E770B505460E46144662
:10026000002C0CD0206A08B102F032FD3046FEF7B7
:1002700014FF206221462846BDE87040DFE770BDCC
:1002800070B506460D461446002C10D0A089800596
:1002900003D4206A08B102F01BFD2562E06840F437
:1002A0000070E06021463046BDE87040C7E770BD91
:1002B00010B504460846FFF7ABFF01462046BDE8EF
:1002C0001040BCE770B504460D461046FFF7A0FF8E
:1002D000024629462046BDE87040BDE702469068C8
:1002E00001E00068491E08B10029FADC90B14168BC
:1002F00009B103680B60016809B143684B609168FC
:10030000814201D101689160002101604160704724
:100310005B5D00000020FAE710B5FFF7DFFFBDE8E6
:100320001040FEF7DDBE2DE9F04106460F460025E0
:10033000B46801E06D1C24682CB13946206AFEF7D0
:1003400086FE0028F6D124B129463046BDE8F041AA
:10035000C4E70020BDE8F08110B5FFF7E4FFBDE879
:100360001040FEF7BDBE30B40C461146836801E074
:100370001B68641E0BB1002CFADC4BB10B605A6891
:100380004A60596082689A4204D1816030BC7047EB
:1003900030BC54E748680160F8E730B40346986819
:1003A00001E00068491E08B10029FADC0028EDD000
:1003B000016811604468546001B14A6099688142E3
:1003C00001D19A6001E051680A600021416001603A
:1003D00030BCFEF785BED9E72DE9F04106468846D8
:1003E00017460025B46801E06D1C24682CB1414615
:1003F000206AFEF72CFE0028F6D1002CAAD0404639
:10040000FEF74BFE38623A4629463046BDE8F041D9
:10041000C3E79FE710B5FEF757FE002801D0022181
:10042000C16010BD10B5FEF74FFE002801D00121BC
:10043000C16010BD10B5FEF747FE002801D00021B5
:10044000C16010BD10B50446FEF73EFE002804D082
:100450000CB1012100E00021C16010BD70B504465F
:100460000D46FEF731FE064646B10320F060C6E9B0
:100470000645204629460AF02FFF7061304670BDC0
:1004800070B50546FEF720FE04462CB10420E0605E
:100490002846FEF702FE2061204670BD10B5FEF72B
:1004A00013FE002801D00521C16010BD10B5FEF774
:1004B0000BFE002801D00621C16010BD2DE9F047D8
:1004C000804689460027FFF7E9FF064600240DE035
:1004D00058F824000AF05DFFFFF7C0FF05465CB145
:1004E00029463846FFF791FE2F46641C0EB14C4555
:1004F000EEDB3046BDE8F087B560F5E72DE9F04763
:10050000804689460027FFF7C9FF064600240DE014
:1005100058F824000BF0B4FAFFF7A0FF054654B1D9
:1005200029463846FFF771FE2F46641C0EB14C4534
:10053000EEDB3046DEE7B560F6E72DE9F0478046B2
:1005400089460027FFF7AAFF064600240CE008EBC7
:10055000C40103C9FFF782FF054654B12946384656
:10056000FFF753FE2F46641C0EB14C45EFDB3046BF
:10057000C0E7B560F6E72DE9F047074688464FF03B
:100580000009FFF78BFF064600240BE057F8240014
:10059000FFF776FF054654B129464846FFF735FE7A
:1005A000A946641C0EB14445F0DB3046A2E7B560B5
:1005B000F6E72DE9F04106460F460024002E1DD037
:1005C000FEF782FD054628001AD0F06820F48070FE
:1005D000E86070696861D6E90601C5E9060130691D
:1005E00018B1FEF75AFD286160B1306A18B1FEF704
:1005F00054FD286258B17FB1B66821E00020A9E619
:100600000020A7E62846FEF76BFD0020A2E628465C
:10061000FEF766FD00209DE628469BE60121304658
:10062000FFF7C7FF20B144B120604460044606E0F4
:100630002846FEF755FD00208CE6A8600446366883
:10064000002EEBD1284685E6014626E0202A08D078
:10065000092A08D00D2A08D00A2A08D02F2A08D043
:100660000AE0401C19E0401C17E0401C15E0401C4B
:1006700013E043782F2B03D02F2A06D008E0401C2C
:10068000027852B10A2A08D0F9E743782A2B0BD016
:10069000222A12D001F8012B401C0278002AD5D161
:1006A0000020087033E6401C027822B12A2AFAD1D1
:1006B00042782F2AF7D1801CEFE701F8012B401C6C
:1006C00008E05C2A02D101F8012B401C10F8012B34
:1006D00001F8012B02780AB1222AF2D110F8012B7D
:1006E00001F8012BD9E710220921042003F0EEBD07
:1006F0000921042003F050BE10B5FFF7F9FF4FF4B5
:10070000C87004F092FBBDE81040F1E738B506244C
:100710000C23482219460020009403F0F3FD08231F
:1007200048220B210020009403F0ECFD082348220E
:1007300009210220009403F0E5FD08234822072147
:100740000220009403F0DEFD082348220621022047
:10075000009403F0D7FD082348220F2103200094C2
:1007600003F0D0FD082348220D210320009403F05C
:10077000C9FD48220B21032003F0A8FD48220821CF
:10078000002003F0A3FD48220921022003F09EFD72
:1007900048220821022003F099FD48220E2103205F
:1007A00003F094FDBDE8384048220C21032003F0FB
:1007B0008DBD10220A21042003F088BD0A210420E7
:1007C00003F0EABD10B5FFF7F9FF4FF4C87004F06D
:1007D0002CFBBDE81040F1E710B50A460146114870
:1007E00002F057FB002804D0BDE810400EA002F034
:1007F000CDBA10BD10B504460A4802F041FB0123F2
:100800000C222146002002F03BFEAFF23301BDE88E
:100810001040002002F008BE0A460146002002F007
:1008200064BF0000401100207355736251756575F7
:1008300065D2E7B3F6A3A10010B50A4601461148F8
:1008400002F027FB002804D0BDE810400EA002F003
:100850009DBA10BD10B504460A4802F011FB0523ED
:100860000C222146042002F00BFEAFF23301BDE85A
:100870001040042002F0D8BD0A460146042002F0D0
:1008800034BF000046150020735253323332517585
:10089000657565D2E7B3F6A3A100000010B50A465E
:1008A0000146184802F0F5FA002804D0BDE81040CF
:1008B00015A002F06BBA10BD10B50446102200213D
:1008C000032003F003FD154B00221A600D4802F0CF
:1008D000D7FA05230C222146032002F0D1FDAFF206
:1008E0004301BDE81040032002F09EBD10B50A464A
:1008F0000A4C012121600146032002F0F6FE00208F
:10090000206010BD4C190020735253343835517596
:10091000657565D2E7B3F6A3A1000000808122428D
:100920000320401EC0B2FCD27047F0B5034600253C
:1009300000260127FE4C01290CD00022C4F8986142
:10094000C4F89061C4F894613AB118060DD5C4F8A2
:100950009C610CE0C4F89871F2E7180602D5C4F85F
:100960009C7104E0C4F89C6101E0C4F89C71C4F877
:100970009471FFF7D5FF5806030E6D1CEDB2082DDC
:10098000E0D3C4F89071C4F89871F0BD10B5044676
:10099000B031C8B200221146FFF7C7FFA41CC4F350
:1009A0000310002240F010001146FFF7BEFF04F0D4
:1009B0000F000022BDE810401146B6E72DE9F041D6
:1009C000804606980E461F4600242038C5B2B8F16E
:1009D0007F0F02D9A046B61CF6B20C2A06D0102A08
:1009E00019D0BDE8F041D3A002F0D0B9761CF1B225
:1009F0004046FFF7CBFFD44905EB450001EB40052E
:100A00003A46285D0121FFF790FF641CE4B2062CF2
:100A1000F6D3BDE8F08131464046FFF7B7FFCB483B
:100A200000EB05153A46285D0121FFF77EFF641CA7
:100A3000E4B2082CF6D3761CF1B24046FFF7A6FFCD
:100A4000002428193A46007A0121FFF76EFF641C42
:100A5000E4B2082CF5D3DCE72DE9F8430446DDF8D1
:100A600020800E4691461F46002510E000904B4620
:100A7000424631462046FFF7A1FF04EB5800C4B2BE
:100A8000782C02D90024761CF6B26D1CEDB2785D8C
:100A90000028EBD1BDE8F88308B51021400600918D
:100AA000010E0022AAA31046FFF7D6FF08BD0FB41F
:100AB0002DE9FE4F0C46934600254FEA540880204E
:100AC000B0FBF8F64FEA4B07102C1BD00420029025
:100AD0000DF14409CDF80490701C02F0BFF8824675
:100AE0004B46711C5046109A07F042FA8146B145B8
:100AF0000BD90AEB060010F8010C7F2805D9A6F1E6
:100B0000010905E04A200290E2E7B14500D9B1466B
:100B10000C98012802D002280AD105E0A6EB0900B2
:100B2000400808FB00F503E0A6EB090008FB00F510
:100B3000B9F1000F7CDD5846FFF7AEFF00268BE0D1
:100B40001AF806107F2909D80091F9B2E8B22246B6
:100B50000F9BFFF733FF05EB54057CE0002077E0A7
:100B6000102C02D00C2C38D071E0C0EBC00202EB8C
:100B700082037C4A03EB020898F82020914266D158
:100B80000AEB060298F8213052789A425FD1F9B206
:100B9000E8B2FFF7FBFE4FF0000B07E018F80B0080
:100BA00001210F9AFFF7C1FE0BF1010BA345F5D30D
:100BB000781CC1B2E8B2FFF7E9FEA34607E018F8D7
:100BC0000B0001210F9AFFF7B0FE0BF1010BBBEBFD
:100BD000440FF4D32544761C3DE000EBC00202EB49
:100BE0004203604A6C3A03EB020898F818209142DD
:100BF0002DD10AEB060298F8193052789A4226D184
:100C0000F9B2E8B2FFF7C2FE4FF0000B07E018F8A8
:100C10000B0001210F9AFFF788FE0BF1010BA34592
:100C2000F5D3781CC1B2E8B2FFF7B0FEA34608E0E6
:100C300016E018F80B0001210F9AFFF776FE0BF172
:100C4000010BBBEB440FF4D32544761C03E0401C9E
:100C5000029A904284D3761C4E45FFF471AF08E0AF
:100C600007D0B12240A146A007F09CF935A007F0BB
:100C700099F95046BDE8FE0F5DF814EB02F028B874
:100C800030B5002505F1B0000022C0B21146FFF7D3
:100C90004CFE002211460220FFF747FE00221146BB
:100CA0001020FFF742FE0024002201211046FFF72A
:100CB0003CFE641CE4B2802CF6D36D1CEDB2082D12
:100CC000E0D330BD38B510220421002003F0FEFA35
:100CD00010220521002003F0F9FA1022062100203D
:100CE00003F0F4FA10220721002003F0EFFA10229B
:100CF0000521022003F0EAFA254C01252560642035
:100D000004F093F800202060642004F08EF8256041
:100D100000221146AE20FFF708FE002211460220F5
:100D2000FFF703FE002211461020FFF7FEFD31E021
:100D3000000021424E6F2020434841524849474815
:100D40005F65202E0000000013C802083BCA02089D
:100D50002020202020202020202020202020202093
:100D600000000000F5BD02082E2E5C484152445799
:100D70004152455C4F4C45445C6F6C65642E63008A
:100D80004C6F674572723A2025732C256400000071
:100D900094012242002211464020FFF7C6FD0022A6
:100DA00011468120FFF7C1FD00221146FF20FFF709
:100DB000BCFD00221146A120FFF7B7FD002211461D
:100DC000C820FFF7B2FD00221146A620FFF7ADFDB7
:100DD00000221146A820FFF7A8FD002211463F205F
:100DE000FFF7A3FD00221146D320FFF79EFD00224E
:100DF00011461046FFF799FD00221146D520FFF756
:100E000094FD002211468020FFF78FFD002211463D
:100E1000D920FFF78AFD00221146F120FFF785FD5A
:100E200000221146DA20FFF780FD00221146122031
:100E3000FFF77BFD00221146DB20FFF776FD002245
:100E400011464020FFF771FD002211462020FFF7D8
:100E50006CFD002211460220FFF767FD00221146BB
:100E60008D20FFF762FD002211461420FFF75DFD83
:100E700000221146A420FFF758FD00221146A620AB
:100E8000FFF753FD00221146AF20FFF74EFD002271
:100E90001146AF20FFF749FDFFF7F2FE002108469B
:100EA000FFF774FD9AA0002300901A46102101203C
:100EB000FFF7FDFD38BD00B5002211468D20FFF77C
:100EC00034FD002211461420FFF72FFD00221146A9
:100ED000AF205DF804EB28E500B5002211468D2017
:100EE000FFF723FD002211461020FFF71EFD002210
:100EF0001146AE205DF804EB17E52DE9FF5F804653
:100F00000E9D8B461F46002459464046FFF73EFD86
:100F10000BF101090C2D08D0102D4DD0AFF2EC10C3
:100F200004B0BDE8F05F01F031BFDFF8F0A13CE0B4
:100F30006C221B2300203D1932E000EBC00606EBBB
:100F400046065644395D96F818C0614527D1697840
:100F500096F819C0614522D159464046FFF716FD63
:100F600000250121705D029AFFF7DFFC6D1CEDB2D8
:100F70000C2DF6D309F0FF014046FFF707FD0C25C5
:100F80000121705D029AFFF7D0FC6D1CEDB2182DA7
:100F9000F6D308F10C0808F0FF08641C04E0401CBC
:100FA00092FBF3F18142C8D8641C384607F019FB64
:100FB000A042BDD8BDE8FF9FDFF860A10AF16C0A2E
:100FC00038E000203A5D3B19C0EBC00101EB810124
:100FD00001EB0A0696F820108A4227D1597896F834
:100FE0002150A94222D159464046FFF7CFFC0025A7
:100FF0000121705D029AFFF798FC6D1CEDB2102D77
:10100000F6D309F0FF014046FFF7C0FC102501218F
:10101000705D029AFFF789FC6D1CEDB2202DF6D3AE
:1010200008F1100808F0FF08641C02E0401C4A2880
:10103000CAD3641C384607F0D4FAA042C1D8B9E735
:101040002DE9F04F8146DDE909BA0E460025580723
:1010500005D0012000EBD30702EB090815E0DF08FB
:10106000FAE731464846FFF791FC4C4609E028462E
:101070006D1C1AF800005A460121FFF756FC641C4B
:10108000E4B2A045F3D8761CF6B2BE42E9D3BDE87F
:10109000F08F10B586B00121080304F0A4FD0422EE
:1010A0000621002003F012F918220521002003F088
:1010B0000DF918220721002003F008F9102204215D
:1010C000002003F003F90020ADF804004FF4827112
:1010D000ADF80610ADF80800ADF80A00ADF80C0048
:1010E0004FF40071ADF80E100821ADF81010ADF8F6
:1010F00012000720ADF81400094C01A9204606F0A3
:1011000093FD0121204606F014FE06B010BD00003C
:10111000EACC20B3CF20BFC620BCBC0089BD0208EA
:101120000030014010B57E4C204606F05DF92046A7
:10113000BDE8104014227B4904F07FB870B506F07A
:101140001AF90024784D05EBC42006F04DF9641C13
:10115000E4B2002CF7D0734800214160C160FFF772
:10116000E1FFBDE8704006F012B92DE9F0410546F7
:101170000E464FF40067384601F070FD8046C6F316
:10118000CF240BE03A464146284603F0B3FF3A46E7
:101190004146002002F0A9FA05F50065641EA4B2DC
:1011A000F0D23946404607F011FBC6F30A04224646
:1011B0004146284603F09EFF22464146002002F0A9
:1011C00094FA4046BDE8F04101F082BD70B51422AA
:1011D0005449534803F08EFF524C4FF050300025D5
:1011E0002268011182420ED122698A420BD12189E3
:1011F0004EA001F071FD4C486168FFF7B6FF2581F4
:10120000BDE870408EE7206021612581BDE8704017
:1012100094E72DE9F84F0546284607F0E2F9002843
:101220007BD0284607F0DDF914301FFA80F84046DD
:1012300001F014FD074600260024464B46A2414615
:101240003846009506F0D0FE80B200F0010101EBB7
:10125000500506F090F8352006F0B1FA10E00A20AB
:1012600003F0E3FD0A2C09D93EA001F08FFD06F042
:1012700082F83846BDE8F84F01F02ABD641CA4B2DC
:10128000012006F08DFA0128E9D0DFF89890DFF808
:1012900098A031E0202006F092FA701C81B2B85D6F
:1012A00008B940F02D004A1C795C96B240EA01244E
:1012B000200A01D144F43454D9F80400C8F500617F
:1012C000884207D30020C9F80400B9F80800401C80
:1012D000A9F80800D9F804005044410501D106F0EE
:1012E00083F8D9F804002146504406F04DF9D9F8A6
:1012F0000400801CC9F804006D1EADB2CAD2FFF70D
:1013000011FF06F044F81CA0D9F8041001F0E4FC29
:101310003846BDE8F84F01F0DBBCBDE8F88F0000AF
:1013200000F00708541D002000F80708B1BEB5D82A
:10133000C8D5D6BEB4E6B4A2D2E7B3F6A3BA256444
:10134000B4CE202E0D0AB1BEB5D8C8D5D6BE3A202F
:10135000000000002F5D00202A25732025732A201D
:1013600000000000D0B4466C617368C3A6B5C8B471
:10137000FDB3ACCAB1A3A100466C617368C6ABD221
:10138000C6B3A4B6C83A252378000000072813D2B4
:10139000DFE800F00406080A0C0E1000E3A0704716
:1013A000E4A07047E6A07047E8A07047EAA0704745
:1013B000ECA07047EEA07047F1A070474FF4A07109
:1013C000F24807F003BA4FF4A071F14807F0FEB9F4
:1013D00070B505460C46EF480078002806D0224636
:1013E0002946BDE87040EA4807F08EB8EAA12846D1
:1013F00001F0DCFE002821DBE9A1284601F0D6FE41
:1014000000280DDB22462946E94801F042FD00286C
:1014100030D0BDE870407122E6A1EFA001F0B6BC6B
:1014200022462946F34801F034FD002822D0BDE8C9
:1014300070407822DFA1F0A001F0A8BCD34807F0EB
:10144000D0F8C0F5A070A04205D92946BDE870408B
:10145000CE4807F030B98422D6A1EEA001F096FC68
:10146000FFF7ACFF2946BDE870404FF4A072C748B3
:1014700007F0F5B970BD0FB42DE9F84F82464FF073
:101480000408C448CAEBCA01001D00EB8104667E53
:1014900060680B904FF4A165284601F0DFFB83469E
:1014A0000CAB0093294658460B9A06F061FD07469F
:1014B0004FF00009002F01DDAF423EDDB622BDA195
:1014C000DBA001F063FC584601F002FC0220BDE8FD
:1014D000F80F5DF814FBFFF771FF0025BAB259460B
:1014E000022002F002F916E0642003F09EFCE1689D
:1014F000A64801F05BFE20612069002802DB4FF066
:1015000003081DE06169A14801F050FE002802DBDC
:101510004FF0020814E028466D1C2189EDB2884284
:10152000E2D3607E801B00EBC00101EB00104FF4A2
:10153000FA7101EB800003F078FC761EF6B2CAD295
:10154000584601F0C5FBCDF80090B8F1050F0ED25A
:10155000DFE808F0030507090B00BCA408E0BEA4FF
:1015600006E0C0A404E0C1A402E0C2A400E0C3A459
:101570005046FFF70BFF01462246C3A001F0DAFBFD
:101580004046A4E770B50446002020602071002189
:101590000620FFF770FF0546032D05D0BCA12046AD
:1015A00006F0F0FF284670BD2C21784807F00EF8B1
:1015B000411C04230D22204601F01BFDF2E770B50B
:1015C00005461521284607F001F900210520FFF7FF
:1015D00052FF0446032C09D10D216C4806F08AFF06
:1015E000811C14230D22284601F003FD204670BD06
:1015F00010B500210220FFF73EFF032808D000218C
:101600000320FFF738FF0021BDE81040022032E739
:1016100010BD002101202EE79F490120086070477E
:1016200070B500240425FFF7F7FFFFF7C7FE4FF45E
:101630007A7610E0641CE4B2304603F0F6FB97A122
:10164000524801F0B3FD002805DB214694A001F0CB
:1016500071FB032501E0142CECD3284670BD8E49A4
:101660000020086040F6B83003F0DFBB10B5102250
:101670000F21042002F02AFEFFF7F1FF10220B21B8
:10168000042002F023FE844900201039086010BDB8
:1016900010B501230C224FF4E131022001F0F0FEDD
:1016A000FFF78CFEFFF78FFE414801F0E9FB514840
:1016B00001F0E6FBAFF2E721BDE81040022001F0A7
:1016C000B3BE70B5FFF7E4FFFFF7D0FFFFF7A8FF49
:1016D000FFF79FFFFFF78CFF04462C483838FFF7D1
:1016E0006EFF2A4A1421383A73A001F0F5FA274810
:1016F00023380546FFF746FF294674A001F0ECFAAF
:10170000204670BD10B500210846FFF7B4FE044620
:10171000032C02D073A001F039FB4FF47A7003F070
:1017200084FBFFF79CFF204610BD00005455524E2D
:101730004F46460048414E445348414B4500000047
:101740005155455259434F4E46494700434C4F531C
:101750004545434F0000000053415645434F4E4618
:1017600049470000515545525952454C4553450093
:101770005155455259564F4C5441474500000000C1
:10178000CEDEB4CBC3FCC1EE00000000A01D0020E3
:10179000E01E00201C0200202B51495552433A0004
:1017A0002B51495552433A2022726563762200003C
:1017B000202000202E2E5C48415244574152455C67
:1017C0004C54455C454332305C656332306D6F6428
:1017D000756C652E6300000025732C25643A7354E4
:1017E00063705175657565207370696C6C6F766593
:1017F00072A3A1002624002025732C25643A73557A
:1018000072635175657565207370696C6C6F766570
:1018100072A3A10025732C25643A656332304174AC
:10182000427566207370696C6C6F7665722E20004D
:1018300025732C25643A636D645061636B2073706B
:10184000696C6C6F766572A3A1000000496E5061EF
:1018500072616D45727200004F7574506172616DF6
:101860004572720052554E455252000052554E4F2D
:101870004B00000054494D454F555400CEB4D6AAF4
:10188000B4EDCEF3000000002573202573000000A6
:101890003335303000000000BC012342524459006F
:1018A0004543323020537461727420576169746506
:1018B000643A2564205300004543323020C8EDBC13
:1018C000FEB0E6B1BEA3BA252E2A730045433230DE
:1018D00020B9A9B5E7B5E7D1B9A3BA2573206D56EC
:1018E000000000004543323020C8EDB9D8BBFACA29
:1018F000A7B0DCA3ACBCB4BDABB6CFB5E7B9D8BB21
:10190000FAA3A1000FB42DE9F84F81460427F3484C
:10191000C9EBC90100EB8104667E60680B908020F2
:1019200001F09CF982460CAB0093802150460B9A43
:1019300006F01EFB8046B8F1000F02DDB8F1800F03
:101940002FDD6522E6A1EEA001F020FA02272BE0B0
:10195000FFF734FD00251FFA88F25146022001F0FE
:10196000C4FE14E0642003F060FAE168EB4801F083
:101970001DFC20612069002801DB032714E0616958
:10198000E64801F013FC002801DB02270CE02846A2
:101990006D1C2189EDB28842E4D34FF47A7003F0D4
:1019A00044FA761EF6B2D3D2504601F091F90020E7
:1019B0000090052F0ED2DFE807F0030507090B00A2
:1019C000D7A408E0D9A406E0DBA404E0DCA402E08C
:1019D000DDA400E0DEA4484600F05AF901462246A4
:1019E000DEA001F0A7F93846BDE8F80F5DF814FB5A
:1019F00002460021DBA3072084E7024600210820DD
:101A000080E70246002109207CE72DE9F0410446E9
:101A10000F46224600210A20FFF774FF0646032ED8
:101A200020D1AE4D012C20D0022C25D0032C2AD061
:101A3000CEA1BA4801F0BAFBC5F82801D5F82801B3
:101A400000280EDBD5F82811B44830340830085C83
:101A5000A04206D1D5F82811B0480A30085C3128D8
:101A600018D002263046BDE8F081C0A1AB4801F095
:101A70009DFBC5F82801E1E7BFA1A84801F096FB4E
:101A8000C5F82801DAE7BFA1A44801F08FFBC5F82B
:101A90002801D3E7D5F82811A04810230F300144BE
:101AA0002222384601F0A5FADCE72DE9F0410425B1
:101AB0002D2400210120FFF725FF984E874F09367E
:101AC0004FF4FA6815E0404603F0AFF90021022018
:101AD000FFF718FF0546032D0BD1B86C002807DD72
:101AE000B86C805D312807D0B86C805D352803D094
:101AF0000225641E601CE6D12846B4E72DE9F041BA
:101B000004251E2400210320FFF7FCFE834E734FA3
:101B10000A364FF4FA6818E0404603F086F90021CF
:101B20000420FFF7EFFE0546032D0ED1D7F8800005
:101B3000002809DDD7F88000805D312808D0D7F86B
:101B40008000805D352803D00225641E601CE3D12F
:101B5000284688E770B505461921284606F036FE66
:101B600000210846FFF7CEFE0446032C09D15B484E
:101B700001696A481923083001440D22284601F002
:101B800038FA204670BD10B500210520FFF7BAFED7
:101B9000032801D07EA010BD504C9C3420685F49C2
:101BA00008440D2106F0A6FC0021017021685B4865
:101BB0000A30084410BD70B5054600202860002199
:101BC0000620FFF79FFE0446032C0AD14348D0F8B5
:101BD000B81052481923801D01442C22284601F0D8
:101BE00008FA204670BD2DE9F04105460E466D48C5
:101BF0000446FFF7AFFF032809D06BA23146284601
:101C000006F0F2F96BA001F0C1F802202BE72246A2
:101C100019216CA001F060F8FFF747FF0446032C80
:101C200009D06DA23146284606F0DEF96DA001F01C
:101C3000ADF8022017E7FFF761FFFFF7A4FF0146A9
:101C40006EA001F049F85748001F0746FFF7B3FFA1
:101C50003B466EA23146284606F0C6F93A460321B5
:101C60006DA001F039F82046FDE670B505460E4638
:101C70002846FFF7BDFE2846FFF7BFFE0446032CAB
:101C800003D131462846FFF7C0FE204670BDB8E6B6
:101C900010B50B281DD2DFE800F006080A0C0E1064
:101CA000121416181A0060A010BD62A010BD63A027
:101CB00010BD64A010BD65A010BD66A010BD69A0D8
:101CC00010BD6BA010BD6DA010BD6FA010BD72A0A7
:101CD00010BD75A001F05AF879A010BDE4020020F3
:101CE0002E2E5C48415244574152455C4C54455C51
:101CF000454332305C656332306E65742E6300009C
:101D000025732C25643A636D645061636B20737096
:101D1000696C6C6F766572A3A1000000A01D0020A5
:101D2000496E506172616D45727200004F7574505A
:101D30006172616D4572720052554E4552520000FB
:101D400052554E4F4B00000054494D454F555400DD
:101D5000CEB4D6AAB4EDCEF3000000002573202542
:101D600073000000434D494F540000002B5149417E
:101D700043543A20310000002B51494143543A204A
:101D8000320000002B51494143543A2033000000F7
:101D9000BBF1C8A1CDF8C2E7D0C5CFA2CAA7B0DCBD
:101DA00021000000861D0020C7EBB2E5C8EB5349B7
:101DB0004DBFA800CEB4BCECB2E2B5BD53494DBF97
:101DC000A800000053696DBFA84943434944A3BA22
:101DD000252E2A730000000053494DBFA8C7B7B78E
:101DE000D100000053494DC7B7B7D1CEDEB7A8D751
:101DF000A2B2E1C9CFCDF8C2E7000000CDF8C2E73A
:101E0000D0C5CFA2A3BA257300000000D0C5BAC5C3
:101E1000D6CAC1BF3A2573004C544520435351A341
:101E2000BA252E2A730000005155455259494343A3
:101E30004944000053455443530000005155455256
:101E400059435300534554505300000051554552D7
:101E50005950530051554552594E4554494E464FDD
:101E600000000000515545525943535100000000F5
:101E7000434F46434F4E544558540000414354434A
:101E80004F4E5445585400004445414354434F4E2F
:101E900054455854000000005155455259434F4E87
:101EA00054455854000000004543323020CEDED067
:101EB000A7654E6574436D644E756D21000000008A
:101EC000CEDEB4CBC3FCC1EE0000000005280ED26C
:101ED000DFE800F0030507090B00D7A07047D9A081
:101EE0007047DBA07047DCA07047DDA07047DEA024
:101EF000704705280ED2DFE800F0030507090B0044
:101F0000DCA07047DEA07047E0A07047E2A07047F9
:101F1000E4A07047E6A0704770B5102000F09EFE68
:101F2000054629460120FFF770FD032807D0294602
:101F30000120FFF79AFE0446032C02D005E003209F
:101F400070BD2946DDA000F0C7FE284600F0C0FEA7
:101F5000204670BD0FB42DE9F84F81464FF00408BC
:101F6000DA48C9EBC90100EB8104667E60680B901A
:101F7000802000F073FE82460CAB00938021504617
:101F80000B9A05F0F5FF0746002F01DD802F2FDDAE
:101F9000CFA000F0FBFE4FF002082CE0FFF70EFA96
:101FA0000025BAB25146022001F09FFB16E06420E2
:101FB00002F03BFFE168D24801F0F8F820612069A7
:101FC000002802DB4FF0030815E06169CC4801F0FE
:101FD000EDF8002802DB4FF002080CE028466D1CEB
:101FE0002189EDB28842E2D34FF47A7002F01DFFEE
:101FF000761EF6B2D2D2504600F06AFE4046FFF797
:1020000065FF04464846FFF774FF01462246BDA01F
:1020100000F090FE4046BDE8F80F5DF814FB7CB57B
:10202000024600210220FFF795FF0646032E2BD122
:10203000002000900190162000F010FE0446A34DF1
:10204000A96CAF480A30085C2070A96CAC4810231A
:10205000133001442C22601C00F0CBFF601C06F002
:10206000C0FAA96C1430A64A0523114401442C225D
:10207000684600F0BEFF21786B46621CA3A000F00A
:1020800059FE204600F024FE30467CBD1CB50446B7
:10209000CDE900230B46002122460846FFF75AFFF0
:1020A00003280ED189490B69954A303409329A5C6C
:1020B000A24205D10A6992490B31515C302900D006
:1020C00002201CBD02460021012043E770B50446F2
:1020D0002078FFF7F7FF03280CD1A38A628A2078C3
:1020E000611CFFF7D3FF0546032D02D12078FFF7CF
:1020F00096FF284670BD2DE9F84F06468A46914660
:10210000B9F1000F0DD00025A84600240427FFF7E1
:1021100055F932786D4EB16D4B46022001F02EFB21
:102120000DE00320BDE8F88F142002F07EFE3E2172
:10213000734806F0DFF910B14FF0010804E02846BB
:102140006D1CEDB24628EFD3B8F1010F10D0384620
:10215000FFF7BCFE04460320FFF7CBFE01466848AC
:10216000009077A3224679A000F010FE3846D9E708
:102170004A465146022001F0B8FA30E0642002F0ED
:1021800054FEF16F5E4801F011F8C6F88000D6F8F1
:10219000800000280DDB03273846FFF797FE044632
:1021A0000420FFF7A6FE0146224656A000F0C2FD1D
:1021B000DCE7D6F88410524800F0F8FF00280EDB68
:1021C00002273846FFF782FE04460420FFF791FEFF
:1021D00001464B4B224660A000F0D8FDC6E72046E2
:1021E000641CB6F87810A4B28842C7D3BEE770B5B5
:1021F000054605245BA1284600F0D8FF002801DD34
:10220000002416E05CA1284600F0D0FF002801DD84
:1022100004240EE05DA1284600F0C8FF002801DD7F
:10222000022406E05EA1284600F0C0FF002800DD81
:102230000324204670BD0000496E506172616D45F7
:10224000727200004F7574506172616D4572720058
:1022500052554E455252000052554E4F4B00000011
:1022600054494D454F555400CEB4D6AAB4EDCEF3E3
:10227000000000004F50454E534F434B4554000063
:10228000434C4F5345534F434B45540051554552D2
:1022900059534F434B45540054435053454E4443C8
:1022A0004D44000054435053454E444255460000AF
:1022B000CEDEB4CBC3FCC1EE00000000544350B1ED
:1022C000BEB5D84950A3BA257300000018040020F9
:1022D00054637020636D645061636B20D2E7B3F682
:1022E000A3A12D2DD4F6BCD35443505F434D44508D
:1022F00041434B5F4C454ECAFDD6B5A1A30000003B
:10230000A01D002025732025730000005443502099
:102310004368616E6E616CA3BA256320A1A320B7E8
:10232000FECEF1C6F74950A3BA2573A1A320B7FE8C
:10233000CEF1C6F7B6CBBFDAA3BA25730000000012
:10234000CEB4CAD5B5BD223E22000000257320259B
:102350007320257320257300257320257320257392
:10236000000000002B51495552433A2022636C6F04
:1023700073656422000000002B51495552433A20F6
:102380002270647064656163742200002B514955AA
:1023900052433A2022696E636F6D696E67220000B6
:1023A0002B51495552433A2022696E636F6D696E15
:1023B000672066756C6C220005280ED2DFE800F0FD
:1023C000030507090B00D5A07047D7A07047D9A017
:1023D0007047DAA07047DBA07047DCA0704709287F
:1023E00018D2DFE800F00507090B0D0F11131500D7
:1023F000D9A07047DBA07047DDA07047DFA0704711
:10240000E1A07047E3A07047E4A07047E6A07047E2
:10241000E8A07047EAA070470FB42DE9F84F814655
:102420004FF00408E948C9EBC90100EB8104667E5E
:1024300060680B904FF49675284600F00FFC8246BA
:102440000CAB0093294650460B9A05F091FD0746C8
:10245000002F01DDAF422EDDDDA000F097FC2DE066
:10246000FEF7ACFF0025BAB25146022001F03DF95B
:1024700016E0322002F0D9FCE168E14800F096FE57
:1024800020612069002802DB4FF0030816E0616933
:10249000DB4800F08BFE002802DB4FF002080DE065
:1024A00028466D1C2189EDB2B0EB410FE1D34FF40A
:1024B0007A7002F0BAFC761EF6B2D1D2504600F025
:1024C00007FC4046FFF778FF04464846FFF787FFC2
:1024D00001462246CBA000F02DFC4046BDE8F80F97
:1024E0005DF814FB10B500210846FFF795FF03289F
:1024F00009D100210120FFF78FFF032803D1BDE898
:102500001040002188E710BD70B5102000F0A6FB38
:10251000054629460220FFF778FA032807D0294606
:102520000220FFF7A2FB0446032C02D005E00320A3
:1025300070BD2946B5A000F0CFFB284600F0C8FBCF
:10254000204670BDF8B50446204606F04AF80A3029
:10255000064600F083FB0546B0A3B2A231462846EA
:10256000009405F041FD284606F03BF802460021A4
:102570000420FFF751FF0446032C0BD12A4600210B
:102580000520FFF749FF0446032C03D12946A7A0E5
:1025900000F0A2FB284600F09BFB2046F8BD10B5DA
:1025A0000424FFF79FFF032801D0204610BDBDE89B
:1025B0001040A9E72DE9FF4104460F466068FFF788
:1025C000C1FF4FF49676304600F048FB054638468A
:1025D00006F007F8D4E90131CDE90207CDE900138F
:1025E00031462846226805F0FFFC0246002A01DD3C
:1025F000B24204DD022491A000F0C8FB0CE00021EF
:102600000620FFF709FF0446032C05D12A460021C6
:102610000720FFF701FF0446284600F059FB04B0ED
:102620002046BDE8F081002808D0A0F50070BD3834
:1026300007D0012808D08EA000F04EBB92A000F079
:102640004BBB98A000F048BB9CA000F045BB2DE917
:10265000F04100240426FEF7B6FE9D4F012038709D
:102660005A4DD5F8E40005F0BCFFD5F8E41082B26D
:10267000022001F03AF839E0642002F0D6FB55F868
:10268000EC1F944800F092FD68606868EC3D0028FB
:1026900023DBD5F8F0108F480C30085C302819D0B7
:1026A00055F8F01F8B482A68401C095C64203039BB
:1026B00041438848801C105C2A68303800EB800059
:1026C00001EB40018348C01C105C08440226FFF760
:1026D000AAFF12E000200326F9E7D5F8F4104848D5
:1026E00000F064FD002801DB022606E02046641CA1
:1026F000B5F8E810E4B28842BED300203870304606
:10270000FFF75AFE04460820FFF769FE01462246FD
:102710003CA000F00FFB304683E70000496E50619B
:1027200072616D45727200004F7574506172616D17
:102730004572720052554E455252000052554E4F4E
:102740004B00000054494D454F555400CEB4D6AA15
:10275000B4EDCEF30000000048545450434F4E54A3
:1027600045535400454E5245514845414445520059
:10277000434C4F534554494D45000000424F445986
:10278000545950450000000053455455524C434D98
:10279000440000004854545055524C00504F53547C
:1027A000524551434D440000504F535452455142FD
:1027B0005546000048545450524541440000000022
:1027C000CEDEB4CBC3FCC1EE00000000A4040020A8
:1027D0004874747020636D645061636B20D2E7B3FA
:1027E000F6A3A12D2DD4F6BCD3485454505F434DCD
:1027F000445041434B5F4C454ECAFDD6B5A1A300A2
:10280000A01D00202573202573000000485454505B
:10281000B1BEB5D84950A3BA25730000687474706E
:102820003A2F2F002573257300000000504F53549A
:102830002055524C3A25732E0000000068656164F3
:102840006572426F647942756620D2E7B3F6A3A140
:102850002D2DD4F6BCD3485454505F434D445041C1
:10286000434B5F4C454ECAFDD6B5A1A30000000006
:1028700048545450285329206F746865722065723B
:10288000726F722E0000000048747470204F7065E3
:10289000726174696F6E20737563636573736675B7
:1028A0006C2E00004854545028532920756E6B6ECE
:1028B0006F776E206572726F722E0000485454500C
:1028C0002853292074696D656F75742E000000000F
:1028D0001C020020E01E00200FB42DE9F84F8146B5
:1028E0000427A448C9EBC90100EB8104667E606837
:1028F0000B90802000F0B2F982460CAB009380214F
:1029000050460B9A05F034FB8046B8F1000F02DD0B
:10291000B8F1800F2FDD522297A19FA000F036FA68
:1029200002272BE0FEF74AFD00251FFA88F25146E8
:10293000022000F0DAFE14E0642002F076FAE1688A
:102940009C4800F033FC20612069002801DB03274C
:1029500014E06169974800F029FC002801DB022798
:102960000CE028466D1C2189EDB28842E4D34FF477
:102970007A7002F05AFA761EF6B2D3D2504600F0C0
:10298000A7F900200090052F0ED2DFE807F003051D
:1029900007090B0088A408E08AA406E08CA404E0E0
:1029A0008DA402E08EA400E08FA4B9F1050F0ED231
:1029B000DFE809F0030507090B008EA10BE090A1E9
:1029C00009E090A107E092A105E094A103E096A0A0
:1029D00000F0DCF99AA122469CA000F0ABF9384641
:1029E000BDE8F80F5DF814FB0021084674E70021EC
:1029F000012071E7002102206EE7002104206BE72F
:102A000070B5044600210320FFF766FF0546392113
:102A1000204605F0DBFE032D1DD15648406E65496A
:102A200008448CA105F060FD8AA1002005F05CFD42
:102A300001460A22204605F012FF86A1002005F07B
:102A400053FD0146012204F10A0005F008FFA07AB7
:102A5000412802D00425284670BD7EA1002005F043
:102A600043FD01460C2204F10B0005F0F8FE79A1AC
:102A7000002005F039FD0146012204F1170005F0A0
:102A8000EEFE74A1002005F02FFD01460D2204F199
:102A9000180005F0E4FE6FA1002005F025FD0146B9
:102AA000012204F1250005F0DAFE6AA1002005F0FC
:102AB0001BFD0146062204F1260005F0D0FE65A1AB
:102AC000002005F011FD0146062204F12C0005F05E
:102AD000C6FE60A1002005F007FD0146072204F1B3
:102AE000320005F0BCFEB6E770B504460D46022282
:102AF00059A1204605F0B3FE022205F13601A01CC3
:102B000005F0ADFE022205F13401601D05F0A7FEBF
:102B1000022205F1320104F1080005F0A0FE04F1E3
:102B20000B0002222946064605F099FE304605F0C4
:102B3000CDFC08300A2190FBF1F23032E27290FBBA
:102B4000F1F201FB1200303020730222A91C04F1C3
:102B50000E0005F084FE0222291D04F1110005F08B
:102B60007EFE2E20207460732D20E07120712020C5
:102B7000A07270BDA00500202E2E5C484152445723
:102B80004152455C4C54455C454332305C65633290
:102B900030676E73732E630025732C25643A636D62
:102BA000645061636B207370696C6C6F766572A39F
:102BB000A1000000A01D0020496E506172616D45AA
:102BC000727200004F7574506172616D45727200CF
:102BD00052554E455252000052554E4F4B00000088
:102BE00054494D454F555400CEB4D6AAB4EDCEF35A
:102BF000000000004F50454E4E4D45410000000082
:102C000053454C464F50454E474E5353000000002D
:102C10005155455259524D4300000000434C4F530B
:102C200045474E53530000004543323020CEDED09E
:102C3000A765476E7373436D644E756D2100000088
:102C4000CEDEB4CBC3FCC1EE00000000257320250E
:102C5000730000002C0000003230000070B5064602
:102C60003146002000F0AEFB0446002000F017FBC8
:102C700005464B2D08D918225AA161A005F092F9FA
:102C8000294663A005F08EF924B13146204605F0AF
:102C90009DFD1BE0202253A159A005F083F9294690
:102CA00063A005F07FF9002000F0E0FA3146002033
:102CB00000F088FB04464CB925224AA150A005F03B
:102CC00071F968A005F06EF904F0BAFE204670BDF7
:102CD0000146002000F06DBB0FB4F8B507AD0095BC
:102CE0004FF400742046FFF7B9FF06465EA2214666
:102CF000304605F079F90446C4F5007130192B46C9
:102D0000069A05F035F9002806DD204482B23146E6
:102D1000002000F0EAFC07E0502232A138A005F0C4
:102D200041F950A005F03EF93046FFF7D1FFF8BC5D
:102D30005DF814FB0FB4F8B507AD00954FF40074BF
:102D40002046FFF78BFF064649A22146304605F094
:102D50004BF90446C4F5007130192B46069A05F06C
:102D600007F9002806DD204482B23146002000F039
:102D7000BCFC07E06E221BA121A005F013F939A0CD
:102D800005F010F93046FFF7A3FFD0E70FB4F8B510
:102D900007AD00954FF400742046FFF75FFF06462D
:102DA00035A22146304605F01FF90446C4F50071EE
:102DB00030192B46069A05F0DBF8002806DD204482
:102DC00082B23146002000F090FC07E08B2205A182
:102DD0000BA005F0E7F823A005F0E4F83046FFF774
:102DE00077FFA4E72E2E5C53595354454D5C53593D
:102DF00053504F52545C737973706F72742E63002A
:102E00004C6F674572723A2025732C2564000000D0
:102E10000D0AB6AFCCACC4DAB4E6D5BCD3C3D2D1BC
:102E2000B3ACB9FDA3BA25642525A3A10D0A000002
:102E30000D0AC4DAB4E6D5BCD3C3A3BA25642525EC
:102E40002D2DB6AFCCACC4DAB4E6D2E7B3F6A3A16D
:102E5000B3F5CABCBBAFB6AFCCACC4DAB4E6BFD531
:102E6000BCE4A3A1000000004C6F674170703A0001
:102E70004C6F674465623A004C6F674572723A0066
:102E800000210180418081804FF48061801D05F028
:102E90009DBC2DE9F0418388161D33444FF48067B3
:102EA000BB4202D30120BDE8F08145881223841D76
:102EB0002B5543885B1CC3F30903438045883423A7
:102EC0002B5543885B1CC3F30903438000230BE0AD
:102ED00011F8015BB0F802C00CF8045045886D1C75
:102EE000C5F3090545805B1C9342F1DB42885621FE
:102EF00011554188491CC1F309014180428878215C
:102F000011554188491CC1F3090141808188314430
:102F100081808188B94209D3FFF7B2FF4322BFA164
:102F2000C5A005F03FF8C8A005F03CF80020BAE7BE
:102F300070B58388002B08D003889B1CC3F309035A
:102F4000038000231380831D21E0022070BD1488BC
:102F5000641C14800488E45C01F8014B0488641C40
:102F6000C4F30904048014888588AC4203D2048821
:102F7000B4F5806F0BD3FFF783FF6622A7A1AEA045
:102F800005F010F8B0A005F00DF8022070BD04881F
:102F9000E45C562CDBD10488641CC4F309040444AB
:102FA000A479782CD3D10188891CC1F3090101804F
:102FB00081881288891A091F8180002070BD2DE93F
:102FC000F04105460C461746284605F00AFB064622
:102FD000384605F006FB3118A14204DB00212A190E
:102FE000101A00F8011C39462846BDE8F04105F0EA
:102FF00062BB30B5054600205B1E04E02C549842AD
:1030000004DA401C80B20C5C9442F7D130BD70B53C
:103010000446084611461D46049E05F06BFA02461A
:10302000012006E0231803F8011CB04204D8401C1C
:1030300080B2115CA942F5D170BD30B500231144B6
:10304000491E18E00C7824090A2C01D2302500E032
:1030500037252C4400F813400C7804F00F040A2C98
:1030600001D2302500E037252C4400EB43056C707D
:103070005B1C9BB2491E9342E4D330BD30B50023A4
:103080001AE0CD5C2C0905F00F053034392C03D93A
:10309000E41D00F8134001E000F813403035ECB2B5
:1030A000392C04D900EB4305E41D6C7002E000EB01
:1030B00043056C705B1C9BB29342E2D330BDF0B50C
:1030C00003460025084600260A2A01D00670F0BDF6
:1030D000002B1DD005DA4FF02D0200F8012BC3F1B3
:1030E000000342F210724FF00A0793FBF2F454EA25
:1030F000050C06D004F1300500F8015B04FB123327
:10310000012592FBF7F2002AEFDC06700846F0BDBD
:103110003022027046700846F0BDF0B50546002327
:10312000002042F210720A26B5FBF2F4E4B254EA2F
:10313000000704D030340746401CC0B2CC55B5FB64
:10314000F2F402FB1455B2FBF6F25B1CDBB2052B6A
:10315000EAD308B9302008700846F0BD2DE9F041E7
:1031600005460C46284605F03CFA80B2002100B125
:1031700021700122002312E0AE5CEF5CBE420CD154
:10318000521C92B25B1C9BB2AE5CEF5CBE4201D0A3
:10319000A35404E0E65CA65401E01BB1E35C824268
:1031A000EAD380E6521C92B2A154F8E72DE9F04729
:1031B00082468946504605F014FA87B2484605F023
:1031C00010FA86B2002500243046FFF747FD8046FE
:1031D00041464846FFF7C2FF0DE01AF8050019F80E
:1031E0000410884204D16D1CADB2641CA4B202E08C
:1031F0006CB118F80440BD4201D2B442EDD3404650
:10320000FFF766FDB44205D3A81BBDE8F0876D1C2F
:10321000ADB2F0E74FF0FF30F7E700002E2E5C5321
:10322000595354454D5C5359534C49425C7379731F
:103230006C69622E630000004C6F674572723A2021
:1032400025732C25640000000000000003E011F845
:10325000013B00F8013B521E531CF8D1704701E0BE
:1032600000F8011B521E531CFAD1704770B504467A
:103270006B486C4E002150F8240006EB8405420098
:103280002869FFF7ECFF66480021103050F8242031
:10329000A868FFF7E4FF01203119087670BD10B56A
:1032A000002200215E4B5F4C53F8203004EB80007D
:1032B00005E0046934F8114004B1521C491C8B42EA
:1032C000F7D864204243B2FBF3F0C0B210BD2DE941
:1032D000F04105460F460024DFF8488108EB050061
:1032E000007E002803D1D8F80010284688474FF008
:1032F000FF32FFB14A4E083656F82500B7FBF0F30F
:10330000B7FBF0F100FB117000B15B1C444850F8B2
:103310002510491E002921DB08EB8507386930F8A4
:1033200011C0BCF1000F08D000249C4213D1002230
:1033300098B20AE01046BDE8F081641CF5E73C69EC
:1033400001EB020C24F81C00521C9A42F7D356F8E9
:1033500025004843EFE7491E0029E0DA1046EAE776
:1033600070B5304A13181B7E002B13D02C4B103332
:1033700053F820308B421AD9294B083353F82030A8
:10338000B1FBF3F102EB8002106930F8113000203C
:10339000002408E011688847012070BD15690E18E7
:1033A00025F81640401C9842F8DB002070BD022032
:1033B00070BD002905D01B4A02EB80029268891A71
:1033C000CEE7704710B504462046FFF780FF411C4A
:1033D00005D0144901EB84018968084410BD002020
:1033E00010BD2DE9F041064688461746394630465D
:1033F000FFF76DFF0446601C0FD00A483A4600EB09
:1034000086054146A8682044FFF720FF4146304624
:10341000FFF7CFFFA86820448DE700208BE700006E
:103420002CD00208D406002010B50C46F24A52F8FF
:103430002030002B09D05222F0A1F6A004F0B2FDFA
:10344000F8A004F0AFFD204610BD42F82040FAE796
:1034500030B40C46E84951F82030002B03D0204608
:1034600030BC1146184730BC704770477047F4496C
:10347000C2B20B689A8009680A885206FCD5704768
:103480002DE9F04387B004460D46164698460121C3
:10349000084602F0A8FBEA4818220F38015D401FD9
:1034A000005D00F013FFE6480422401F015D401F4D
:1034B000005D00F00BFFE348002C7CD050F82400A6
:1034C000012102F09BFB02950025ADF80C50ADF8F0
:1034D0000E50ADF81050ADF81450ADF81260D84E43
:1034E00002A956F8240002F01DFC56F824004FF4FF
:1034F000587102F067FDBDF8120006F114090007CB
:1035000022D5042C20D056F824000122802102F07C
:10351000ABFCCC4F00950195183F59F82410385D4D
:103520001023002200F02BFC06F12400002150F8AB
:103530002420385D00F01CFBAF480121303850F8E2
:103540002420385D00F014FBBDF81200400759D567
:10355000BC481038005D8DF818008DF819808DF882
:103560001A5001208DF81B0006A802F076F856F8D4
:103570002400012240F2244102F05BFC042C3BD0E9
:1035800056F824000122402102F06EFCCDE90058DB
:10359000AC4859F824101430A0F1280550F8242024
:1035A000285D002300F0EBFB05F10A00A64F30F880
:1035B0001410285D00E01AE057F8200004F0D0F95C
:1035C0008D480021203850F82420285D00F0D0FAE2
:1035D00089480121103850F82420285D00F0C8FAED
:1035E000285D012157F8200004F0A3F90AE00068E3
:1035F000012102F0F8FA66E7012240F22551306914
:1036000002F017FC56F82400012102F006FC07B076
:10361000BDE8F0831CB5044689480122802150F89A
:10362000240002F021FC06200021CDE9001084488E
:1036300010231430002250F8241082481838005DFE
:1036400000F09DFB1CBD7CB504467D480122402155
:1036500050F8240002F008FC06200021CDE90010FB
:103660007848784D1430143D50F8242074480023D5
:10367000143050F82410285D00F081FB05F10A0099
:10368000714E30F81410285D56F8200004F068F9E7
:10369000285D012156F82000BDE87C4004F049B9BE
:1036A0002DE9F0410446674D674E143D0021285D29
:1036B00056F8200004F03DF905F10A0705F128004D
:1036C00037F8141050F8240005F080F8285D37F81A
:1036D000141056F8200004F043F9285D012156F833
:1036E0002000BDE8F04104F024B92DE9F04704467C
:1036F00088461646B8F1000F25D0002E23D0042CA2
:1037000023D0504FDFF84091183F0021385D59F821
:10371000200004F00EF94A4D0020183D2855385D70
:1037200059F82000C0F80C80385D314659F8200067
:1037300004F016F9385D012159F8200004F0F9F879
:10374000285D0028FCD0BDE8F08700253C4F4021D3
:10375000386902F030FC0EE018F8051057F8240024
:1037600002F0BCFB57F82400402102F024FC0028A2
:10377000F8D06D1CADB2B542EED3E4E70FB470B52E
:1037800086B004460CA801902D4E10E05C2916D09E
:1037900025295BD0401C0B9056F8240002F09EFBBC
:1037A00056F82400402102F006FC0028F8D00B98BF
:1037B00001780029EAD106B070BC5DF814FB401C0A
:1037C0000B9001786E290DD0722902D0401C0B900D
:1037D000E6E756F824000D2102F080FB0B98401C10
:1037E0000B90DDE756F824000A2102F077FB0B98D6
:1037F000401C0B90D4E70000705700202E2E5C5325
:10380000595354454D5C55534152545C7573617224
:10381000742E63004C6F674572723A2025732C2515
:1038200064000000556172742043616C6C626163D6
:103830006B207265706561742072656721000000FD
:103840000C0700205CD0020844070020401C0B90AD
:10385000017864291BD0732902D0401C0B909FE78C
:10386000019820C801900BE056F8240002F036FBC6
:1038700056F82400402102F09EFB0028F8D06D1C71
:1038800029780029F0D10B98401C0B9088E701980B
:1038900001990068091D01910A2202A9FFF70FFC96
:1038A00002AD0BE056F8240002F018FB56F8240095
:1038B000402102F080FB0028F8D06D1C29780029F7
:1038C000F0D10B98401C0B906AE770B59C4C40F20D
:1038D0002441204602F07AFBA0B19A4D00212869CC
:1038E00004F027F82088201D0088286904F03AF8A1
:1038F000C0F5807082B294490020FFF7A9FD002036
:10390000FFF7CEFE40F225552946204602F05EFB29
:1039100018B12946204602F079FB40F22775294666
:10392000204602F053FB002806D029462046BDE879
:103930007040002202F07DBA70BD70B5834C40F239
:103940002441204602F042FBA0B17E4D002168696F
:1039500003F0EFFF2088201D0088686904F002F85A
:10396000C0F5807082B27A490120FFF771FD012015
:10397000FFF796FE40F225552946204602F026FB29
:1039800018B12946204602F041FB40F2277529462E
:10399000204602F01BFB002806D029462046BDE841
:1039A0007040002202F045BA70BD70B5694C40F21B
:1039B0002441204602F00AFBA0B1624D0021A86814
:1039C00003F0B7FF2088201D0088A86803F0CAFF15
:1039D000C0F5807082B260490220FFF739FD0220F5
:1039E000FFF75EFE40F225552946204602F0EEFA2A
:1039F00018B12946204602F009FB40F227752946F6
:103A0000204602F0E3FA002806D029462046BDE809
:103A10007040002202F00DBA70BD70B54F4C40F2FC
:103A20002441204602F0D2FAA0B1464D0021686A36
:103A300003F07FFF2088201D0088686A03F092FF52
:103A4000C0F5807082B246490320FFF701FD0320D4
:103A5000FFF726FE40F225552946204602F0B6FA29
:103A600018B12946204602F0D1FA40F227752946BE
:103A7000204602F0ABFA20B100222946204602F08F
:103A8000D8F92046BDE87040402102F09BBA2DE9EC
:103A9000F041344D40F22551284602F097FA324C5D
:103AA000002658B1AA882168481C20602F4842543B
:103AB000216846542068FF2800DB266040F2244736
:103AC0003946284602F082FA88B12888A8882068FA
:103AD000264982B20420FFF7BBFC4FF480712348D3
:103AE00004F096FE26603946284602F08FFA40F22E
:103AF00027742146284602F069FA002806D021469C
:103B00002846BDE8F041002202F093B9BDE8F081FB
:103B100015490120091D0870704713490120091D2E
:103B20004870704710490120091D887070470E4980
:103B30000120091DC8707047704770477047704773
:103B40000038014044070020845700200044004012
:103B5000845800200048004084590020004C004058
:103B6000845A002000500040F0060020845B0020B2
:103B700010B5144600290BD0012919D04E22E9A115
:103B8000EDA004F00FFAF0A004F00CFA204610BDEE
:103B9000F64951F8202042B14322E2A1E6A004F008
:103BA00001FAF3A004F0FEF9F0E741F82040EDE758
:103BB000EE49303151F8202042B14A22D9A1DEA08D
:103BC00004F0F0F9F1A004F0EDF9DFE741F820404E
:103BD000DCE730B4E549B0F1007F01F1300271D08B
:103BE00036DCB0F5005F6ED018DC80287AD00ADCB5
:103BF00002286DD0082870D0202868D14868002895
:103C000065D030BC0047B0F5007F71D0B0F5006FD3
:103C10005DD1906800285AD030BC0047B0F5002F25
:103C200077D00ADCB0F5004F6ED0B0F5003F4ED132
:103C3000086900284BD030BC0047B0F5001F6DD09C
:103C4000B0F5000F43D15069002840D030BC004788
:103C5000D54C031BA0427CD01ADCD44CA0EB04034F
:103C6000A0426CD00BDCB0F1006F61D0A0F18050AD
:103C7000801E2CD1C86900287FD030BC0047182B8B
:103C800062D0782B79D1106A002876D030BC0047FA
:103C9000B3F5FC4F67D00ADCB3F5C06F5ED0B3F567
:103CA000F05F6AD1886A002867D030BC0047B3F55E
:103CB000FF3F5DD0BE48C3425FD1D06A00285CD0D0
:103CC00030BC00472FE018E00CE001E005E054E0D4
:103CD0000868002851D030BC0047106800284CD03C
:103CE00030BC00475068002847D030BC0047FFE791
:103CF0008868002841D030BC0047C86800283CD004
:103D000030BC004705E0FFE7D068002835D030BC64
:103D100000471069002830D030BC004748690028AF
:103D20002BD030BC00478869002826D030BC004723
:103D30009069002821D030BC00470AE0FFE7D06935
:103D400000281AD030BC0047086A002815D030BCC3
:103D50000047486A002810D030BC0047506A00284D
:103D60000BD030BC0047906A002806D030BC00471A
:103D7000C86A002801D030BC004730BC70472DE92C
:103D8000F0478CB00446DDE914980D4617469A4674
:103D9000072C04D20121084601F01AFF03E001219B
:103DA000022001F015FF834E56F8240003F020FD99
:103DB00001950297CDF80CA000250495059580206B
:103DC000069007950895CDF8249040010A900B9530
:103DD00056F8240001A903F082FD774810F824006A
:103DE0008DF800008DF801808DF8025001208DF8CB
:103DF0000300684601F031FC56F82400012202213C
:103E000003F0A4FD0CB0BDE8F08710B5022003F06C
:103E1000ACFD012805D1022003F0CFFD0220FFF701
:103E2000D8FE082003F0A1FD01280ED1082003F0E0
:103E3000C4FDD5223BA140A004F0B4F85FA004F07B
:103E4000B1F8BDE810400820C3E610BD10B5202031
:103E500003F08BFD012805D1202003F0AEFD2020CA
:103E6000FFF7B7FE802003F080FD01280ED18020EF
:103E700003F0A3FDEB222BA12FA004F093F852A096
:103E800004F090F8BDE810408020A2E610BD10B507
:103E90004FF40074204603F068FD012805D1204648
:103EA00003F08BFD2046FFF794FE4FF4006420469C
:103EB00003F05BFD01280FD1204603F07EFD40F2A8
:103EC000011218A11CA004F06DF842A004F06AF8D9
:103ED0002046BDE810407CE610BD10B54FF40054FC
:103EE000204603F042FD012805D1204603F065FD80
:103EF0002046FFF76EFE4FF40044204603F035FDE8
:103F0000012874D1204603F058FD40F2171205A194
:103F100009A004F047F832A004F044F82046BDE8B8
:103F2000104056E62E2E5C53595354454D5C444D7B
:103F3000415C646D612E63004C6F674572723A207C
:103F400025732C2564000000446D61546520436195
:103F50006C6C6261636B2022654972715479706583
:103F600022206572726F722100000000845C0020C4
:103F7000446D6154632043616C6C6261636B2072B9
:103F8000657065617420726567210000446D61543D
:103F9000652043616C6C6261636B20726570656162
:103FA00074207265672100000002001008000010F4
:103FB0000002F8FF4407002080D00208444D413140
:103FC0005F54453121000000444D41315F5445327A
:103FD00021000000444D41315F5445332100000071
:103FE000444D41315F54453421000000FFE710BDCE
:103FF00010B54FF40034204603F0B7FC012805D17A
:10400000204603F0DAFC2046FFF7E3FD4FF40024DE
:10401000204603F0AAFC012811D1204603F0CDFC74
:1040200040F22D12AFF20411AFF2F40003F0BAFF28
:104030008AA003F0B7FF2046BDE81040C9E510BDD7
:1040400010B54FF40014204603F08FFC012805D171
:10405000204603F0B2FC2046FFF7BBFD4FF40004FE
:10406000204603F082FC012811D1204603F0A5FC74
:1040700040F24312AFF25411AFF2441003F092FF3A
:1040800079A003F08FFF2046BDE81040A1E510BDE8
:1040900010B54FF00074204603F067FC012805D1ED
:1040A000204603F08AFC2046FFF793FD4FF00064A2
:1040B000204603F05AFC012811D1204603F07DFC74
:1040C00040F25912AFF2A411AFF2941003F06AFF5C
:1040D00068A003F067FF2046BDE8104079E510BDF9
:1040E00010B5674C204603F040FC012805D120465E
:1040F00003F063FC2046FFF76CFD614CA41D2046D5
:1041000003F033FC012811D1204603F056FC40F2A5
:104110006F12AFF2F011AFF2E01003F043FF59A0BD
:1041200003F040FF2046BDE8104052E510BD10B539
:10413000534C1E34204603F018FC012805D12046BC
:1041400003F03BFC2046FFF744FD4D4C7E342046F7
:1041500003F00BFC012811D1204603F02EFC40F2A5
:104160008512AFF24021AFF2302003F01BFF45A0D3
:1041700003F018FF2046BDE810402AE510BD10B539
:10418000434C204603F0F1FB012805D1204603F003
:1041900014FC2046FFF71DFD3E4C204603F0E5FBD6
:1041A000012811D1204603F008FC40F29B12AFF227
:1041B0008C21AFF27C2003F0F5FE37A003F0F2FE75
:1041C0002046BDE8104004E510BD10B5354C204632
:1041D00003F0CBFB012805D1204603F0EEFB20467F
:1041E000FFF7F7FC304C204603F0BFFB012810D14D
:1041F000204603F0E2FB40F2B112AFF2D821AFF259
:10420000C82003F0CFFE29A003F0CCFE2046FFF724
:10421000E0FC294C204603F0A8FB012805D12046EC
:1042200003F0CBFB2046FFF7D4FC244C204603F0E0
:104230009CFB012811D1204603F0BFFB4FF4DF7235
:10424000AFF22031AFF2103003F0ACFE1CA003F04F
:10425000A9FE2046BDE81040BBE410BD444D4131ED
:104260005F54453521000000444D41315F544536CF
:1042700021000000444D41315F54453721000000CA
:1042800002000010444D41325F54453221000000CD
:104290000002001000080010444D41325F544533C5
:1042A000210000000020001000800010444D413229
:1042B0005F54453421000000000002100000081087
:1042C000444D41325F54453521000000F8B50446A5
:1042D0000D4616469848012150F8240001F083FC51
:1042E00095481C3030F81500ADF800008DF80360DB
:1042F00003208DF802009148694650F8240001F02F
:104300006CFAF8BD2DE9FE430646DDF828900C4610
:10431000154698462A4621463046FFF7D7FF282DF6
:1043200001D0482D36D10121084601F05CFC824FB6
:104330008C37385D8DF800008DF8019000258DF8E0
:1043400002508DF80350684601F087F9A7F150003C
:10435000015D4438805D01F0FCFAA7F1400656F893
:10436000240001908DF808508DF8098001258DF802
:104370000A5001A802F09AF856F8240002F0F5F865
:10438000385700F01F018D404009800000F1E02007
:10439000C0F80051BDE8FE83684A52F82000C268A8
:1043A000654B1C3333F811104A40C260704710B59A
:1043B0000C46634A52F82030002B09D0952261A1A7
:1043C00065A003F0EFFD68A003F0ECFD204610BDF2
:1043D00042F82040FAE770B5064600204FF08041D1
:1043E00005F03EFE04460D46304606F0E9FF05F0B6
:1043F00037FE22462B4606F0DBFD06F06DFF5049E6
:1044000051F82000002802D0BDE87040004770BD80
:1044100010B5012002F08EF828B1012002F093F8C7
:104420000120FFF7D8FFBDE81040012002F09DB841
:1044300010B5022002F07EF8012805D1022002F01A
:1044400082F80220FFF7C7FFBDE81040022002F00B
:104450008CB810B5042002F06DF828B1042002F0E9
:1044600072F80420FFF7B7FFBDE81040042002F007
:104470007CB810B5082002F05DF8012805D10820AD
:1044800002F061F80820FFF7A6FFBDE81040082001
:1044900002F06BB810B5102002F04CF828B11020D3
:1044A00002F051F81020FFF796FFBDE810401020F1
:1044B00002F05BB830B591B005241F4D4C3555F86E
:1044C000240002F044F888B155F8240002F03BF8CB
:1044D000402101A804F09CF9234629A2402101A80B
:1044E00003F082FD55F82400FFF775FF641C092CCA
:1044F000E5DD11B030BD30B591B00A240E4D4C351C
:1045000055F8240002F023F888B155F8240002F091
:104510001AF8402101A804F07BF9234618A2402193
:1045200001A803F061FD55F82400FFF754FF641C57
:104530000F2CE5DDDDE70000B8D00208740700208D
:10454000E45C00202E2E5C53595354454D5C494F7A
:104550005C696F2E630000004C6F674572723A20F1
:1045600025732C2564000000494F2043616C6C6268
:1045700061636B20726570656174207265672100EC
:1045800045585449256420495251210000210160B9
:104590004160018181720B2210A104F060B90EB557
:1045A000114A12680092104A121D126801920E4AB6
:1045B00008321268029200290BD0012904D00C2283
:1045C0006946FEF75BFD0EBD0C226946FEF756FDFF
:1045D0000EBD0C22694604F042F90EBD4D617220F9
:1045E0003234203230323100E8F7FF1F10B50C466C
:1045F000F54901280BD0022816D03D22F3A1F8A0DE
:1046000003F0D0FCFAA003F0CDFC204610BD4868B2
:1046100040B13222EDA1F2A003F0C4FCFBA003F0F4
:10462000C1FCF2E74C60F0E7886840B13922E7A1AD
:10463000EBA003F0B7FCFDA003F0B4FCE5E78C6051
:10464000E3E7E149012805D0022807D1886800285E
:1046500004D000474868002800D00047704710B5D4
:10466000012002F042F838B1012002F04CF802F0CB
:104670001DF80120FFF7E5FF022002F036F80028C0
:1046800008D0022002F03FF802F010F8BDE8104018
:104690000220D6E710BD10B5022002F026F800284F
:1046A0000CD04FF4003001F060FF022002F02BF834
:1046B00001F0FCFFBDE810400220C2E710BD30B59C
:1046C0006423B0FBF3F4E4B2B0FBF3F503FB150095
:1046D000132C01D96430C0B200EB90030724B3FB64
:1046E000F4F504FB1533D94D1A440D4415F8015C5B
:1046F0002A4492B2800703D1032901D2521E92B2FA
:10470000B2FBF4F004FB102030BD810701D0002083
:1047100070476421B0FBF1F201FB120109B10120E5
:1047200070474FF4C871B0FBF1F201FB120008B101
:1047300000207047012070472DE9F04788B00446FB
:1047400001F0BAFF01F089FF0646DFF80483B6FBEB
:10475000F8F39D480A270188994279D0038040F2F6
:10476000B2754FF4B7794FF4B67A0FE02846FFF7E9
:10477000CCFF38B14B4502D3A3F5B77304E06D1CF1
:10478000ADB205E0A3F26D136D1CADB25345EDD88B
:104790000195BDF804104FF47A70B1FBF0F130319F
:1047A0002170BDF80410B1FBF0F200FB121264217D
:1047B000B2FBF1F230326270BDF80420B2FBF0F5CA
:1047C00000FB1520B0FBF1F201FB1200B0FBF7F08B
:1047D0003030A070BDF80400B0FBF7F107FB11000A
:1047E0003030E0700025DFF8649209F10C090DE02B
:1047F000BDF80400FFF789FF08B1012D7AD019F840
:104800000500984204D81B1A6D1CADB21C2BEFD2C8
:104810006D1C04955B1C03939DF81000B0FBF7F032
:10482000303060719DF81000B0FBF7F107FB11000C
:104830003030A0719DF80C00B0FBF7F030302072E2
:104840009DF80C00B0FBF7F107FB110030306072EF
:10485000B6FBF8F008FB10604FF46161B0FBF1F2B9
:104860000792B0FBF1F201FB12033C22B3FBF2F31F
:104870000693B0FBF1F301FB1300B0FBF2F102FB76
:10488000110005909DF81C00B0FBF7F03030E0728D
:104890009DF81C00B0FBF7F107FB110030302073CE
:1048A0009DF81800B0FBF7F03030A0739DF81800A9
:1048B000B0FBF7F107FB11003030E0739DF81400F6
:1048C000B0FBF7F0303060749DF81400B0FBF7F1E6
:1048D00007FB11003030A0749DF80C209DF81010DB
:1048E000BDF80400FFF7EBFE029008B00320BDE81E
:1048F000F087FFE71D2B8BD31D3B85E755481BE752
:1049000008B503218DF800108DF8010000208DF806
:10491000020001208DF80300684600F09EFE08BDED
:104920002DE9F041074600244A48202181722D21BB
:10493000C17101713A210174417301214FF0C050DE
:1049400001F05CF90121084601F04DF9012001F068
:1049500021FE042001F078FD45F25006B04232D02D
:1049600001F048FD012001F0C8F801F068FE01F0F7
:104970009DFE6FF07F4500E0641C412001F042F88D
:1049800008B9AC42F8D3DFF8D080444505D24FF4E3
:10499000807001F0C7F8012466E00024012001F0D6
:1049A000BEF800E0641C612001F02CF808B9AC42AC
:1049B000F8D3444570D24FF4007001F0B3F8CA2226
:1049C00002A107A04AE079E0900700202E2E5C5358
:1049D000595354454D5C5254435C7274632E6300CA
:1049E0004C6F674572723A2025732C2564000000D5
:1049F0005274635F526567486F6F6B43616C6C62A2
:104A000061636B204661696C6564210052746320A8
:104A100053656354692043616C6C6261636B2072FF
:104A200065706561742072656721000052746320AF
:104A3000416C7254692043616C6C6261636B2072DB
:104A400065706561742072656721000054D10208A9
:104A500080510100245D0020F0FFFF0003F0A2FA66
:104A6000C9A003F09FFA0024012001F060F801F0D2
:104A70001DFEF4B147F6FF7001F0FFFD01F016FED8
:104A800001F014FE01F0E2FD01F010FE31460420B9
:104A900001F0D2FC18E0FFE7CF22AFF2D001AFF275
:104AA000C00003F07FFAB8A003F07CFA0220BDE852
:104AB000F08149F6404001F0E0FDDFE701F0F6FD4E
:104AC0000121084601F0B0FD01F0F0FD012108468A
:104AD00001F0AAFD01F0EAFD0121022001F0A4FD90
:104AE00001F0E4FD002001F055FD3846FFF708FF16
:104AF000A648FFF721FEAFF2FB110120FFF776FD7C
:104B00000320D4E72DE9F05F00230178C278303923
:104B100001EB4104C4EBC11102EBC10442786421F2
:104B2000303A4A438178303901EB810102EB41018F
:104B3000214430398DB241798279303901EB8104D9
:104B40006FF02F0101EB44042244D7B2027A447A79
:104B5000303A02EB820201EB42022244D6B2C27A20
:104B6000047B303A02EB820201EB4202224402F063
:104B7000FF08827BC47B303A02EB820201EB4202E7
:104B8000224402F0FF09827C407C303800EB800038
:104B900001EB4000104400F0FF0AA5F2B270822839
:104BA00002D30220BDE8F09F40F2B274DFF8E0B11A
:104BB00009E02046FFF7A9FD08B15B4401E0754814
:104BC0000344641CA4B2AC42F3D37F1EFFB20024A2
:104BD000DFF8C4B110E01BF8040040F2A321484301
:104BE00003EBC0132846FFF790FD18B1012C01D14B
:104BF0006A480344641CA4B2BC42ECD3761E40F263
:104C0000A320464303EBC610C8EB4811C1EB0821B3
:104C100000EB0110C9EB091100EB810000EB0A0465
:104C2000012001F0B7FC01F00AFD01F03FFD204634
:104C300001F01CFD01F03AFD01F008FD01F036FD28
:104C40000320AFE72DE9F05F00230178C278303907
:104C500001EB4104C4EBC11102EBC10442786421B1
:104C6000303A4A438178303901EB810102EB41014E
:104C7000214430398DB241798279303901EB810498
:104C80006FF02F0101EB44042244D7B2027A447A38
:104C9000303A02EB820201EB42022244D6B2C27ADF
:104CA000047B303A02EB820201EB4202224402F022
:104CB000FF08827BC47B303A02EB820201EB4202A6
:104CC000224402F0FF09827C407C303800EB8000F7
:104CD00001EB4000104400F0FF0AA5F2B2708228F8
:104CE00001D302205EE740F2B274DFF8A4B009E01D
:104CF0002046FFF70AFD08B15B4401E02548034464
:104D0000641CA4B2AC42F3D37F1EFFB20024DFF8D0
:104D100088B010E01BF8040040F2A321484303EBE5
:104D2000C0132846FFF7F1FC18B1012C01D11B4834
:104D30000344641CA4B2BC42ECD3761E40F2A32010
:104D4000464303EBC610C8EB4811C1EB082100EB4A
:104D50000110C9EB091100EB810000EB0A040120EE
:104D600001F018FC01F06BFC01F0A0FC204601F002
:104D70008CFC01F09BFC01F069FC01F097FC002029
:104D800001F008FC03200DE700000000245D002076
:104D90000085E2018033E10160D102088051010009
:104DA000704710B5042000F09BFC27482749284A8B
:104DB0000068B0FBF1F31370B0FBF1F142F2107038
:104DC00041430A2050804FF0E020026942F0020285
:104DD00002614161016941F00101016110BD70B5DD
:104DE00005461C48854208D905464A221AA121A039
:104DF00003F0D8F823A003F0D5F800214FF0E02607
:104E00007469134800784543B369B2699A42FCD08B
:104E100003D2A3EB0200014403E0A4EB0200184418
:104E200001441346A942F0D370BD70B50546002475
:104E30004FF47A7605E000F05BF93046FFF7CFFFDC
:104E4000641CAC42F7D370BDCC07002040420F0079
:104E50009C070020E3388E032E2E5C535953544593
:104E60004D5C5359535449434B5C73797374696374
:104E70006B2E63004C6F674572723A2025732C25A8
:104E8000640000000000000010B50C46794A52F89A
:104E90002030002B09D0342277A17DA003F082F8C6
:104EA0007FA003F07FF8204610BD42F82040FAE7CB
:104EB000704951F82000002800D0004770472DE9C4
:104EC000FF4104460F4615461E4641F6991087429B
:104ED00008D907465E2268A16DA003F063F870A0B0
:104EE00003F060F86F48012150F8240000F086FEBE
:104EF0006C480838005D8DF80C008DF80D500025C9
:104F00008DF80E5001208DF80F0003A800F0A5FBCE
:104F100041F61F40ADF80000ADF80650ADF8025064
:104F2000384606F04DFA604A604B06F041F8002220
:104F30005F4B06F0BBFC06F0FFF9ADF804008DF8FE
:104F400008505C4D694655F8240001F0CDFC012263
:104F500055F82400114601F0B2FF55F824003146FF
:104F600001F093FF55F82400012102F0E7F9BDE8B4
:104F7000FF81504951F82000002102F0A7B970B517
:104F800004464C4D002155F8240002F09FF955F8D5
:104F90002400BDE87040012101F077BF454951F878
:104FA0002000002101F071BF10B501218C072046BF
:104FB00002F0B8F9012807D10121204602F0BEF91C
:104FC000BDE81040002073E710BD10B53A4C012138
:104FD000204602F0A7F9012807D10121204602F05E
:104FE000ADF9BDE81040012062E710BD10B5334CAB
:104FF0000121204602F096F9012807D1012120461F
:1050000002F09CF9BDE81040022051E710BD10B538
:105010002B4C0121204602F085F9012807D10121FE
:10502000204602F08BF9BDE81040032040E710BD98
:1050300010B5244C0121204602F074F9012807D153
:105040000121204602F07AF9BDE8104004202FE744
:1050500010BD10B51C4C0121204602F063F9012857
:1050600007D10121204602F069F9BDE81040052072
:105070001EE710BD385D00202E2E5C535953544559
:105080004D5C54494D45525C74696D65722E6300E8
:105090004C6F674572723A2025732C25640000001E
:1050A0000000000074D102089A9999999999B93F22
:1050B0000000F03FA007002000040040000800406E
:1050C000000C0040001000400014004010B545F2F4
:1050D000555001F071F9062001F071F940F20D30E0
:1050E00001F070F901F071F9BDE8104001F072B9FA
:1050F00001F06BB903E010F8013B01F8013B521ECF
:1051000092B2F8D270472DE9F04105460E46174697
:10511000002407E0284602F035FA26F81400AD1CFA
:10512000641CA4B2BC42F5D3BDE8F0812DE9F04186
:105130000E4617460546002409E036F814102846A6
:1051400002F022FA0428EFD1AD1C641CA4B2BC42C8
:10515000F3D3E9E72DE9F04FADF6040D82460F4693
:105160001546AAF10064B4F1005F04D300200DF6E7
:10517000040DBDE8F08F212000F044FC012809D087
:105180006B22A3A1A8A002F00DFFABA002F00AFFC2
:105190000220ECE702F0EFF84FEAD428C4F3490606
:1051A000C6F58064A54200D82C460DF1040B37E00B
:1051B00032183BF812208A4203D1401C80B2A04230
:1051C000F6D3A04214D2484602F00EF9002006E0C1
:1051D000821937F810102BF81210401C80B2A04230
:1051E000F6D348464FF4806201A9FFF79FFF04E021
:1051F000224639465046FFF799FFA54203D102F0F7
:10520000C6F80320B3E708F10108002607EB4407BE
:10521000A244281B85B24FF48064A54200D82C46D6
:105220004FF0006000EBC829421401A94846FFF77F
:105230006AFF00204FF6FF71C1E72DE9F0410746F4
:105240000E46002402F0010000EB5205212000F080
:10525000D9FB012809D0A8226DA173A002F0A2FEFB
:1052600075A002F09FFE02205EE702F084F8A7F12D
:105270000060B0F5002F01D278050BD0AE2264A1FA
:1052800069A002F08FFE6CA002F08CFE02F07FF8A5
:10529000022049E7B5F5006F0BD9B4225CA162A0EA
:1052A00002F080FE64A002F07DFE02F070F80220A1
:1052B0003AE7352002F083FA384602F095F80428E0
:1052C0001BD0BB2252A158A002F06CFE5AA002F0E3
:1052D00069FE12E00A20FFF7A8FD0A2C0BD9C222B2
:1052E0004BA151A002F05EFE53A002F05BFE02F063
:1052F00042F8022018E7641CA4B2012002F050FA20
:105300000128E7D023E0202002F059FA30787178A4
:10531000B61C40EA0121384602F036F9002410E0BC
:105320000A20FFF782FD1E2C09D9D32238A13EA006
:1053300002F038FE40A002F035FE0220F4E6641CC4
:10534000A4B2202002F02CFA0128E9D1BF1C6D1E66
:10535000ADB2D8D202F01BF80320E5E62DE9F04704
:105360008146884600260024002702F0010000EB59
:105370005205212000F046FB01280AD0F12224A189
:1053800029A002F00FFE2CA002F00CFE0220BDE8C6
:10539000F08701F0F0FF352002F011FA12E00A2048
:1053A000FFF743FD0A2C0BD9FB2219A11EA002F026
:1053B000F9FD21A002F0F6FD01F0DDFF0220E6E795
:1053C000641CA4B2012002F0EBF90128E7D018E038
:1053D000202002F0F4F9701C18F8061080B2421C6C
:1053E00018F8000096B241EA002A09EB07046005AC
:1053F00002D1204601F0F8FF2046514602F0C4F8E1
:10540000BF1C6D1EADB2E3D201F0C1FF0320BEE7A9
:105410002E2E5C53595354454D5C464C4153485CC9
:10542000666C6173682E63004C6F674572723A2038
:1054300025732C25640000000000000010B586B024
:1054400001214FF4017000F0CEFB4FF4004000F05A
:105450004DFB494C204600F0EBFD002101918DF8F9
:1054600008108DF809104FF4602203920491012175
:105470008DF8141001A9204600F006FE012000F06E
:1054800065FF0121204600F027FE204600F047FE80
:10549000204600F049FE0028FAD1204600F04BFEDD
:1054A000204600F04DFE0028FAD106B010BD10B520
:1054B000314C014607230122204600F06FFE0121F6
:1054C000204600F044FE0221204600F04DFF002857
:1054D000F9D02046BDE8104000F0A6BE70B500250A
:1054E00000241020FFF7E3FF284485B20A20FFF7CD
:1054F0009CFC641CE4B2052CF3D30520B5FBF0F052
:1055000070BD2DE9F04107460E460025002408E055
:105510003846FFF7CCFF05440A20FFF786FC641CE1
:10552000E4B2B442F4D3B5FBF6F080B2BDE8F0814A
:1055300010B50A211020FFF7E4FF06F0CDFA06F0BF
:105540009FFA4FF066320D4B05F08AFF02460B467C
:105550000B480C4906F0AAF90B4A0C4B05F028FD44
:1055600000220B4B05F068FC00220A4B05F078FF87
:1055700005F0B2FE00B210BD0024014066664A3F4D
:10558000E17A14AE47E1F63F22FDF675E09C713FEB
:105590000000394000005940FEB505460E46012185
:1055A000084600F020FB4FF48037019700248DF867
:1055B00008408DF8095001258DF80A5001A800F027
:1055C00075FF384600F0D1FF8DF800508DF801606E
:1055D0008DF802408DF80340684600F03EF81B4904
:1055E00002200860C02000F0DBFF012000F0D5FFA2
:1055F000FEBD3EB50121080700F000FB01248DF837
:1056000008408DF8094000258DF80A508DF80B40B0
:1056100002A800F022F8684600F07FFF2004009006
:105620008DF8045008208DF805008DF80640684676
:1056300000F03CFFC02000F0B3FF012000F0ADFF00
:105640003EBD4FF4803000F090BF000000E100E06C
:105650002A4908432A490860704770B50F23C27869
:1056600001260178002A1ED0254A126802F4E06261
:10567000C2F5E062120AC2F10404D3404578A540A5
:1056800082781A402A43120101F1E02181F80024B6
:10569000007800F01F018E404009800000F1E020FA
:1056A000C0F8006170BD01F01F008640480980000D
:1056B00000F1E020C0F8806170BD124A1140014342
:1056C0000F48001F016070470D4A121D002903D0CA
:1056D0001168014311607047116881431160704780
:1056E0004FF0E021042804D0086920F0040008618C
:1056F0007047086940F00400086170470000FA052F
:105700000CED00E080FFFF1F10B59C49884209D1D5
:105710000121042000F07DFA0021BDE810400420A2
:1057200000F077BA9649884209D10121082000F09B
:1057300070FA0021BDE81040082000F06ABA9149D3
:10574000884209D10121102000F063FA0021BDE850
:105750001040102000F05DBA8B49884209D1012128
:10576000202000F056FA0021BDE81040202000F073
:1057700050BA8649884209D10121402000F049FAF7
:105780000021BDE81040402000F043BA8049884223
:1057900009D10121802000F03CFA0021BDE8104031
:1057A000802000F036BA7B4988420AD18415012155
:1057B000204600F02EFA2046BDE81040002100F0FF
:1057C00028BA10BD10B50121084600F022FA0021C8
:1057D000BDE81040012000F01CBA2DE9F041002284
:1057E000CC7804F00F03E40601D58C7823430C78C1
:1057F0004FF00F0714F0FF0F4FF0010C1CD005689D
:105800000CFA02F40E882640A64211D1960007FA3F
:1058100006F825EA080503FA06F848EA0505CE78F1
:10582000282E02D0482E02D002E0446100E004613C
:10583000521C082AE4D305600A88FF2A1ED945684D
:10584000002202F108060CFA06F40E882640A64251
:1058500010D1960007FA06F825EA080503FA06F8BB
:1058600048EA0505CE78282E00D14461CE78482E2E
:1058700000D10461521C082AE3D34560BDE8F081E1
:105880004FF6FF710180022181700421C1707047C1
:105890000246002092680A4200D0012070478068CA
:1058A00080B2704702460020D2680A4200D0012030
:1058B0007047C06880B270470161704741617047AE
:1058C000002A01D00161704741617047C160704793
:1058D00041F48032826181618261816980697047AF
:1058E00010B52D4B1A684FF68074224042EA001022
:1058F0000843186010BD2949C8617047F0B5264CAF
:10590000002801DAE36900E06368C0F30346420D52
:10591000120185B2C0F301579540032F07D0C20290
:105920000CD50322B240934343F0706209E023F0A8
:105930007062636823F07063636002E0AB4343F01E
:10594000706201B12A43002801DAE261F0BD6260B1
:10595000F0BD10B58A07120F0F23934021F0030406
:105960000D4921448C689C438C608B6890400343B4
:105970008B6010BD0949DC310860704700080140A8
:10598000000C0140001001400014014000180140CB
:10599000001C0140002001400000014000002042A6
:1059A000B448016841F0010101604168B24A114008
:1059B00041600168B14A11400160016821F4802111
:1059C0000160416821F4FE0141604FF41F018160D4
:1059D0007047A8490A6822F480320A600A6822F4F3
:1059E00080220A60B0F5803F07D0B0F5802F03D148
:1059F000086840F4A02008607047086840F48030D0
:105A0000086070470346002059099A4A01290AD0C4
:105A100002290AD0516A03F01F02012393400B426E
:105A200000D0012070471168F5E7116AF3E718B557
:105A3000002000904FF4A0643120FFF7E3FF0099AD
:105A4000491C00910099A14201D00028F4D03120D6
:105A5000FFF7D8FF08B1012018BD002018BD854A06
:105A6000116821F0F80141EAC000106070478449D4
:105A7000086070477F4B5A6822F47C120843104339
:105A8000586070477E49086670477A4A516821F02D
:105A900003010143516070477648406800F00C00F4
:105AA0007047744A516821F0F0010143516070471A
:105AB000704A516821F4E0610143516070476D4ABA
:105AC000516821F4605141EAC00050607047694A52
:105AD000002903D0517A014351727047517A8143B2
:105AE000517270476649D83108607047614A516801
:105AF00021F440410143516070475E49002220314A
:105B00000A7001F82029012805D0042802D10520B7
:105B100081F820007047012081F820007047594922
:105B20000860704753490A6A02430A627047554940
:105B300044390860704710B54E4A516801F00C01B5
:105B4000514B002927D0042927D0082927D00360EA
:105B5000516801F0F00109094C4B5C5C0168E140BF
:105B60004160546804F4E064240A1C5D21FA04F4E2
:105B70008460546804F46054E40A1B5DD940C16039
:105B8000526802F44042920B404B1B1F9A5CB1FBDF
:105B9000F2F1016110BD0360DAE70360D8E75168F4
:105BA00001F47011536803F48033022404EB914133
:105BB00033B153689B0307D5354B59430160C7E7A1
:105BC000334B59430160C3E72F4B59430160BFE793
:105BD000284A002903D05169014351617047516936
:105BE000814351617047234A002903D091690143E1
:105BF0009161704791698143916170471D4A002905
:105C000003D0D1690143D1617047D1698143D1612A
:105C10007047184A002903D0D1680143D16070470A
:105C2000D1688143D1607047124A002903D01169BD
:105C30000143116170471169814311617047114936
:105C40004039086070470E49C86470470949C871F7
:105C500070470848416A41F08071416270470146CF
:105C60000020044A92680A4200D00120704701498E
:105C700088727047001002400000FFF8FFFFF6FE38
:105C8000000042428004424200127A00BC07002019
:105C900000093D0010B5E14988420AD101218C0379
:105CA0002046FFF7B6FF2046BDE810400021FFF771
:105CB000B0BFDB4988420AD101214C042046FFF7DE
:105CC000B3FF2046BDE810400021FFF7ADBFD54926
:105CD00088420AD101218C042046FFF7A5FF204607
:105CE000BDE810400021FFF79FBFCF4988420AD18D
:105CF0000121CC042046FFF797FF2046BDE8104065
:105D00000021FFF791BFC94988420AD101210C0542
:105D10002046FFF789FF2046BDE810400021FFF72D
:105D200083BF10BD30B585B004460D46208A4CF6C1
:105D3000FF710840E98801432182A0894EF6F311E2
:105D40000840A9882A8911436A8902431143A18125
:105D5000A08A4FF6FF410840A9890143A182684605
:105D6000FFF7E9FEAD48844201D1039800E00298B4
:105D7000A189090408D500EBC00101EB00102968D6
:105D80004900B0FBF1F007E000EBC00101EB0010AF
:105D900029688900B0FBF1F06422B0FBF2F109013F
:105DA0000B096FF018056B4300EB8300A3891D04FA
:105DB0004FF0320307D503EBC000B0FBF2F000F068
:105DC0000700084306E003EB0010B0FBF2F000F020
:105DD0000F000843208105B030BD4FF4165101601B
:105DE00000218180C18001810C2242818181704724
:105DF00010B5038A4FF2FF0213400A884C882243F1
:105E00008C88C9880C4322431A43028210BD0021AA
:105E1000018041808180C1807047002904D0818940
:105E200041F4005181817047818921F400518181C1
:105E3000704710B540F66A13C1F3421301F01F0416
:105E40000121A140012B07D0022B07D014303AB119
:105E500002680A43026010BD0C30F8E71030F6E724
:105E600002688A43026010BD002A03D0828A0A4376
:105E700082827047828A8A4382827047028A22F035
:105E80000F020282028A0A4302827047828922F448
:105E90000062828182890A4382817047002904D08E
:105EA000818941F0020181817047818921F00201DD
:105EB00081817047028A22F020020282028A0A430C
:105EC00002827047002904D0018A41F48041018296
:105ED0007047018A21F4804101827047C1F30801B3
:105EE000818070478088C0F308007047818941F045
:105EF000010181817047028BD2B20283028B42EA98
:105F0000012101837047028B02F47F420283028BDE
:105F10000A4302837047002904D0818A41F020019E
:105F200081827047818A21F0200181827047002997
:105F300004D0818A41F0100181827047818A21F06A
:105F4000100181827047002904D0818A41F0080144
:105F500081827047818A21F008018182704700297F
:105F600004D0818941F40041818170478189C1F366
:105F70000E0181817047002904D0818A41F40061BB
:105F800081827047818A21F4006181827047828A10
:105F900022F004028282828A0A43828270470029A8
:105FA00004D0818A41F0020181827047818A21F008
:105FB0000201818270470246002012880A4200D006
:105FC000012070478A05C9430180704770B50024DD
:105FD00040F66A12C1F3421301F01F05012606FACA
:105FE00005F2012B0CD0022B0DD0838A1340090A35
:105FF0008E40008830400BB100B10124204670BDB6
:1060000083891340F3E7038A1340F0E740F66A12EE
:106010000A0A01219140C9430180704700380140BC
:106020000044004000480040004C00400050004048
:1060300010B5DB4988420AD1441501212046FFF7FB
:10604000E8FD2046BDE810400021FFF7E2BDD5493C
:1060500088420AD1041501212046FFF7DAFD2046C7
:10606000BDE810400021FFF7D4BDCF4988420AD1D6
:106070000121CC032046FFF7CCFD2046BDE81040AF
:106080000021FFF7C6BD10BD10B54268C74B1A40CE
:106090000C790B6842EA0422134343608268C44BC4
:1060A0001A40D1E9024323434C7942EA44021343A4
:1060B0008360C26A22F47002097C491EC9B242EAB6
:1060C0000151C16210BD0021016001714171816007
:1060D000C160012101747047002904D0816841F03A
:1060E000010181607047816821F001018160704782
:1060F000002904D0816841F4807181607047816813
:1061000021F4807181607047C9B2002A03D04268CF
:106110000A434260704742688A4342607047816820
:1061200041F0080181607047014600208968090735
:1061300000D501207047816841F0040181607047FB
:10614000014600208968490700D5012070470029D1
:1061500004D0816841F4A00181607047816821F416
:10616000A00181607047014600208968490200D57E
:1061700001207047426822F46042491E42EA4131E0
:1061800041607047002904D0416841F400614160DA
:106190007047416821F400614160704770B507267F
:1061A00009290AD9C568A1F10A0404EB4404A640F0
:1061B000B543A3401D43C56007E0056901EB4104F9
:1061C000A640B543A3401D4305611F23072A09D2FA
:1061D000446B521E02EB820293409C4391400C435D
:1061E000446370BD0D2A09D2046BD21F02EB8202F8
:1061F00093409C4391400C43046370BDC46A0D3AC4
:1062000002EB820293409C4391400C43C46270BDF8
:10621000002904D0816841F4801181607047816851
:1062200021F4801181607047C06C80B270475C4877
:106230004C3000687047002904D0416841F4806107
:1062400041607047416821F48061416070470029D6
:1062500004D0416841F4805141607047416821F4A5
:10626000805141607047826822F4E0420A438260B4
:106270007047002904D0816841F400418160704773
:10628000816821F4004181607047002904D0816851
:1062900041F4021181607047816821F4021181602C
:1062A0007047014600208968890200D501207047A7
:1062B00070B5072609290AD9C568A1F10A0404EBBB
:1062C0004404A640B543A3401D43C56007E00569EB
:1062D00001EB4104A640B543A3401D430561836B18
:1062E000C3F30154121B921C02EB82021F24944040
:1062F000A34391400B43836370BD826B22F4401231
:10630000491E42EA01518163704708B50090009828
:10631000084400900098026008BD08B500900098FD
:106320000844283000900098006880B208BD426898
:10633000204B1A400A4342607047416282627047B4
:10634000426822F01F020A43426070471449083134
:10635000002804D0086840F400000860704708680E
:1063600020F40000086070470246002012680A42CC
:1063700000D001207047C9430160704710B5024644
:1063800000200B0A5468C9B20C401168194202D0AF
:10639000002C00D0012010BD090AC94301607047DC
:1063A0000024014000280140003C0140FFFEF0FFB6
:1063B000FDF7F1FFFFFD3FFF0D49086070470C49F5
:1063C000486070470A498860704709494AF6AA2020
:1063D0000860704706494CF6CC400860704701469B
:1063E0000020034AD2680A4200D001207047000012
:1063F0000030004010B50120FFF721FCBDE810403F
:106400000020FFF71CBC2049086070471E49091F87
:10641000086070471C498431086070471B4A118826
:1064200021F46071014311807047184A118821F0EE
:106430007F0101431180704708B5144A2C3A10447B
:1064400000900098016008BD08B510492C39084437
:1064500000900098008808BD0B489C300068C0B2CE
:1064600070470A480830018841F0010101807047F7
:106470000548A0300068C0B2704704480830018861
:1064800041F002010180704704860D422C6C0040EF
:10649000384900200860091D0860091D0860091DB1
:1064A00008603449344814310860704730B5314AC7
:1064B00083790168002B2AD013688B431360111D68
:1064C0000B680468A3430B60017911440B680468EE
:1064D00023430B60274C08342168036899432160EB
:1064E000231D19680568A94319604179102905D051
:1064F00011440A68006802430A6030BD21680268DE
:1065000011432160196800680143196030BD0079AA
:10651000104402688A43026030BD002101600171AD
:106520000C22427181717047124910310A6802438E
:106530000A607047014600200E4A143212680A426F
:1065400000D0012070470B491431086070470146A4
:106550000020084A12680A40064B14331B680B429D
:1065600002D0002A00D0012070470249143108608F
:106570007047000000040140FFFF0F0010B501212B
:106580000C072046FFF750FB2046BDE810400021D5
:10659000FFF74ABB214908627047204908617047EC
:1065A0001F4A116821F0E0010143116070471B4947
:1065B000A031086070471A4B1A6822F003020243A8
:1065C0001A601848026842F004020260012905D0EE
:1065D00020BF016821F004010160704730BFF8E777
:1065E0000F48016841F004010160016841F00201B7
:1065F00001600C48016841F00401016030BF704740
:1066000001460020064A52680A4200D00120704725
:1066100003490A6842EA80000860704700000E42A1
:106620000070004010ED00E03A4A002903D01188C4
:1066300001431180704711888143118070473548AC
:10664000001D018841F01001018070473148001D94
:10665000018821F01001018070472E481C3000880D
:106660002C491831098840EA01407047294A010C39
:1066700018321180111D08807047264AC0F303416B
:1066800008321180111D0880E0E7224A010C2032F7
:106690001180111D088070471E48103000880007C7
:1066A000010B1C4814300088084370471948001D2E
:1066B00001888906FCD570471648001D018821F025
:1066C0000801018001880907FCD5704701460020B8
:1066D000104A121D12880A4200D0012070470D494D
:1066E000091D0A8882430A8070470A49091D0988E2
:1066F000C2B21140074A1288024202D009B10120F9
:106700007047002070470349091D0A8882430A80A8
:10671000704700000028004010B5FE4988420AD1A9
:10672000C41401212046FFF774FA2046BDE810404A
:106730000021FFF76EBAB0F1804F0CD0F6498842C5
:1067400013D101210220FFF76FFA0021BDE81040AC
:106750000220FFF769BA01210846FFF765FA002118
:10676000BDE810400120FFF75FBAEC49884209D12B
:1067700001210420FFF758FA0021BDE81040042051
:10678000FFF752BAE649884209D101210820FFF7F4
:106790004BFA0021BDE810400820FFF745BAE14957
:1067A000884209D101211020FFF73EFA0021BDE8FF
:1067B00010401020FFF738BADB49884209D1012187
:1067C0002020FFF731FA0021BDE810402020FFF71C
:1067D0002BBAD64988420AD1441401212046FFF73A
:1067E00018FA2046BDE810400021FFF712BAD04940
:1067F00088420AD10121CC042046FFF70AFA20463C
:10680000BDE810400021FFF704BACA4988420AD106
:1068100001210C052046FFF7FCF92046BDE8104099
:106820000021FFF7F6B9C44988420AD101214C057D
:106830002046FFF7EEF92046BDE810400021FFF7A3
:10684000E8B9BE49884209D101214020FFF7ECF99F
:106850000021BDE810404020FFF7E6B9B849884262
:1068600009D101218020FFF7DFF90021BDE81040A8
:106870008020FFF7D9B9B34988420AD18415012194
:106880002046FFF7D1F92046BDE810400021FFF770
:10689000CBB9AD4988420AD101210C042046FFF74B
:1068A000B8F92046BDE810400021FFF7B2B9A7496A
:1068B00088420AD101214C042046FFF7AAF920465C
:1068C000BDE810400021FFF7A4B9A14988420AD1D0
:1068D00001218C042046FFF79CF92046BDE81040BA
:1068E0000021FFF796B910BD30B50288894C8F4D55
:1068F000A0420DD0A8420BD0B0F1804F08D0864BFB
:10690000984205D0854B984202D0854B984203D1DE
:1069100022F070034A881A43824B984206D0824B79
:10692000984203D022F44073CA881A4302808A88AE
:1069300082850A880285A0420AD0A84208D0824AED
:10694000904205D0814A904202D0814A904201D1C2
:10695000097A01860121818230BD30B5028C22F096
:1069600001020284028C8388048B24F0700424F0DA
:1069700003050C882C4322F002020D8915434A8836
:106980002A43644DA8420BD0684DA84208D06E4DF2
:10699000A84205D06D4DA84202D06D4DA8420FD13E
:1069A00022F008054A892A4322F004058A882A43EE
:1069B00023F4807323F400738D891D43CB892B430B
:1069C00083800483C9888186028430BD70B5028CBF
:1069D00022F010020284028C8388048B24F4E044A9
:1069E00024F440760D884FF6FF7404EA05253543FC
:1069F00022F020020E8904EA061616434A8804EAA9
:106A000002123243434EB04202D0484EB04217D138
:106A100022F080024E8904EA0616164326F040064C
:106A20008A8804EA0212324323F4806323F4006369
:106A30008E8904EA86061E43CB8904EA8303334326
:106A400083800583C9880187028470BD70B5028C7C
:106A500022F480720284028C8388848B24F0700478
:106A600024F003040D88254322F400720E894FF6AA
:106A7000FF7404EA062616434A8804EA02223243D7
:106A8000244EB04202D0294EB04217D122F4006603
:106A90004A8904EA0222324322F480668A8804EAA0
:106AA0000222324323F4805323F400538E8904EAF4
:106AB00006161E43CB8904EA031333438380858380
:106AC000C9888187028470BD70B5028C22F480521F
:106AD0000284058C8288838B23F4E04323F4407680
:106AE0000C884FF6FF7303EA0424344325F4005561
:106AF0000E8903EA06362E434D8803EA05353543F1
:106B0000044EB04202D0094EB04226D122F4804653
:106B10008A891FE0002C014000040040000800406A
:106B2000000C004000100040001400400034014000
:106B3000004C01400050014000540140001800404A
:106B4000001C004000200040004001400044014083
:106B50000048014003EA8212324382808483C9885C
:106B6000A0F84010058470BD828B22F440628283BD
:106B7000828B4FF6FF7303EA01210A438283704739
:106B8000F0B5048C24F480540484868B048C4FF676
:106B9000FF7505EA013726F4734605EA02223243FF
:106BA00005EA03331343F74A90420ED0F64A904267
:106BB0000BD0B0F1804F08D0F44A904205D0F44A8F
:106BC000904202D0F34A904205D124F40051394357
:106BD00041F4805104E024F402420A4342F480511B
:106BE00083830184F0BD828B22F00C028283828B2E
:106BF0000A4382837047F0B5048C24F480740484C3
:106C0000858B048C4FF6FF7707EA012625F0F30504
:106C100007EA031313432B43DA4A90420ED0DA4AB1
:106C200090420BD0B0F1804F08D0D84A904205D0A6
:106C3000D74A904202D0D74A904205D124F400713D
:106C4000314341F4807104E024F420620A4342F4A9
:106C5000807183830184F0BD028B22F44062028341
:106C6000028B4FF6FF7303EA01210A430283704748
:106C7000F0B5048C24F010040484068B048C4FF6C9
:106C8000FF7505EA011726F4734605EA033333431B
:106C900005EA02221A43BB4B98420ED0BA4B9842E7
:106CA0000BD0B0F1804F08D0B84B984205D0B84B0C
:106CB000984202D0B74B984205D124F020013943C5
:106CC00041F0100104E024F0A0030B4343F0100155
:106CD00002830184F0BD028B22F00C020283028B3E
:106CE0000A430283704770B5048C24F001040484C5
:106CF000058B048C25F0F3054FF6FF7606EA0313A7
:106D000013432B439F4A90420ED09F4A90420BD090
:106D1000B0F1804F08D09D4A904205D09C4A9042E5
:106D200002D09C4A904205D124F002020A4342F06C
:106D3000010104E024F00A020A4342F00101038346
:106D4000018470BD70B505460C468E48854209D059
:106D50008D48854206D0B5F1804F03D08B488542DF
:106D600000D08B4820886188A288238958B10428E4
:106D700011D0082817D02846FFF702FFE1882846DF
:106D8000BDE87040F0E62846FFF7ADFFE1882846F1
:106D9000BDE870409FE72846FFF76AFFE188284674
:106DA000BDE8704058E72846FFF725FFE1882846F0
:106DB000BDE8704017E72DE9F04107460C46002575
:106DC00001266188002900D10225A288012A00D16C
:106DD00002262088238988B13846FFF749FFE188D9
:106DE0003846FFF739FF2389324629463846FFF7F0
:106DF0007AFFE1883846BDE8F0416CE73846FFF796
:106E000072FFE1883846FFF766FF2389324629463C
:106E10003846FFF72DFFE1883846BDE8F0411BE713
:106E200010B50A884B88CC881A438B8823431A43B1
:106E30000B891A434B8989891A430A43A0F84420D5
:106E400010BD4FF6FF71818000210180C18041801B
:106E5000017270470021018041808180C1800181E1
:106E600041818181C18170470021018041800122DF
:106E70008280C18001817047002101804180818032
:106E8000C1800181418181817047002904D001883E
:106E900041F0010101807047018821F0010101806A
:106EA0007047002905D030F8441F41F400410180AB
:106EB000704730F8441FC1F30E0101807047002A6B
:106EC00003D082890A438281704782898A43828102
:106ED0007047818270471143A0F848107047002A1C
:106EE00003D082890A438281704782898A438281E2
:106EF0007047018921F0070101817047028922F062
:106F000070020A430281704700B503461846FFF736
:106F1000F5FF188940F00700188100BD70B50D46D7
:106F200004461146602D0CD001222046FFF7DBFEFF
:106F300029462046FFF7E2FF208940F00700208124
:106F400070BD01222046FFF793FEF1E730B50489BA
:106F5000E4B24FF6FF7505EA032313430B432343C3
:106F6000038130BD10B504462046FFF7EFFF2089AE
:106F700020F0070040F0070020F0700040F07000A3
:106F8000208110BD002C014000340140000400406D
:106F900000080040000C004010B504462046FFF7F2
:106FA000D5FF208940F480402081EAE70185828274
:106FB0007047028822F070020A430280704770B561
:106FC0000589048B068C25F007050D434FF6FC411F
:106FD0000C4040F201110C4326F022064FF6FF71DF
:106FE00001EA03111143314305810483018470BD1B
:106FF000028B22F070020A4302837047028B22F454
:10700000E0424FF6FF7303EA012111430183704709
:10701000828B22F070020A4382837047828B22F4B3
:10702000E0424FF6FF7303EA012111438183704769
:10703000002904D0018841F0800101807047018857
:1070400021F0800101807047002904D0818841F03F
:10705000040181807047818821F00401818070479C
:10706000002904D0818841F008018180704781881F
:1070700021F0080181807047002904D0818841F007
:10708000010181807047818821F001018180704772
:10709000028B22F008020A4302837047028B22F41B
:1070A00000624FF6FF7303EA012111430183704729
:1070B000828B22F008020A4382837047828B22F47B
:1070C00000624FF6FF7303EA012111438183704789
:1070D000028B22F004020A4302837047028B22F4DF
:1070E00080624FF6FF7303EA012111430183704769
:1070F000828B22F004020A4382837047828B22F43F
:1071000080624FF6FF7303EA0121114381837047C8
:10711000028B22F080020A4302837047028BC2F383
:107120000E024FF6FF7303EA0121114301837047FA
:10713000828B22F080020A4382837047828BC2F3E3
:107140000E024FF6FF7303EA01211143818370475A
:10715000028C22F002020A4302847047028C22F061
:1071600008020A4302847047028C22F020024FF684
:10717000FF7303EA0111114301847047028C22F06E
:1071800080024FF6FF7303EA011111430184704737
:10719000028C22F400724FF6FF7303EA01211143BF
:1071A00001847047028C22F400624FF6FF7303EAF9
:1071B0000121114301847047028C22F400524FF6E2
:1071C000FF7303EA013111430184704710B50123B5
:1071D0008B40048C9C430484038C8A4013430384B7
:1071E000CFE610B504238B40048C9C430484038CAD
:1071F0008A4013430384C4E630B500F11803012428
:107200008C40058CA5430584002911D008290FD096
:10721000091FC1F34E001844016821F4E0410160E8
:1072200001684FF6FF7303EA02221143016030BD8B
:1072300003EB5100016821F0700101600168114306
:10724000016030BD002904D0018841F002010180B5
:107250007047018821F0020101807047002904D0A5
:10726000018841F0040101807047018821F0040188
:1072700001807047002904D0818841F0800181801D
:107280007047818821F0800181807047028822F058
:107290000802028002880A4302807047828822F036
:1072A0007002828082880A4382807047028922F0BD
:1072B0000702028102890A4302817047028922F093
:1072C0008002028102890A430281704781847047EB
:1072D0008185704781867047018770478187704735
:1072E000A0F840107047028822F4407202800288A1
:1072F0000A4302807047808E7047008F7047808FEE
:107300007047B0F840007047808C7047008D704720
:1073100002460020128A0A4200D001207047C94369
:107320000182704702460020138A0B4092890A406E
:10733000002B02D0002A00D001207047C9430182EF
:1073400070470000FE4A116801F0380101431160E6
:107350007047FB490A6822F008020A600A68024383
:107360000A607047F6490A6822F010020A600A684B
:1073700002430A607047F248F2494160F2494160B5
:107380007047EF48EF494160EF4941607047EC4872
:10739000016941F0800101617047E948016941F0EC
:1073A0008001016170470420E549CA68D20701D015
:1073B00001207047CA68520701D502207047C9688A
:1073C000C906FBD50320704700B50346FFF7EBFF66
:1073D00002E0FFF7E8FF5B1E012801D1002BF8D186
:1073E000002B00D1052000BD70B505464FF43026B6
:1073F0003046FFF7E9FF042811D1D14C206940F055
:10740000020020616561206940F040002061304643
:10741000FFF7DAFF216941F6FD721140216170BD6D
:1074200030B54FF430252846FFF7CEFF042810D1A1
:10743000C34C206940F004002061206940F0400006
:1074400020612846FFF7C0FF216941F6FB72114019
:10745000216130BD00B50346FFF7A5FF02E0FFF74D
:10746000A2FF5B1E012801D1002BF8D1002B00D117
:10747000052000BD30B54FF430252846FFF7EAFF60
:10748000042810D1AE4C206940F00400206120692E
:1074900040F0400020612846FFF7DCFF216941F6FB
:1074A000FB721140216130BD0020A549C9698907DF
:1074B00000D50120704770B5A525FFF7F5FF00B195
:1074C00000254FF430263046FFF77EFF042818D100
:1074D0009B4C9C48A0609C48A060206940F0200024
:1074E0002061206940F0400020613046FFF76CFFCA
:1074F00041F6EF76042805D0052802D021693140F5
:10750000216170BD206941F6DF710840206120696A
:1075100040F0100020618D4805804FF40050FFF7C7
:1075200053FF0528EDD021693140216170BD2DE95F
:10753000F84105460E46002000904FF400573846AB
:10754000FFF742FF04280FD17D4C206940F0010075
:1075500020612E80B8464046FFF736FFBF1E042844
:1075600004D0216939402161BDE8F881AD1C009546
:107570000099300C08804046FFF726FF216939400A
:107580002161F1E700887047F0B506460D464FF4DB
:1075900000573846FFF718FF04280CD1684C2069C3
:1075A00040F00100206135803846FFF70DFF21696A
:1075B000BA1E11402161F0BDF0B505460E464FF4EC
:1075C00000573846FFF700FF042813D15C4C5D4894
:1075D000A0605D48A060206940F0100020612E800E
:1075E0003846FFF7F1FE052804D0216941F6EF7215
:1075F00011402161F0BD2DE9F043C043C4B2C0F396
:107600000725C0F30746070E4FF400594846FFF719
:10761000DBFE04283CD1DFF828814A49C8F808106D
:107620004949C8F80810D8F8101041F01001C8F8FE
:107630001010FF2C05D04548083004804846FFF75D
:10764000C3FE042807D1FF2D05D040480A3005802D
:107650004846FFF7B9FE042807D1FF2E05D03B4866
:107660000C3006804846FFF7AFFE042807D1FF2FF5
:1076700005D036480E3007804846FFF7A5FE05289E
:1076800006D0D8F8101041F6EF721140C8F810106B
:10769000BDE8F08370B505464FF430263046FFF75D
:1076A00093FE042818D1264C2648A0602648A060E6
:1076B000206940F020002061206940F040002061F6
:1076C0003046FFF781FE41F6DF71042805D005281A
:1076D00002D022690A40226170BD20690840206101
:1076E000206940F010002061184815B10021018088
:1076F00001E0A52101803046FFF766FE0528EBD0AA
:10770000216941F6EF721140216170BD2DE9F04110
:1077100006460D4617460A4C0A48A0600A48A06073
:107720004FF400584046FFF74FFE04281DD1206952
:1077300040F0100020613D43354345F0F80007E07C
:107740000020024023016745AB89EFCD00F8FF1F01
:107750002549891C08804046FFF736FE052804D0DD
:10776000216941F6EF7211402161BDE8F0811F48A7
:10777000C069800870471D48006A704700201B4997
:107780000968890600D501207047184A002903D0EE
:10779000116901431161704711698143116170479B
:1077A00001460020114A012904D0D2680A4200D0C3
:1077B00001207047D169C907FBD0012070470B49F0
:1077C000C860704704200949CA68D20701D0012067
:1077D0007047CA68520701D502207047C968C906B8
:1077E000FBD503207047000000F8FF1F0020024077
:1077F00001684FF6FE721140016000210160416096
:107800008160C1607249724A0839904204D1486867
:1078100040F00F00486070476D4A1432904204D126
:10782000486840F0F00048607047694A283290424A
:1078300004D1486840F4706048607047644A3C3244
:10784000904204D1486840F4704048607047604AF4
:107850005032904204D1486840F47020486070472C
:107860005B4A6432904204D1486840F4700048603A
:107870007047574A7832904204D1486840F07060AF
:1078800048607047534A111F904204D1086840F085
:107890000F00086070474F4A1432904204D10868C4
:1078A00040F0F000086070474A4A2832904204D104
:1078B000086840F4706008607047464A3C32904265
:1078C00004D1086840F4704008607047414A503263
:1078D0009042FAD1086840F470200860704730B5D3
:1078E000026847F6F0739A430C6A8B682343D1E928
:1078F00004452C4323438C692343CC6923434C6ABE
:1079000023438C6A234313430360CA6842600A68B6
:1079100082604968C16030BD0021016041608160C2
:10792000C160016141618161C16101624162816245
:107930007047002904D0016841F0010101607047DF
:1079400001684FF6FE72114001607047002A03D0B3
:1079500002680A430260704702688A430260704707
:1079600041607047406880B2704702460020D100F5
:1079700003D518490839096802E01549083909682A
:10798000114200D001207047C10003D51149091FE1
:10799000086070470E490839486070470246002069
:1079A000D10003D50B490839096802E008490839B4
:1079B0000968114200D001207047C10003D5054974
:1079C000091F086070470249083948607047000085
:1079D00008000240080402407047162205A10FA0CB
:1079E00000F0E0FA11A000F0DDFAFEE7FEE7FEE7A6
:1079F000FEE770472E2E5C53544D333246313078BB
:107A00005F46574C69625C7372635C73746D3332AA
:107A1000663130785F69742E630000004C6F6745F3
:107A200072723A2025732C2564000000486172644C
:107A30004661756C745F48616E646C65722100000C
:107A400071B65A4801685A4A01F4E0611143016075
:107A5000BFF34F8FFEE70CB500220192009255480C
:107A6000016841F4803101604FF4A063016801F4C2
:107A7000003100910199491C0191009911B90199B6
:107A80009942F3D10168890302D50121009100E0F8
:107A900000920099012930D147490A6842F010024A
:107AA0000A600A6822F003020A600A6842F00202D1
:107AB0000A604168416041684160416841F4806109
:107AC0004160416821F47C114160416841F4E81152
:107AD0004160016841F08071016001688901FCD555
:107AE000416821F003014160416841F002014160B9
:107AF0004168C1F381010229FAD10CBDABE710B591
:107B00002C48016841F00101016041682B4A114095
:107B1000416001682A4A11400160016821F4802116
:107B20000160416821F4FE0141604FF41F01816052
:107B3000FFF7E4FF1D494FF00060091F086010BD0A
:107B400010B51C4A506800F00C011E4B1E4800295D
:107B50000ED004290ED008290ED0036051681A4AAD
:107B6000C1F30311121D515C0268CA40026010BDCE
:107B70000360F3E70360F1E7516801F470115368A3
:107B800003F48033022404EB914133B153689B0327
:107B900007D50E4B59430160E0E70C4B5943016098
:107BA000DCE7084B59430160D8E700000CED00E02A
:107BB0000400FA0500100240002002400000FFF817
:107BC000FFFFF6FE00127A00CC07002000093D00FE
:107BD00010B5A94988420AD1841401212046FEF734
:107BE00018F82046BDE810400021FEF712B8A3495E
:107BF00088420AD1041401212046FEF715F82046D8
:107C0000BDE810400021FEF70FB89D4988420AD117
:107C1000C41301212046FEF707F82046BDE81040B6
:107C20000021FEF701B810BD30B5028802F44153BF
:107C30000A884C88CD8822438C882C4322430C89A7
:107C400022434C8922438C892243CC8922431A4304
:107C50000280828B22F400628283098A018230BD15
:107C6000F0B585B005460C46022000210126AA8BFE
:107C70004FF240031A40AA8302222A84AF8BA268E3
:107C8000022A21D0A08800B102266846FDF753FFE2
:107C90000098E188B1F5007F2CD07101B0FBF1F0C4
:107CA00000EB8000A1684000B0FBF1F0401D80B205
:107CB0000A21B0FBF1F000F00101401AC0F34F00BF
:107CC0004FF6FF7202EA0121821EFE2A01D3022032
:107CD0000021E288084302432A8420886188A2891F
:107CE0000843A18811430843384340F40060A88347
:107CF00005B0F0BD000A00EB8000A1684000B0FBB9
:107D0000F1F0401D80B2D3E70021018041808180E5
:107D1000C180018141818181C18107210182704738
:107D20000021018041808180C180022282608181A6
:107D30007047002904D0018841F04001018070475C
:107D4000018821F0400101807047002904D0818B17
:107D500041F4806181837047818B21F4806181834C
:107D60007047090901238B4099B2002A03D0828809
:107D70000A438280704782888A4382807047002A43
:107D800003D082880A438280704782888A43828037
:107D900070478181704780897047A1F57E42FF3A24
:107DA00004D0018841F4807101807047018821F47A
:107DB000807101807047002904D0818841F004015E
:107DC00081807047818821F004018180704702889A
:107DD00022F40062028002880A4302807047018810
:107DE00041F4805101807047002904D0018841F49A
:107DF000005101807047018821F4005101807047D3
:107E0000012901D0008B7047808A7047008A704733
:107E1000B1F5804F04D0018821F480410180704782
:107E2000018841F480410180704702460020128998
:107E30000A4200D001207047C9430181704730B524
:107E40000246002001F00F03012505FA03F4A3B256
:107E5000090905FA01F4A4B29188214012891A4255
:107E600002D0002900D0012030BD01F00F02012115
:107E70009140C94301817047003001400038004003
:107E8000003C004030B50446039D2F4800EB031032
:107E900004600024047141718260C560102B00DB16
:107EA000002030BD29A10160002101714A1E8260BD
:107EB000C160704701210171704700210171704755
:107EC00070B5234D2868401C2860286810F1100FF9
:107ED00001D30020286000241B4E06EB041001791A
:107EE00001290BD14179022908D181682A68B2FBA6
:107EF000F1F301FB132109B9C0688047641C102C01
:107F0000EBDB70BD70B5124D6868401C6860686836
:107F100010F1100F01D30020686000240A4E06EB18
:107F20000410017901290BD14179012908D1816817
:107F30006A68B2FBF1F301FB132109B9C0688047FD
:107F4000641C102CEBDB70BD505D00202000000095
:107F5000E0070020704710B5044600F0AFFC006851
:107F6000005DC00602D504F1200010BD204610BD02
:107F70007CB51D4616460C00009001D02044401EE2
:107F8000074B7B442A4669460190304600F01BFFB0
:107F900005461CB10020694600F028FF28467CBD3C
:107FA000710E00000FB4044910B503AA029800F046
:107FB00041FF10BC5DF814FB400700200FB41CB556
:107FC000084B06AA7B4469460090059800F0FBFE2A
:107FD00004460020694600F009FF20461CBC5DF8FD
:107FE00014FB0000250E00000FB47CB50C0009AA9C
:107FF000009001D02044401E084B7B44694601900C
:10800000089800F0E0FE05461CB10020694600F02B
:10801000EDFE28467CBC5DF814FB0000F90D000065
:1080200070B5044685690068C10601D5302600E0B8
:108030002026C00707D070BDD4E901213046904703
:10804000206A401C20626D1EF6D570BD70B50446D6
:1080500085690078C00707D170BDD4E901212020CF
:108060009047206A401C20626D1EF6D570BD0968DD
:108070004A0501D540B27047C905FCD500B270472A
:1080800009684A0501D5C0B27047C905FCD580B260
:10809000704770B50C460546012A05D02878800641
:1080A00000D5EA69002302E0012305E05B1C93424E
:1080B00002D2E05C0028F9D1A869E618C01AA861CC
:1080C000286A184428622846FFF7AAFF04E0D5E989
:1080D000012114F8010B9047B442F8D32846FFF76A
:1080E000B5FF70BD2DE9F0410646002410687529E2
:1080F000314616A510D0FFF7BAFF002802DA404239
:1081000013A507E031688A0701D512A502E04907E7
:1081100004D511A5012401E0FFF7B2FF00210A22D6
:1081200006F1240709E0B0FBF2FCB0FBF2F302FB1E
:108130001C00303078541846491C0028F3D12346DF
:108140002A463046BDE8F04100F0CFBB00000000F9
:108150002D0000002B0000002000000011680268C4
:10816000006A530501D508700AE0D30501D50880DF
:1081700006E0130603D5C217C1E9000200E008605B
:10818000012070472DE9FF5F15468A460446DFF857
:10819000AC80F8440027D8E900103E46CDE9001035
:1081A00010E03AF816106A4602A800F0E1FE411C01
:1081B00007D02178890603D5E269391891420DD894
:1081C0000744761C2078800602D5E069B84205DDB8
:1081D000AE42E6DB3AF816000028E2D1A069C01BE7
:1081E000A0612046FFF71CFFD8E90010CDE9001080
:1081F000002017E03AF818106A4602A800F0B8FE0E
:10820000B0F1FF3F81460BD000250DF1080B05E0D2
:10821000D4E901211BF8050090476D1C4D45F7D3AB
:1082200008F10100B0428046E4DB206A3844206255
:108230002046FFF70BFFBDE8FF9F0000F64F000050
:1082400030B4002100F1240408E002F00705D20850
:10825000303542EA4372DB086554491C52EA030593
:10826000F3D10468002310A2250707D5A40600D483
:1082700021B1C46901230DA2641EC46130BC00F0A9
:1082800034BB10B5044621461068FFF7F9FE0246DC
:108290002046BDE810400023D2E7D21D22F007019E
:1082A000D1E90023CCE7000000000000300000000E
:1082B000F0B40D460188090502D5214C7C4402E04A
:1082C0001F4C7C440E34002100F1240608E002F02B
:1082D0000F071209E75D42EA03721B097754491C34
:1082E00052EA0307F3D102780023120704D5702D58
:1082F00006D009B1022311342246F0BC00F0F5BAD1
:1083000001231034F8E770B504460D462146106885
:10831000FFF7B6FE024629462046BDE8704000231E
:10832000C6E7D21D22F00703D3E90023C0E70368A4
:10833000126843F0200303600823C3610023B7E7FA
:10834000D44E00002DE9F05F894604464FF0000A44
:10835000DFF874B1FB44C0F820A02046E1688847EC
:10836000002874D0252806D0D4E901219047206A3E
:10837000401C2062F1E700265F462046E1688847FE
:108380002028054607DB312D05D2781910F8200C7E
:1083900008B10643F1E7B00701D526F00406C4F89A
:1083A0001CA00027C4F818A02A2D09D0284601F0E7
:1083B000E1FD38B304EB8708303DC8F8185019E0E8
:1083C00059F8041B204604EB87029161E168884755
:1083D000012F054618D1E069002820DA26F0200692
:1083E0001DE0D8F8180000EB800005EB40003038A5
:1083F000C8F818002046E1688847054601F0BAFD34
:108400000028EED1012F0AD02E2D08D12046E16898
:1084100088477F1C0546022F46F02006C4DBA06972
:10842000002803DA404246F00106A061F00701D0BF
:1084300026F010066C2D0BD0682D09D04C2D39D0AC
:108440006A2D35D0742D35D07A2D33D016E038E032
:10845000E1682F4620468847B842054609D16C2F6F
:1084600026D04FF48060E1680643204688470546E1
:1084700004E06C2F1AD04FF4807006430DB3A5F1C1
:108480004100192802D8203546F400664A4629469C
:10849000204626604E46F3F7A5FE80B101280BD09A
:1084A000F61D26F0070000F1080956E74020E4E732
:1084B0008020D8E70020D6E706F104094DE72846DA
:1084C00052E7206ABDE8F09F644E000070B5064692
:1084D00000F0FCF90468054630460A22002100F04D
:1084E0000FFD2C6070BD0000014A00F061BD00006E
:1084F000E8070020401ECAB210F8011F8A4202D0CD
:108500000029F9D10020704710B5431E13F8014F20
:10851000002CFBD105E011F8014B002C03F8014BB6
:1085200003D0521EF7D20021197010BD40EA01039A
:1085300010B59B070FD1042A0DD310C808C9121F0C
:108540009C42F8D020BA19BA884201D9012010BD46
:108550004FF0FF3010BD1AB1D30703D0521C07E013
:10856000002010BD10F8013B11F8014B1B1B07D177
:1085700010F8013B11F8014B1B1B01D1921EF1D1E8
:10858000184610BD40EA0103024630B59B0710D1E2
:108590004FF0013400E008C208C91D1B9D4315EAD5
:1085A000C41FF8D013F0FF0102F8011B0DD01B0A05
:1085B000F8E711F8013B002B02F8013B05D011F858
:1085C000013B002B02F8013BF3D130BD0022CBB2BE
:1085D00010F8011B994200D1421E0029F8D1104623
:1085E000704710B5431C02E010F8011B71B1810700
:1085F000FAD14FF0013202C88C1A8C4314EAC2112E
:10860000F9D0C01A0A0603D0C01E10BDC01A10BD92
:108610000A0401D0801E10BD0902FCD0401E10BD0E
:1086200040EA010370B59B072ED14FF00136042AB2
:108630002AD308C810C99D1B9D43121F15EAC615F1
:1086400017D0D8B2E1B2401A50EA056110D198B201
:10865000A1B2401A50EA05410AD123F07F4024F02C
:108660007F41401A50EA052102D1180EA0EB146098
:1086700070BDA342DBD018BA21BA884201D90120CB
:1086800070BD4FF0FF3070BD0AB9002070BD10F80A
:10869000013B11F8014B63B1A3420AD1521E08D02D
:1086A00010F8013B11F8014B1BB1A34201D1521E3E
:1086B000EDD1181B70BD421E12F8013F002BFBD1FB
:1086C00011F8013B002B02F8013BF9D17047032A56
:1086D00040F2308010F0030C00F0158011F8013BDF
:1086E000BCF1020F624498BF11F801CB00F8013BC6
:1086F00038BF11F8013BA2F1040298BF00F801CB8A
:1087000038BF00F8013B11F0030300F02580083A60
:10871000C0F0088051F8043B083A51F804CBA0E8B7
:108720000810F5E7121D5CBF51F8043B40F8043B0C
:10873000AFF30080D20724BF11F8013B11F801CB41
:1087400048BF11F8012B24BF00F8013B00F801CB12
:1087500048BF00F8012B704710B5203AC0F00B80DD
:10876000B1E81850203AA0E81850B1E81850A0E835
:108770001850BFF4F5AF5FEA027C24BFB1E818508F
:10878000A0E8185044BF18C918C0BDE810405FEAFF
:10879000827C24BF51F8043B40F8043B08BF70477B
:1087A000D20728BF31F8023B48BF11F8012B28BF80
:1087B00020F8023B48BF00F8012B704702F0FF038E
:1087C00043EA032242EA024200F002B84FF00002FC
:1087D0000429C0F0128010F0030C00F01B80CCF1D3
:1087E000040CBCF1020F18BF00F8012BA8BF20F841
:1087F000022BA1EB0C0100F00DB85FEAC17C24BF95
:1088000000F8012B00F8012B48BF00F8012B70473E
:108810004FF0000200B5134694469646203922BF19
:10882000A0E80C50A0E80C50B1F12001BFF4F7AF64
:10883000090728BFA0E80C5048BF0CC05DF804EB46
:10884000890028BF40F8042B08BF704748BF20F8B4
:10885000022B11F0804F18BF00F8012B704710B5A4
:10886000044610F0030F08BF11F0030F40F015800D
:108870004FF0013E121FC0F20E8051F8043BA3EBF3
:108880000E0C2CEA030C1CEACE1C08BF40F8043B7B
:10889000F0D0A1F1040102F10402521E08DB11F82C
:1088A000013B002B00F8013BF7D11146FFF78EFF8B
:1088B000204610BD704770477047704710B500F0F4
:1088C0009DFB001D10BD00BF19250000004870472A
:1088D000505E002010B5FFF7F9FF006810BD10B51D
:1088E0000446FFF7F3FF046010BD2DE9F0470D4685
:1088F00099469246044600F124080168880604D58A
:10890000E06921F01001216000E00120A84201DDB2
:10891000471B00E00027A1697A1902EB0900081A39
:10892000A0612078C00602D42046FFF779FB00261C
:1089300008E0D4E901211AF806009047206A401C9B
:10894000761C20624E45F4DB2078C0060AD520460E
:10895000FFF766FB06E0D4E9012130209047206A4A
:10896000401C2062381EA7F10107F4DC07E0D4E9BF
:10897000012118F805009047206A401C2062281E3B
:10898000A5F10105F3DC2046FFF760FB2078000627
:1089900002D50220BDE8F0870120FBE770472DE9F2
:1089A000FF4F0C461E464FF0FF378BB0D2E9000157
:1089B000DDF860800A908A46C1F30A5505B93D4644
:1089C000002108464FF00000BAF1000F00F440000B
:1089D00005DA00EB80004FF4400101EA50004FEA55
:1089E0009059B9F1010F00DDB9460A9850EA4A00E2
:1089F0000ED044F61050A5F2FF3545432F14B8F1C0
:108A0000000F1ED07542291E1EDDC9F100021CE0B8
:108A1000B8F1010F4FF0000001D0302103E0F24324
:108A200005E02154401CB042FBDB3046002200210F
:108A300021540B99C1F80880C1E900200FB0BDE8AE
:108A4000F08FBD1B6D1CDEE74A4600DA694206A8BE
:108A500000F02CFD06AB93E8070003AB83E80700AA
:108A600050460A9900F032FE8DE80700A0F500504C
:108A70001F3800900398002D0ADD42F21F014A467C
:108A80000844002303A90390684601F09BF809E01D
:108A9000A0F500504A461F38002303A903906846FA
:108AA00001F0A5F88DE807000004000C03D04FF09A
:108AB000FF30410800E01046B8F1000F03D000225B
:108AC000009215461EE0751E05D400F09BFA303268
:108AD00062556D1EF9D5B3460122084302D000222B
:108AE0007F1C04E02078302801D100227F1E002A5C
:108AF000099784D01DE0112D07DA00F083FA303297
:108B000062556D1C50EA0102F5D1084302D000986D
:108B1000C8B10EE00021681E05E0235C625C63546E
:108B20002254401E491C8142F7DBAB46A81B401E65
:108B30000990002004F80B000B98099AC0F80880EF
:108B4000C0E9002B7AE711264FF0000857E72DE91E
:108B5000F04F88460446D21D22F0070191B0D1E9BA
:108B60000001CDE90A0101F079F902460B98C00F26
:108B700001D02D2007E02068810701D52B2002E0DD
:108B8000202101EAC000032A099001D0072A05DB51
:108B900003464146204600F0F9FB0BE120788006B1
:108BA00001D5E06900E00620B8F1650F814606D0E6
:108BB000B8F1660F18D0B8F1670F70D131E000201E
:108BC000B9F1110F009001DB112301E009F101035C
:108BD0000AAA01A90CA8FFF7E2FEDDE90C70002645
:108BE00009F10105834647E001204B4600904FF014
:108BF00000470AAA01A90CA8FFF7D1FEDDE90DB0D4
:108C00000C995D46002610B909F101000D18B9EB69
:108C1000050003D4C0F1FF3609F10105A5EB0900F9
:108C20002BE0B9F1010F01DA4FF001090020B9F191
:108C3000110F0090484601DD112300E003460AAA07
:108C400001A90CA8FFF7ABFEDDE90C704D4600262C
:108C50008346207800070AD4AB4500DA5D4601A8B8
:108C6000012D04DD411911F8011C302907D04F45B1
:108C700002DA17F1040F04DA012082460FE06D1EBC
:108C8000EEE7002F02DCED1B3E4403E0781CA84217
:108C900000DD7D1CB81B00F1010A4FF00047207871
:108CA000000703D4AA4501DB4FF0FF3A0021B7F1DA
:108CB000004F0DF143088DF8431024D002202B23E0
:108CC000002F01DA7F422D230A21021EA0F10100AC
:108CD00000DC5FB197FBF1FC97FBF1F201FB1C7C20
:108CE00017460CF1300C08F801CDEEE7A8F10100B1
:108CF00003702188090501D5452100E06521A0F117
:108D0000010800F8011C09980FA9A1EB0807FF1D35
:108D100000B10120411901EBEA70A1693844081A39
:108D2000401EA0612078C00602D42046FFF778F9E3
:108D3000099828B1D4E901219047206A401C20629B
:108D40002078C00622D52046FFF76AF91EE0002EE3
:108D500004DBB34502DD01A8805D00E03020D4E9EA
:108D600001219047206A401C2062761CAAF1010074
:108D70005FEA000A0AD100F041F9C0680168405C6E
:108D8000D4E901219047206A401C2062281EA5F1E9
:108D90000105DCDC07E0D4E9012118F8010B90475C
:108DA000206A401C2062381EA7F10107F3DC204630
:108DB000FFF74CF9032011B041E6000001694A1C9D
:108DC00002610878704700B58FB0CDE9013100210C
:108DD000059105497944CDE9031011466846FFF72E
:108DE000B1FA0FB000BD0000E5FFFFFF0A6802F80E
:108DF000010B0A607047D1E900239A4202D2531C4A
:108E00000B601070704710B5436913B1AFF3008069
:108E100001E0FFF73EF9012010BD127800F12401B6
:108E20000A7000224A700122EDE711684FF0FF320C
:108E3000E9E70000074B70B50D467B44FFF7C3FF21
:108E40000446284600F0A4FB10B14FF0FF3070BD7F
:108E5000204670BD31A6FFFF10B5436913B1AFF3D3
:108E6000008001E0FFF78EF9012010BD128800F1AB
:108E7000240182840022C2840122EDE711684FF0B0
:108E8000FF32E9E72DE9F0418046D21D22F00702CA
:108E90000025D2E90002F52915A614D0011E72F1B1
:108EA000000106DA0023D0EB030063EB020211A6F7
:108EB00008E0D8F800108B0701D50FA602E049079B
:108EC00001D50EA601251146002408F1240704E06F
:108ED00000F098F830323A55641C50EA0102F7D19C
:108EE0002B46324621464046BDE8F041FFF7FDBC27
:108EF000000000002D0000002B00000020000000FA
:108F00002DE9F04791460F4680460446002614F8A6
:108F1000015B2DB1FFF7D2FC0068405DC007F6D1C0
:108F20002B2D02D02D2D18D0641E4A4639462046DE
:108F300000F06CFA27B13968A14201D1C7F800806E
:108F40004FF0020471050BD54042002803DDFFF706
:108F5000BDFC0460A007BDE8F08746F48066E4E746
:108F60000028F8DAFFF7B2FC04606FF00040F2E787
:108F700070B516460C460546FFF7A0FC036893F84B
:108F80000101012806D0FF2C0FD8185D68B101201F
:108F90002C7070BDD3F807013246214603F2071347
:108FA00003442846BDE8704018474FF0FF3070BDBD
:108FB0002DE9F04115460E46040002D12C6804B993
:108FC0000BA4204600F0F8FA0444207870B127463C
:108FD0003146384600F0E0FA0444207810B1002011
:108FE00004F8010B38462C60BDE8F0810027F9E752
:108FF0000000000000487047505E002000487047A5
:10900000705E002030B5B0F10A024FEA900E71F1A7
:1090100000034EEA817EB0EB0E0061EB91014FEA56
:10902000101E4EEA017E10EB0E0041EB11114FEACB
:10903000102E4EEA016E10EB0E0041EB11214FEAAB
:10904000104E4EEA014E10EB0E0041EB114140185C
:1090500041F100014FEAD00040EA41704FEAD101EE
:1090600010EB80054FEA810444EA907444EB01045C
:109070006D1944EB0404521BA3414FF0000348BF99
:109080000A3200D530BD401C41F1000130BD000066
:109090002DE9F04F04460D46D21D22F0070089B09D
:1090A000D0E900974846394600F0D8FE0246F80F4E
:1090B00001D02D2307E02068810701D52B2302E092
:1090C000202101EAC0038DF820300BB1012000E01F
:1090D0000020032A824601D0072A04DB29462046C5
:1090E00000F054F93FE12078800601D40D2500E01E
:1090F000E569C7F30A560D2D49DA00214FEA175BDF
:1091000008464FF00000002F00F4400007DA00EBA3
:1091100080004FF4400100EBD07001EA600081153F
:10912000012901DD4FF0FF3100224FEA850CBCF12F
:10913000180F06D31346ACF118004FF08052C2400E
:1091400003E04FF4801323FA0CF30CF10C0CBCF188
:10915000200F04D3ACF1200C09FA0CF001E007FA5F
:109160000CF000294FF0004801DD18B90FE00ED1D6
:1091700040450CD319EB02095F4121B9404502D1AA
:109180009F4329EA0209BBEB175F00D0761C2088B9
:10919000000502D57B48784402E07A4878441938C3
:1091A00008AA302302F80A30037C0AF10101002EDC
:1091B0000AF1020A53546A4602DC4FF0300101E022
:1091C0004FF031014FF001088DF8001002D0A6F2E7
:1091D000FF3603E059EA470100D06B4E002D02DC58
:1091E0002178090704D54FF002082E218DF80110CF
:1091F000C44600210BE0C7F303433F01C35C491C95
:109200006D1E02F80830052908F1010801DA002D69
:10921000F1DC00210CE000EB1973491C1B786D1E7A
:10922000082902F808304FEA091908F1010801DAA3
:10923000002DF0DC21688B0602D516E0A8F10108AC
:10924000E04505DD02EB080313F8013C302BF5D0B7
:10925000B8F1000F09DD02EB080313F8013C2E2BD7
:1092600003D1090701D4A8F10108002D05DD3E2135
:1092700002F808106D1E08F10108407C002E02F86B
:10928000080008F1010804DA2D20764202F80800EF
:1092900002E02B2002F808000A214FF47A7086427F
:1092A00008F101080BDB96FBF0F3303302F80830CD
:1092B00096FBF0F308F1010800FB136601E0642E51
:1092C0000CDB642096FBF0F3303302F8083096FB99
:1092D000F0F308F1010800FB136601E00A2E06DB3B
:1092E00096FBF1F0303002F8080008F1010896FB17
:1092F000F1F001FB1060303002F80800A16908F1BC
:10930000010808EB050202EB0A00081AA0612078A8
:10931000C00602D42046FEF783FE216A08AE01EBA8
:109320000A00206204E0D4E9012116F8010B9047FD
:10933000BAF1010AF7D22078C00602D52046FEF71E
:109340006FFE6E4609E016F8010B3E280FD0D4E9F7
:1093500001219047206A401C2062B8F10108F2D236
:109360002046FEF773FE09B00320BDE8F08F206AA7
:109370002844206203E0D4E90121302090476D1E8B
:10938000EBD3F8E71141000002FCFFFF2DE9F041AB
:109390001F46044603260168072A01F4006004DB27
:1093A00008B116A505E016A503E008B115A500E073
:1093B00015A521F010002060A069C01EA0610FB1AA
:1093C000401EA0612046FEF72BFE4FB1D4E90121DB
:1093D00038469047206A401C2062C01C206206E08C
:1093E000206AFAE7D4E9012115F8010B9047761EAF
:1093F000F8D22046FEF72AFEBDE8F0814E414E002D
:109400006E616E00494E4600696E66002DE9F05FA0
:10941000824615468B4600270AF10104B9460078BA
:10942000302801D09DB113E014F8010B01277828F2
:1094300003D0582801D045B10AE00DB1102D07D155
:10944000002714F8010B102502E0082500E00A258A
:109450000026B0460EE005FB080005FB06F10127DB
:109460001FFA80F801EB1046B6F5803F00D3B946ED
:1094700014F8010B294600F0D2F80028EBDABBF112
:10948000000F05D00FB1641E00E05446CBF8004039
:10949000B9F1000F06D0FFF719FA02210160C81ECA
:1094A000BDE8F09F48EA0640FAE700002DE9F047E2
:1094B000814616468AB0354878440DC88DE80D00BF
:1094C00032487844801C03AC0DC884E80D0041F696
:1094D0009B300844372190FBF1F290FBF1F5A5F1A8
:1094E000800501FB12041B3C02D56442012000E010
:1094F0000020DFF898A080460027FA44AAF1BE0AAF
:109500000EE0E0070AD03246684607EB4701012328
:109510000AEB810100F06BFB8DE8070064107F1CF3
:10952000002CEED1194F7F44AE3F19E0E80715D06B
:1095300007EB04100DF1180A90E80E008AE80E00FF
:10954000C068F04201D1981908903246012306A95B
:1095500003A800F04CFB03AB83E807006D10641C0C
:10956000002DE3D14FF0010332466946B8F1000FF8
:1095700003A802D000F026FB01E000F038FBC9E9A7
:109580000001C9F808200AB0BDE8F087803E00005D
:10959000007B00F08000704730B503461D781DB198
:1095A0000A4603E0AC4201D1181A30BD12F8014B53
:1095B000002CF7D15B1CF1E730B503461D783DB1B7
:1095C0000A4612F8014B1CB1AC42FAD15B1CF5E71C
:1095D000181A30BD7546FFF70DFDAE460500694609
:1095E000534620F00700854618B020B5F2F772FE0A
:1095F000BDE820404FF000064FF000074FF0000894
:109600004FF0000B21F00701AC46ACE8C009ACE814
:10961000C009ACE8C009ACE8C0098D4670473A28DB
:1096200000D2303820F02002412A01D3A2F13700C5
:10963000884201D34FF0FF30704710B50446AFF3B6
:1096400000802046BDE81040F2F72FBE4FF0013CED
:1096500050F8042B51F8043B9A4221D1A2EB0C03A1
:10966000934313EACC1317D150F8042B51F8043B61
:109670009A4215D1A2EB0C03934313EACC130BD1FE
:1096800050F8042B51F8043B9A4209D1A2EB0C0389
:10969000934313EACC13DBD04FF00000704700BFB8
:1096A000D01A01BAB1FA81F101F0180122FA01F0E1
:1096B000CB40C1F12001DBB2C0B2C01A2CFA01F3D9
:1096C000D11A914311EAC311E6D170475FEA400C09
:1096D00008BF91F0000F4FEA8C234FEAC12243EA02
:1096E00051514FEA1C5018BF00F5F0404FEA3000CE
:1096F00018BF41F000415FEA6C5C00F02980BCF1CA
:10970000FF3F08BF40F080407047130C06BF1204B3
:109710004FF0100C4FF0000C130E04BF12020CF1AE
:10972000080C130F04BF12010CF1040C930F04BFBB
:1097300092000CF1020CD30F04BF52000CF1010C8B
:1097400011464FF00002A0F11F00A0EB0C00704783
:1097500011F0004F08BF704731F000413FF4D5AF22
:109760000B0C06BF09044FF0100C4FF0000C0B0E51
:1097700004BF09020CF1080C0B0F04BF09010CF126
:10978000040C8B0F04BF89000CF1020CCB0F04BF3B
:1097900049000CF1010CCCF12003A0EB0C0022FAE3
:1097A00003F302FA0CF241EA030100F101007047F1
:1097B00020F07F4C80EA030023F07F47ACEB0703E7
:1097C00003F57C5300F0004003F1FF032DE98049CD
:1097D0004FEA154B09B44FEA144325EA0B4E24EA2D
:1097E00003480FF2042606EB132749083E785FEA88
:1097F000320203FB0667C7F5000707FB06F64FEAD0
:1098000054374FEAD64606F1020607FB066CCCF148
:10981000005C4FEA1C472CEA074C07FB06F40CFBE4
:1098200006F504EB15464FEA961634BF00204FF0BC
:1098300000404FEAD13706FB07FC4FEA1C4C0CFBFB
:109840000BF7D21B03FB0CF761EB07010CFB0EF7C8
:10985000B0EB074072EB17420CFB08F734BFA2EBEA
:109860000742B2EB074261EB17414FEA0C444FEA63
:10987000910706FB07FC4FEA1C4C0CFB0BF7B0EB07
:10988000C74072EB573203FB0CF734BFA2EBC74261
:10989000B2EBC74261EB57310CFB0EF7B0EBC700E0
:1098A00072EB57720CFB08F734BFA2EBC702B2EBA6
:1098B000C70261EB5771039F4FEA816141EA921140
:1098C00004EBCC044FEAD1374FEA826206FB07FC77
:1098D00042EA90124FEA80604FEA1C4C0CFB0BF7F7
:1098E000D21B03FB0CF761EB07010CFB0EF7B0EB8F
:1098F000074072EB17420CFB08F734BFA2EB07429C
:10990000B2EB074261EB17414FEA8C554FEA9107E2
:1099100004EB9C2406FB07FC4FEA1C4C0CFB0BF7EA
:10992000B0EBC74072EB573203FB0CF734BFA2EB2E
:10993000C742B2EBC74261EB57310CFB0EF7B0EBFD
:10994000C70072EB57720CFB08F734BFA2EBC702DB
:10995000B2EBC70261EB577115EB4C254FEA816101
:1099600041EA92114FEA82624FEAD13742EA9012FD
:1099700006FB07FC44F100044FEA80604FEA1C4CF0
:109980000CFB0BF7D21B03FB0CF761EB07010CFB85
:109990000EF7B0EB074072EB17420CFB08F734BF31
:1099A000A2EB0742B2EB074261EB174115EB1C1526
:1099B0004FEA813141EA92414FEA823242EA9042D3
:1099C0004FEA80304FEA0C7644F1000448EA034342
:1099D0004EEA0B484FF0000EB2EB080C71EB030798
:1099E00024BF624639464EEB0E0E4FF0000B0018B6
:1099F000524149414BEB0B0BB2EB080C71EB0307E7
:109A00007BF1000B24BF624639464EEB0E0E4FF041
:109A1000000B0018524149414BEB0B0BB2EB080C09
:109A200071EB03077BF1000B24BF624639464EEB16
:109A30000E0E51EA020718BF46F0010616EB0E762D
:109A400055F1000254F1000103D5BDE88901BDE8DC
:109A50000088BDE88901BDE80048B619524141EBD4
:109A60000101A3F10103704780807F7E7D7C7B7ABA
:109A70007978777676757473727171706F6E6E6DBA
:109A80006C6C6B6A6A696868676666656464636360
:109A900062616160605F5F5E5E5D5D5C5C5B5B5AE6
:109AA0005A59595858575756565555555454535353
:109AB00052525251515050504F4F4F4E4E4D4D4DAE
:109AC0004C4C4C4B4B4B4A4A4A49494948484847F9
:109AD0004747474646464545454444444443434337
:109AE0004342424242414141002B9C4630D47700E0
:109AF0002BD01CB54FEA370703B44FF010004FF0DE
:109B00001001BAF1000F06D0BCF1000FDCBF40F02D
:109B1000080040F008014FF000000FBCBDE8104005
:109B20000BF1010BBBF1010F08BF5FEA170722BF62
:109B300012F1010211F101014FF0004143F1000364
:109B400000F0004043EA00007047F9D35708D0E71F
:109B500046EA064613F1400F4FEA16461FDD13F1A1
:109B6000200FDFBF16430A46002120335B42BED0E0
:109B7000C3F1200746EA064602FA07F74FEA1646FF
:109B800046EA0706C3F1200722FA03F201FA07F7B3
:109B900021FA03F14FF0000342EA0702A7E746EA81
:109BA000020646EA06464FEA164646EA0106BCBFEA
:109BB00046EA0646360C4FF000034FF000024FF025
:109BC000000194E72DE9804C9A46934670B491E8E1
:109BD000380007C831EA400C48BF34EA430C03D5CB
:109BE000FFF7E6FDFFF780FFF0BCBDE8008C2DE934
:109BF000804C9A46934670B491E8380007C810F03C
:109C0000804F08BF13F0804F03D100F005F8FFF735
:109C10006BFFF0BCBDE8008C20F07F4780EA0300BA
:109C200023F07F4C07EB0C03A3F57C5300F00040BE
:109C3000A3F1FE0392F0000F00F0B38095F0000F47
:109C400000F077802DE901494FEA11404FEA1446B0
:109C500021EA004800FB06FC24EA064708FB06F65A
:109C600007FB08F800FB07F718EB06484CEB164C0F
:109C70004FEA124B18EB07484FEA15464CEB1740DA
:109C800022EA0B4E0BFB06FC25EA06470EFB06F606
:109C900007FB0EFE0BFB07F71EEB064E4CEB164CBC
:109CA0004FF000061EEB074E4CEB174B18EB0B0862
:109CB00040F1000018EB0E0B58EB000840F10000DB
:109CC0008F1A4FF000013CBFC943661B14BFB5EBB0
:109CD000040C00213CBFC943F61B4FEA17444EEA6F
:109CE0008E0E27EA04454FEA1C4704FB07622CEA64
:109CF000074C05FB07F70CFB05F604FB0CFC16EB09
:109D0000074642EB174216EB0C4642EB1C421BEB9C
:109D1000060658EB0202414146EA9E0601D5BDE81F
:109D20000189B619524141EB0101A3F10103BDE8DC
:109D300001894FEA14454FEA114724EA054621EA12
:109D4000074C05FB07F406FB07F70CFB06F105FBC8
:109D50000CFC11EB074144EB17444FEA124711EB9F
:109D60000C4144EB1C4422EA074C05FB07F206FBBE
:109D700007F70CFB06F605FB0CFC16EB074642EB5F
:109D8000174216EB0C4642EB1C456A1854F10001D1
:109D900048BF7047B619524141EB0101A3F10103DD
:109DA000704795F0000F37D04FEA11424FEA144741
:109DB00021EA024624EA074C02FB07F106FB07F7FB
:109DC0000CFB06F402FB0CFC14EB074441EB1741BF
:109DD0004FEA154714EB0C4441EB1C4125EA074CB4
:109DE00002FB07F506FB07F70CFB06F602FB0CFC73
:109DF00016EB074645EB174516EB0C4645EB1C42A8
:109E0000121951F1000148BF7047B619524141EB98
:109E10000101A3F1010370474FEA14454FEA1147CE
:109E200024EA054621EA074C05FB07F106FB07F784
:109E30000CFB06F24FF0000605FB0CFC12EB074290
:109E400041EB174112EB0C4251EB1C4148BF7047EC
:109E5000921841EB0101A3F101037047490050EA58
:109E6000C12018BF04204A0D18BF40F0010040F285
:109E7000FF72B2EB515F08BF40F00200012808BF3B
:109E8000052070472DE9F0414F1E00EBC701044645
:109E9000D1E9000115461E4637F006020DD02A46CC
:109EA000334601F0DDFA7F1E04EBC703D3E900233C
:109EB00000F0C2FF37F00602F1D1022F25D0042FA7
:109EC00013D0062F18BFBDE8F0812A46334601F0B3
:109ED000C7FAD4E90A2300F0AFFF2A46334601F05F
:109EE000BFFAD4E9082300F0A7FF2A46334601F061
:109EF000B7FAD4E9062300F09FFF2A46334601F063
:109F0000AFFAD4E9042300F097FF2A46334601F064
:109F1000A7FAD4E9022300F08FFF2A46334601F066
:109F20009FFAD4E90023BDE8F04100F085BF0000AE
:109F3000002213461046014901F03AB80000F03FF4
:109F4000012201F058BE00F077BF002213461046F0
:109F5000114601F02DB840F2013200204FF0E041EF
:109F600001F049BE024A0020110701F044BE000082
:109F700001FDFFFF30380A2801D201207047002080
:109F8000704700002DE9F041C1F30A52A2F2FF36FA
:109F90002F4A304B0D460446142E2FDA002E12DACB
:109FA00000F04AFF0022134601F058FB4CD2002D6E
:109FB000A4BF0024254647DA25F00040204318BFFF
:109FC000254D41D018E0DFF894C02CFA06F705EAD9
:109FD000070C5CEA040C08BFBDE8F08100F02CFF20
:109FE0000022134601F03AFB2ED2002D03DA4FF483
:109FF0008010F0400544BD43002425E0332EC8BF47
:10A00000BDE8F081A6F1140C4FF0FF3727FA0CF7EA
:10A010003C4208BFBDE8F08101F056FB0022134628
:10A0200001F01CFB10D2002D0DDA142E08BF6D1CA0
:10A0300009D0C6F13400012101FA00F02044A04209
:10A0400038BF6D1C0446BC4329462046BDE8F0815C
:10A050009C7500883CE4377E0000F0BFFFFF0F00D6
:10A060002DE9F04DC84A002490B0914205DA21F064
:10A070000043934201D805D120B110B0BDE8F04DA6
:10A08000FFF75EBFB1F5801F1BDA53EA000209D06B
:10A09000002911DA0120FEF722FC10B0BDE8F04DD6
:10A0A000FFF753BF0220FEF71AFCFFF741FF10B085
:10A0B00081F00041BDE8F08D6FF03504362201F0EB
:10A0C0009AFD04EB2152C1F31308B049A2F2FF3309
:10A0D000414401F4801282F07F6103EB225281F04F
:10A0E0004051009241EA08010022A94B01F0DEFB39
:10A0F000044608F10200A74EC0F313000D467E444B
:10A10000032867D2D6E90023204601F0A9F81ED122
:10A110000098002802BFD6E9000110B0BDE8F08D1C
:10A1200001F037F907460C469B4A9C4B01F098F921
:10A1300006460D469A4A9B4B3846214601F090F957
:10A1400010B032462B46BDE8F04D00F075BE4FF022
:10A150005532954B2046294601F082F90022934B57
:10A1600001F0B2FA06460F4622462B461046194623
:10A1700001F076F932463B4601F072F90646009846
:10A180000F46F0B101F005F980468A46824A834BBA
:10A1900001F066F932463B4601F096FA22462B461C
:10A1A00001F084FB05460C467D4A7E4B40465146F5
:10A1B00001F056F910B02A462346BDE8F04D01F0F3
:10A1C00075BB0B4610B0324620462946BDE8F04D1F
:10A1D00001F06CBB00224FF08043204600F02CFEC3
:10A1E00002460B462046294600F0E2FE06460F4690
:10A1F000009801F0CEF8CDE9040132463B46104606
:10A20000394601F02DF90C9069480C9A40440190B0
:10A2100009910B46104601F023F982460246654833
:10A220008B46C8F151080B4608F5D728032178441E
:10A23000FFF728FE52465B4601F012F90A905E488D
:10A240000D9152465B4604217844FFF71BFE099BA3
:10A250000C9A01F005F9844601980D9B40EA080824
:10A2600060460A9A00F0E8FD83460891B8F1000FB5
:10A270004EDD4FF0FF322046294601F0BCFC22465D
:10A280002B4601F0EDF8804600988A4660B3DDE980
:10A290000401414A414B01F0E3F8099100905A460C
:10A2A00040465146089B00F0C7FD32463B4601F050
:10A2B000D7F8099B009A00F0BFFD4246534601F0D3
:10A2C00003FA22462B4601F0F1FA04460D46DDE979
:10A2D0000401334A334B01F0C3F810B022462B4639
:10A2E000BDE8F04D01F0E2BA5A464046089B00F046
:10A2F000A3FD32463B4601F0B3F84246534601F017
:10A30000E3F910B022462B46BDE8F04D01F0DCB970
:10A31000009840B3DDE904011F4A204B01F0A0F88A
:10A3200080468A465A4620462946089B01F0BEFAD6
:10A3300032463B4601F094F84246534601F0B6FAE5
:10A3400022462B4601F0B2FA04460D46DDE904012F
:10A35000134A144B01F084F810B022462B46BDE896
:10A36000F04D01F0A3BA0B465A462046294601F0AB
:10A370009DFA32463B4601F073F810B022462B4658
:10A38000BDE8F04D01F0A0B90000F07F645F090066
:10A390000000F03F8E310000763C7935EF39EA3D20
:10A3A0000000E0FE422EE63F5555D53F0000E03F5D
:10A3B00086EBF9FF9E2F00009C2F00002DE9F04D49
:10A3C0001D460C4698B0174621F0004123F000438B
:10A3D000002814BF4FF0010C4FF0000C0CEB440CA4
:10A3E000FE4A0CEB02064FEA620C66452BD33E0098
:10A3F00018BF012606EB45061644F94A964222D3B9
:10A40000F84A53EA070C02D0944205D148B918B073
:10A4100000201146BDE8F08D002808BF4FF0000C69
:10A4200001D04FF0010C0CEB440212F5001F0AD8CA
:10A43000002F14BF4FF0010C4FF0000C0CEB450245
:10A4400012F5001F07D918B03A462B462146BDE841
:10A45000F04DFFF778BD0022DFF88CA3002CB8BFC9
:10A46000534526DADFF884C36345A8BF022220DA09
:10A47000DFF870C39C451CDCDFF874C30CEB235C75
:10A48000BCF1140F08DDCCF1340627FA06FC0CFAF7
:10A4900006F6BE420DD108E05FB9CCF1140623FAEE
:10A4A00006FC0CFA06F69E4203D10CF00102C2F142
:10A4B000020251EA000C19D1002D17DA002C18BF46
:10A4C000022A01D0012A07D00220FEF708FA18B0AC
:10A4D000BDE8F04DFFF72CBD0220FEF700FAFFF7B4
:10A4E00027FD18B081F00041BDE8F08DB7F1000CF8
:10A4F0006CD1534525D104F1804212F5801201BF81
:10A5000000280020B74918B008BFBDE8F08DB54855
:10A51000884207DC002DA1BF6046294618B0BDE87F
:10A52000F08D07E0281E05DA80F0004118B0604683
:10A53000BDE8F08DAF497944D1E9000118B0BDE81C
:10A54000F08DDFF8A0C2634525D1002D1FDA19B1C7
:10A55000514512D1D8B909E0002840F0EC82A24A56
:10A56000214618B062F31E01BDE8F08D002021469F
:10A5700018B060F31E01BDE8F08D08DA18B023466C
:10A58000BDE8F04D02460020614600F011BD18B054
:10A590002146BDE8F08D514518DAB5F1804F0DD058
:10A5A000A5F1005CBCF1FF5C10D1B4F1000C0DDB37
:10A5B00018B06146BDE8F04D00F0ECBB234618B082
:10A5C0000246BDE8F04D194600F04ABF060024F0EF
:10A5D000004C3BD1D9B1514533D1002C06DD002DC3
:10A5E000A1BF0020514618B0BDE8F08D002C01DD60
:10A5F000002D1BDB002C13DA002D11DB012A4FF09C
:10A60000000014BF78497C4918B0BDE8F08D022ADB
:10A6100018BF002C0AD0012A08D1002C06DA0AE063
:10A62000002CB8BF002D11DA012A04D0002018B088
:10A630000146BDE8F08D18B000204FF00041BDE8A4
:10A64000F08DA1F14050B0F17F601AD0012000EBF5
:10A65000E47050EA020421D0624C521E4FF0000B0D
:10A66000104304BF4FF0000B644C654883427CDD0F
:10A67000644A654893421FDD884217DB002D25DBC5
:10A6800037E0002C00DA4AB1022A0CBF01204FF05B
:10A69000FF3018B0BDE8F04D00F07BBE0120FEF7A2
:10A6A0001EF918B0BDE8F04DFFF74FBC4D4A8A4285
:10A6B00002DC002D0ADC1CE0814202DA002D18DAEF
:10A6C00004E0484B994220DD002D12DD0220FEF708
:10A6D00006F9FFF740FC05460E4600225346584651
:10A6E000214600F0BDFE18B066F31E012846BDE805
:10A6F000F08D0220FEF7F3F8FFF734FC0A462146FE
:10A7000018B062F31E01BDE8F08D002230466146AC
:10A7100001F0CCF880460E466FF0010201F06BFAB2
:10A720004FF05532394B00F0CFFF4246334600F030
:10A7300097FE0022364B00F0C7FF82464246334662
:10A7400004911046194600F08BFE5246049B00F01F
:10A7500087FE8A4600904FF0C0422E4B404631465D
:10A7600000F07EFE2C4A2B4B00E027E0CDE90601ED
:10A770005146009800F074FE82460191274A284B0A
:10A780004046314600F06CFE5246019B01F08EF8C7
:10A7900082460B4602460591DDE9060100F04CFBBE
:10A7A000DDE9062300268846304601F07FF8524650
:10A7B000059B00F089FF024600F07EB90020B1F54C
:10A7C000801F07DA35223046614601F014FA06464A
:10A7D0006FF0340000EB215024E00000FFFF1F0069
:10A7E000FFFF0F000000F03F0000F07F000040433B
:10A7F00001FCFFFF562D00000000F0FF0000F0BF3D
:10A800000000E0410000F043FFFFEF3F5555D53F0A
:10A810000000E03F4715F73FFE822B6544DF5DF8FF
:10A820000BAE543EA0F2FF300190C1F3130040F094
:10A830007F6141F040510291FE498842D8BF00201B
:10A8400004DDFD498142C8BF012001DD0D9008E013
:10A8500000200D900198401C01900298A0F58010F6
:10A8600002900299F54878440B910D9900EBC100D4
:10A87000D0E900230F9330460A920B9901F016F8A5
:10A88000CDE90601DDE90A2130460F9B00F0D4FA3C
:10A8900002460B460020EA4900F08AFB0591024679
:10A8A0000B460090DDE9060100F0DAFD1490E54862
:10A8B0008A464FF0000878440299006812904FF0E1
:10A8C000005040EA61010D980F9B01EB804000F5BC
:10A8D000002109910A9A129800F0E8FF32460B9B7A
:10A8E00000F0F2FE4246534600F0BAFD06460291E1
:10A8F00040465146099B129A00F0B2FDDDE906235D
:10A9000000F0E2FE3246029B00F0D0FF059B009A69
:10A9100000F0A6FD0091149A049053461046194683
:10A9200000F09EFD06460246C7480B4602910621EE
:10A930007844FFF7A7FACDE90510029B324610468E
:10A94000194600F08DFDDDE9053200F089FD059125
:10A950000646534640461946149A00F06DFA009B8D
:10A96000049A00F07DFD3246059B00F065FACDE9C2
:10A970000510424653461046194600F071FD00226C
:10A98000B24B02910A9000F057FADDE9053200F06F
:10A9900053FA0E464246AD4B404600F087FF029BFD
:10A9A0000A9A00F083FFDDE9053200F08DFE424691
:10A9B00002910A9033461046514600F051FDCDE910
:10A9C00006015346149A02990A9800F049FD8A46F6
:10A9D0000290334642460099049800F041FD5346E8
:10A9E000029A00F029FA82460B4602460591DDE9FB
:10A9F000060100F021FADDE906230020884606461C
:10AA000000F054FF5246059B00F05EFE824609911D
:10AA10004FF060428E4B3046414600F021FD0490DD
:10AA200006918C4A8A4B5046099900F019FD8246DE
:10AA30000291894A894B3046414600F011FD524649
:10AA4000029B00F0F9F9864B7B440D9A03EBC2039D
:10AA5000D3E9002300F0F0F90E900791019800F07F
:10AA600098FC0591DDE9061382460E9A049800F0E1
:10AA7000E3F97C4A7A440D9B02EBC303D3E900233C
:10AA80000093029200F0D8F95246059B00F0D4F9E9
:10AA90000026884652463046059B00F007FF009B83
:10AAA000029A00F003FF069B049A00F0FFFE079B4A
:10AAB0000E9A00F009FE024600200B46029038462E
:10AAC000294600F0CDFC824601912B4638461946B6
:10AAD000029A00F0EBFE3246434600F0C1FC5246BB
:10AAE000019B00F0A9F907468A46324643462946AB
:10AAF000029800F0B5FC05460E463A46534600F073
:10AB00009BF9594A8846914221DBA8EB020353EA9C
:10AB1000000210D12A46334600F0C8FECDE90401F8
:10AB2000524A534B3846514600F086F9DDE904237A
:10AB300000F094FD21D20220FDF7D1FEFFF70BFAC1
:10AB40000A46214618B062F31E01BDE8F08D494B5C
:10AB500028F000429A4210D3474A08EB020353EA16
:10AB600000027FF4C6AD2A46334600F09FFE3A4607
:10AB7000534600F073FD7FF6BCAD0022019228F031
:10AB800000403E493E4A01EB2051824223DA481CF4
:10AB90004FF4801121FA00F040443A4AC0F30A51C0
:10ABA0007A44394BA1F2FF31CB4020EA0303C0F3D2
:10ABB000130040F48010C1F11401C84012680190E4
:10ABC000B8F1000FBCBF404201902846314600F06A
:10ABD0006DFE05460E462A4633463846514600F07D
:10ABE0002BF94FF000084246284B4046059100F0F3
:10ABF00037FCCDE90601264A264B4046059900F070
:10AC00002FFC009102902A4633464046059900F0F9
:10AC10004DFE3A46534600F057FD1F4A1F4B00F0C9
:10AC20001FFC009B029A00F007F90746884602467F
:10AC30000B4635E08E9803007AB60B009E29000083
:10AC40000000F03FD6290000042900000000084061
:10AC500009C7EE3FFD033ADCF5015B14E02F3EBE71
:10AC6000DC270000A027000000009040FE822B653A
:10AC70004715973C00CC904000346F3F01FCFFFF2C
:10AC80000000E03FEC260000FFFF0F00432EE63FF0
:10AC9000396CA80C615C20BEEF39FAFE422EE63F0B
:10ACA000DDE9060100F0C8F8DDE9062305460E4699
:10ACB00000F0FCFD3A46434600F006FD0F462A46EA
:10ACC000334600901046194600F0CAFB8246024601
:10ACD0002E4888460B4605217844FFF7D3F85246A4
:10ACE000434600F0BDFB2A46334600F0EDFC8046AB
:10ACF0008A463B4628463146009A00F0B1FB3B4667
:10AD0000009A00F099F80691009000224FF08043DD
:10AD10004046514600F0CAFD0F460C90424653464D
:10AD20002846314600F09CFB3B460C9A00F040F967
:10AD3000069B009A00F0BAFD2A46334600F0B6FDA5
:10AD40000022134B00F0C0FC054601980E4601EBB3
:10AD500000510815002810DC28463146019A00F001
:10AD60004AFFFFF77BF8042808BFFFF7FBF82846E7
:10AD70003146019A00F03FFF05460B4618B02A46BF
:10AD800058462146BDE8F04D00F06ABB8C25000016
:10AD90000000F03F2DE9F04106460F4600F0A0FC10
:10ADA000041E0D4618BF0120284320F00040C0F1CA
:10ADB0007F6000F1E040C00F0ED0301C18BF0120B2
:10ADC000384320F00040C0F17F6000F1E040C00F48
:10ADD00004BF0120FDF783FD20462946BDE8F08130
:10ADE00010B500290AD00878002807D00548784413
:10ADF000FEF72CFC002801D0002010BD024878444A
:10AE000010BD0000062B0000FE2A000010B500292E
:10AE10000AD00878002807D005487844FEF716FCC9
:10AE2000002801D0002010BD0248784410BD000069
:10AE3000EA2B0000E22B000010B591EA030F48BF97
:10AE400083F0004300F13A85841A71EB030C05D2BC
:10AE5000121943EB0C03001B61EB0C01DFF824E13A
:10AE60004FEA1154A4EB135C1EEA430F18BF9EEA8D
:10AE7000445F73D023EA0E03DCF1200E21EA045173
:10AE800043F4801332D322FA0CFE10EB0E0023FAA7
:10AE90000CFE41EB0E01CCF1200E03FA0EFE10EB7E
:10AEA0000E0051F10001B1F5801FCCF1200E32D21D
:10AEB00001EB045112FA0EF2BDE8104058BF704782
:10AEC000401C38BF5FEA420218BF7047002814BF19
:10AED00020F0010041F100014FEA410313F5001F8A
:10AEE00038BF7047A1F1C04100F0B2BB012A43EB6B
:10AEF0000302ACF1200CDCF11F0E32BF4FF0000E4C
:10AF000023FA0CF310EB030041EB0451B4EB115F97
:10AF1000D0D0A1EB045101F5801149085FEA30005F
:10AF200001EB04510ED350F1000038BF12FA0EFEAF
:10AF300008D1BDE81040C9E7401C38BF5FEA4202B3
:10AF4000CAD1C3E7BDE810404FEA410313F5001F23
:10AF500038BF7047A1F1C04100F07ABB9EEA445F60
:10AF600008D011EA5E0FBDE8104004BF01F00041B7
:10AF700000207047BDE8104070B500F01BFB00BF1B
:10AF800064FBBE3E0000E0FF02494FF0000000F00D
:10AF900000BE00BF0000F87F491058BFC1F140411A
:10AFA0005B1058BFC3F140438B42EFF30080704702
:10AFB0002DE9C04130B4DFF8A0C23CEA111418BF3B
:10AFC0003CEA131400F0EC8081EA03051CEA11143A
:10AFD00044EAD57418BF1CEA131500F0C780A4EB2F
:10AFE00005044FF0004545EAC12145EAC32341EA83
:10AFF000505143EA525304F17F74994204F50034EE
:10B000004FEAC0204FEAC22208BF904200F09C8065
:10B010004FEA13650FF24016765D4FEA134506FBC3
:10B0200005F7C7F1807706FB07F74FEAD737A7FB8D
:10B0300003687642C8F58038A7FB06CE38BFA8F172
:10B04000010807FB08E64FF0000EA6FB028CE6FBAA
:10B0500003CEDCF1000CCEF1004E38BFAEF1010E94
:10B06000A6FB0C584FF000074FF00005E6FB0E87DB
:10B07000A1FB08C6A0FB07CE16EB0E0645F10005A6
:10B08000E1FB076515F1E04E7EBFA4F580345FEA71
:10B0900046066D4116F1800745F100054FEA172776
:10B0A0004FEA066647EA0567A6F1DE46B6F1805F1D
:10B0B0004FEA15251FD9384624F0010C05EBC47161
:10B0C000BCF1FE6F01EB0C1102D8F0BCBDE80081B1
:10B0D00024425CBF01F5801E9EEAC47F02D4F0BC0E
:10B0E000BDE80081244238D4F0BCA1F1C041BDE8E4
:10B0F000004100F0ADBA4FEAD22242EA43524FEA91
:10B10000D323A7FB02864FEAD02040EA415007FB39
:10B1100003661EEA0E0F4FEAD12105FB026658BFF7
:10B12000A6EB0056B6EB00564FEA520E4EEAC37E2F
:10B1300018EB0E0E56EB530EBDD518EB02085E4110
:10B140007F1C55F10005B6E74FF480154FF000075E
:10B150004FF000064FF00008ADE7F0BC4FF00000E4
:10B1600001F1C04101F00041BDE8008111EA0C1F6E
:10B170000CEA131500D00CE013EA0C1F00F0258038
:10B180004FF00000F0BC81EA030101F00041BDE88E
:10B190000081F0BCBDE8004181EA030100F058BA2B
:10B1A000F0BCBDE8004170B500F004FA097EFC3E39
:10B1B00000F007B881EA03014FF0000001F0004100
:10B1C000704781EA030100F043BAF0BCBDE80041DA
:10B1D0004FF0000021497047FFFDFBF9F7F5F4F24D
:10B1E000F0EEEDEBE9E8E6E4E3E1E0DEDDDBDAD822
:10B1F000D7D5D4D3D1D0CFCDCCCBCAC8C7C6C5C480
:10B20000C2C1C0BFBEBDBCBBBAB9B8B7B6B5B4B396
:10B21000B2B1B0AFAEADACABAAA9A8A8A7A6A5A481
:10B22000A3A3A2A1A09F9F9E9D9C9C9B9A99999845
:10B230009797969595949393929191908F8F8E8EE8
:10B240008D8C8C8B8B8A8989888887878685858475
:10B2500084838382828181800000FF070000F87F61
:10B2600051EA030C17D41CF5801F58BFBCF5801F92
:10B2700000F10680994218BF704708BF904270479E
:10B2800007D711F5801F58BF13F5801F19D49942B5
:10B290007047894270471CF5801F08D5BCF5801F98
:10B2A000F7D58B4218BF704708BF824270474FF4F2
:10B2B000001C1CEB410F38BF1CEB430F01D28B422B
:10B2C000704770B500F076F9922449004FF00051B4
:10B2D0004FF08053FFF760BE4FEA41034FEA5353EC
:10B2E000A3F58063D3F11E03C8BFD3F1210C0CDD9D
:10B2F0004FF0004242EAC12242EA505232FA03FCC5
:10B300008CEAE17CACEBE1707047102BC4BF0020ED
:10B31000704703F5787CBCF1FF3F04D06FF000422A
:10B3200082EA2100704770B500F044F94992248008
:10B3300000207047F2E700004FEA1153A3F5806345
:10B34000D3F11E03A8BFD3F1200C08DB4FF000425D
:10B3500042EAC12252EA505232FA03F070470942DF
:10B360000BD4102BC4BF0020704703F5787CBCF1D0
:10B37000FF3F05D04FF0FF3070474FF0000070479F
:10B3800070B500F017F900BF499224800020704783
:10B39000F0E710F0004248BF4042B0FA80F310FAE4
:10B3A00003F10AD0C3F11D0303F580634FEA415056
:10B3B00002EB035202EBD12170474FF000007047BF
:10B3C000B0FA80F310FA03F10AD0C3F11D0303F5BC
:10B3D00080634FEA41504FEA035202EBD12170479C
:10B3E0004FF000007047000051EA030C17D41CF521
:10B3F000801F58BFBCF5801F00F10680994218BF1E
:10B40000704708BF9042704707D711F5801F58BF9B
:10B4100013F5801F19D499427047894270471CF573
:10B42000801F08D5BCF5801FF7D58B4218BF704729
:10B4300008BF824270474FF4001C1CEB410F38BF1D
:10B440001CEB430F01D28B42704770B500F0B2F88D
:10B45000922449004FF000514FF08053FFF79CBDFC
:10B46000DFF848C170B51CEA111E1EBF1CEA131597
:10B470009EEA0C0F95EA0C0F00F06F8081EA03043E
:10B4800023EA4C134EEAD47E21EA4C1141F4801198
:10B4900043F48013AE44A1FB024CA0FB0365AEF164
:10B4A0007F7E361955EB0C05A1FB034C4CF10003D4
:10B4B000A0FB021C16EB0C06654153F10003094288
:10B4C00018BF46F0010613F4007F0BD14FEA033199
:10B4D0004FEA0530340341EA155140EA16506FF047
:10B4E00003020AE04FEAC3214FEAC520F40241EA11
:10B4F000555140EA56506FF0020202EB2E4201EB2A
:10B50000025585EACE710AD05FEA440C18BF24F0D8
:10B51000004450F1000041F1000120EAD47040F2F3
:10B52000FE7C624500D270BDA84214BF4FF080443B
:10B530004FF04044002E08BF0024BEF1806FA8BF2A
:10B54000A1F1C041BDE8704080F282804FF0000060
:10B5500001F1C04101F0004170479EEA0C0F0CEA76
:10B56000131518BF95EA0C0F06D04FF0000081EAC2
:10B57000030E0EF0004170BD00F01CF88900013E82
:10B5800000F007B800F009B84FEA430C5FEA5C5CD2
:10B5900008D081EA030100F05BB84FEA410C5FEA92
:10B5A0005C5CF6D14FF00000014970470000FF07D6
:10B5B0000000F87F0EF1020E2EF0030E5EF8046B11
:10B5C000364205D4012A43EB030515F5001F12D8B6
:10B5D000012841EB010C1CF5001F0CD80ED14FEADD
:10B5E000D17C15F5001F0CEB4C0C0CF1020C08BFC4
:10B5F0004CEBD37C04E04FF0080C01E04FEAD37C25
:10B600000CEB4C0526FA05F606F00706B6F1040C1D
:10B6100006D20EEB860CBDE870404CF0010C604782
:10B62000DFE80CF0090B02024FF000414FF0000080
:10B63000A1F5002170BD19461046012851EB010407
:10B6400018BFD4F5001484BF002001F0004170BD84
:10B650000808A0F500114FEA3101704753EA010CC8
:10B6600017D41CF5801F58BFBCF5801F00F1068061
:10B670008B4218BF704708BF8242704707D713F547
:10B68000801F58BF11F5801F19D48B4270479B4211
:10B6900070471CF5801F08D5BCF5801FF7D599426F
:10B6A00018BF704708BF904270474FF4001C1CEB56
:10B6B000430F38BF1CEB410F01D2994270470FB4C2
:10B6C0000CBC03BCFFF7C1BE91EA030F10B581F0BB
:10B6D00000413FF5B9AB83F0004300F0EFB8000044
:10B6E0002DE9F04101F5801CBCF5001FC0F2C380BC
:10B6F0004FEA115C21EA0C510CF1FD0C41F4801170
:10B700005FEA5C0C0CF5C07C01D3400049413DA4CC
:10B71000890241EA905187028E0E0A0CA45D04FB57
:10B7200004F602FB06F6C6F14046A4FB0662F60DDF
:10B7300046EA422606FB06F4A4FB01235242C3F16B
:10B74000404338BF5B1EA6FB02420024E6FB0324F5
:10B75000D20B42EA4446A6FB0623A1FB02E2A3FB6E
:10B7600007E4A4184FF0000252F10002E3FB01428B
:10B770006442C2F1404E38BFAEF1010EA6FB042375
:10B780004FF00002E6FB0E32A2FB03464FF000042E
:10B79000B61954F10004E2FB0264A1FB06E6A4FB27
:10B7A00007E816EB08064FF0000858F10008E4FB24
:10B7B00001687642C8F1405838BFA8F10108A2FBE1
:10B7C00006E4A3FB08E52D194FF0000454F1000432
:10B7D000E2FB0854A1FB05E6A7FB04E818EB06080A
:10B7E0004FF0000656F10006E1FB048618F1200533
:10B7F00056F10006A809A8F11B08B10908F03F0896
:10B80000B8F10A0F40EA86601CD901EB0C51BDE883
:10B81000F08100BFFCF5EEE8E2DDD8D3CFCBC7C3A3
:10B82000C0BDB9B6B4B1AEACA9A7A5A3A19F9D9B5D
:10B830009A9896959392908F8D8C8B898887868520
:10B8400084838281A0FB006800FB01F208EB4208C0
:10B85000B8EB872807D5341858EB0104D5D5401C20
:10B8600051F10001D1E7341A78EB0104CDD4401E28
:10B8700071F10001C9E75FEA4C0C5FEA9C5C0DD1F5
:10B8800005D34FF0000001F00041BDE8F081BDE8B4
:10B89000F04170B5FFF78EFE6DDBFFBEBDE8F041F5
:10B8A0004FF00000004970470000F87F10B591EAA2
:10B8B000030F48BF83F000433FF5C6AA841A71EB1B
:10B8C000030C07D212198CF0004C43EB0C03001B45
:10B8D00061EB0C01DFF8A4E14FEA1154A4EB135C17
:10B8E0001EEA430F18BF9EEA445F00F0B08023EACF
:10B8F0006E03524221EA0451C3EB6E0338BF5B1E54
:10B90000DCF1200E25D322FA0CFE10EB0E0043FAD8
:10B910000CFE41EB0E01CCF1200E03FA0EFE10EBF3
:10B920000E0051F10001CCF1200E29D412FA0EF2D2
:10B9300001EB0451BDE8104058BF7047401C1CBFCC
:10B94000B2F1004F704700280CBF491C20F00100E5
:10B95000704712EB020E43EB030218BF4FF0010ECB
:10B960004EEA4202ACF1200CDCF11E0E54D943FA2F
:10B970000CFE10EB0E0051F1FF31CCF11E0ED5D5AF
:10B980000EF1010E12FA0EFE404141EB010101EBF6
:10B99000445C5FEA5C5C10D910EBDE7001EB045193
:10B9A00038BFBEF1004FBDE8104018BF70470028F7
:10B9B0000CBF491C20F00100704730D24FEAD42C54
:10B9C00011F5001124F400641BD0B1FA81F20B3A96
:10B9D000A41AA41ED2F12003914030FA03F31943B4
:10B9E000904001EBCC71002C01EB0451BDE81040FC
:10B9F000A8BF704701F1C0414FF0000001F00041C5
:10BA00007047B0FA80F310FA03F100D110BDE41AC8
:10BA1000173C4805C90AE4E701EB045110BD491081
:10BA200001EB0451BDE810404FEA300002E04FF056
:10BA3000000170474A0008BF0042F8D0B2F5001F6D
:10BA400028BF704701F000414FF0000070479EEAA8
:10BA5000445F07D011EA5E0FBDE8104004BF00212B
:10BA600000207047BDE8104070B5FFF7A3FD00BF90
:10BA700040DFF63E83F00041104670470000E0FFD3
:10BA800043004FEAD30C4FEA3C0C43401FBF400732
:10BA90000CF1605113F0FE4F70471CF0006F03D1A2
:10BAA00000200CF0004170470CF0004343EA507056
:10BAB00010B540EACC0000F022F800BF0000009270
:10BAC0004FEA0001FFF7C4BD4FF000414FF0000006
:10BAD000A1F5002170470000B0FA80F310FA03F2DC
:10BAE000C3F19D030AD0D90501EB1220530638BFDC
:10BAF000704700F1010008BF20F0010070470EF10F
:10BB0000020E2EF0030E5EF8044B244204D44FEADA
:10BB10004102B2F17F4F11D84FEA4003B3F17F4F9A
:10BB20000CD80ED14FEAD07CB2F17F4F0CEB4C0C0D
:10BB30000CF1020C08BF4CEBD17C04E04FF0080C78
:10BB400001E04FEAD17C0CEB4C0324FA03F404F03F
:10BB50000704B4F1040C06D20EEB840CBDE81040CF
:10BB60004CF0010C6047DFE80CF0070802024FF0D0
:10BB70000040A0F5800010BD0846420018BFD2F179
:10BB8000807288BF00F0004010BDFCF7E0BFFDF7F9
:10BB90007FBA0CF00F03092B08BF082000F0598072
:10BBA0000A2B0BD0082B18BF704708BF1CF0400FA2
:10BBB0000AD04FF000004FF0000170471CF0400F1A
:10BBC00018BF4FF0004070471CF0100F08D020F055
:10BBD000704300F07F4242EAD3014FEA437070475E
:10BBE00000F0604021F07F4242EA000201F07F4015
:10BBF00040EA727070474FF0FF0C4CF4E06C1CEAA6
:10BC000011531CBF9CEA030C9445C2BFDA4201EBFE
:10BC100002517047002B0DD0BCF1000F0FD0002A4D
:10BC200001F00041A4BF41F0E04141F07F614FF0DD
:10BC30000000704701F000414FF00000704750EAEB
:10BC400001334FF09B0C18BF4CF0806C7FF49CA923
:10BC500070471CF4801F11D01CF4E02F03D06FEA52
:10BC6000CC31490070474FF04050EFF3008222F092
:10BC7000704242EA000282F3008870474FF00000F1
:10BC800070470103070F1FFFFF1F0F07030100008D
:10BC9000000000E0E00000FCFC00000000000000EC
:10BCA000000000000000003F3F0000383800003F67
:10BCB0003F00003F3F00003F3F0000000000000049
:10BCC00000000103070F1FFFFF1F0F070301000004
:10BCD000000000E0E00000000000000000000000A4
:10BCE000000000000000003F3F0000383800003F27
:10BCF0003F00003F3F000000000000000000000087
:10BD000000000103070F1FFFFF1F0F0703010000C3
:10BD10000000000000000000000000000000000023
:10BD2000000000000000003F3F0000383800003FE6
:10BD30003F000000000000000000000000000000C4
:10BD400000000000F808E8E8E8E80808E8E8E8E8A3
:10BD50000808E8E8E8E80808F820E000000000002B
:10BD6000000000001F1017171717101017171717CC
:10BD700010101717171710101F04070000000000FD
:10BD800000000000C0E0F0F8FCC05F5555D57555C7
:10BD900055555FC0000809090B0505050B09090089
:10BDA00000EACC0011F200FC2424E41FE4856600C4
:10BDB00000070A0700020B0403040E00B3CF0012B1
:10BDC000D2FE5190122400FF80800001000F00007D
:10BDD0000101010F000000BFC6008888FF4824E46D
:10BDE000243F24E4040000080F00080805020508A9
:10BDF0000800BCBC000000000000000000000000C3
:10BE000000000000000000363600000000000000C6
:10BE10000000000000A3BA000000000000000000C5
:10BE20000000000000000000000058380000000082
:10BE30000000000000000000A3AC000000000000B3
:10BE40000000000000000000000000000018242492
:10BE50001800000000000000000000A1A300000086
:10BE600000FE0000000000000000000000000000D4
:10BE70000033000000000000000000000000A3A14B
:10BE800000000038340282C27C380000000000004C
:10BE90000000000000003737000000000000000034
:10BEA00000A3BF00008080BEAAAAAAEAAAAAAABECE
:10BEB00080800000048584945C54272424544C44DE
:10BEC00084050400EACC004042CC0000F888888851
:10BED00008FF0809CA080000003F90681F10209F53
:10BEE0004027182641F000B3CF002424A4FEA3224B
:10BEF0000022CC0000FF00000000080601FF000146
:10BF00000404040404FF02020200BFC60010101063
:10BF1000FF109008888888FF888888080004448279
:10BF20007F01808040432C102846818000BCBC00EB
:10BF30001010FF109000FE5252D25252525E00007A
:10BF400042827F8140308F929392FE92939680003E
:10BF5000CED50000002424242424FC2222222322E3
:10BF6000000000020202020242827F02020202027A
:10BF7000020200CAD6000000F010101010FF1010CE
:10BF80001010F000000000000F04040404FF04047B
:10BF900004040F000000D6D000000000000001E201
:10BFA0001CE000000000000000804020100C030096
:10BFB0000000030C3040808000C8EB0000FE02222D
:10BFC000428272022242827202FE000000FF1008CA
:10BFD00006010E100806014E807F0000CDF80040DB
:10BFE0004042CC000444645C47F4444444040000F0
:10BFF00040201F2044444444447F4444444400C1FE
:10C00000AC00101010FF1050445465C644645444F2
:10C0100040000444827F0182824A562322524E828B
:10C020000200BDD3000000FE222222FE00FE82821A
:10C0300092A29E000080601F0242827F00FF402F7C
:10C04000102C438000B7FE00000090884C57A424B9
:10C0500054548C840000000001018042221A07021F
:10C060004282423E01010100CEF10080809E929208
:10C07000929EE0809EB2D2929E80000808F4949234
:10C0800092F10001F2929494F80800C6F700106053
:10C09000028C0008080809FA0808080800000404CF
:10C0A0007E0140404141417F414141414000D7A292
:10C0B00000808080FE8282FE8080FE8282FE808000
:10C0C000000080403F00407F80601F40807F000074
:10C0D00000B2E1000000F8888888880808FF080995
:10C0E0000AC8080080601F0010201F804021161819
:10C0F0002641F800B3C900080808F808080810101D
:10C10000FF101010F000001030101F088848300E8B
:10C11000014080403F0000B9A6000040301E1010D2
:10C1200010FF101010101000000081814121110D2E
:10C130000301030D112141818100CAA70000FE0205
:10C14000FA02FE4020D8171010F01010008047307F
:10C150000F106780402116081621408000B0DC00D7
:10C16000080889EA1888000404FC040404FC0000A0
:10C17000020100FF0186402018074080403F000078
:10C18000B3F5001010F01F10F00040E05847405089
:10C1900060C0004022150816210000FE42424242C3
:10C1A000FE0000CABC00008060F807000000FF40ED
:10C1B000201008040000010000FF000402013F40BD
:10C1C000404040407800BBAF00040444C44F4444A6
:10C1D000C424242FB42404040040442424150C0453
:10C1E000FE040C152424444000B2CB000000F849A2
:10C1F0004A4C48F8484C4A49F80000001010131205
:10C20000121212FF1212121213101000B5A50040E4
:10C210004042CC0000FC24A4242222A3620000009F
:10C2200040201F205847504845424548504000B7DD
:10C23000B5000000FE0202F2121212F20202FE002B
:10C24000000000007F2020272424242720207F00B6
:10C250000000BBD800000022322AA6A262211109E8
:10C260008101000000004222130B42827E02020A7A
:10C270001223460000CFB5002030AC63300088C8E0
:10C28000A8998E88A8C888002267221212804030A0
:10C290000F00003F40407100CDB300808084848453
:10C2A000FE82838280FF8080808000008040201892
:10C2B0000700000000FF0000000000C9FD00203062
:10C2C000AC6330000202FE0202625AC6000022671E
:10C2D00022121240308F80432C102C438000BCB6B9
:10C2E0000008C8B88FE8888840300FC808281800B0
:10C2F0000008180808FF048440300E010E3040800A
:10C3000000C8ED00008060F80780601C1010FF106E
:10C3100010100000010000FF000202020202FF02F2
:10C3200002020200BCFE00004042445840407F40F0
:10C33000405048C600000000404444444444444443
:10C34000444444FF000000B5B1000808E8292E2845
:10C35000E80808C80C0BE80808000000FF09498934
:10C360007F00000F40807F000000C7B00000FE206B
:10C37000203F2000FC24E4242223E20000807F01EF
:10C3800001FF80601F8041261826418000B0E60032
:10C390000010101010D030FF30D01010101000001E
:10C3A00010080402090808FF080809020408100020
:10C3B000B1BE00808080BEA2A2A2A2A2A2A2BE8024
:10C3C00080800000000006050404044484443C000E
:10C3D000000000BAC500404042CC0040A09E8282CE
:10C3E000829EA02020000000003F908840432C1037
:10C3F000284641808000C9E800809090484C57242E
:10C400002424544C4480808000000000FF494949A6
:10C410007F494949FF00000000B1B800008060F882
:10C42000070004242425262424240400010000FFFE
:10C43000000000F94949494949F90000D0C5000008
:10C440000000FC54545655545454FC000000004065
:10C45000300003394141455941417300083000CF54
:10C46000A2000000007F494949494949497F00002D
:10C4700000008141211D214181FF898989898981AC
:10C480008100CAC70000028282422212FA062222DA
:10C490004242820000010100FC44444445444444BB
:10C4A000FC00000100B7F1000010109010101116F0
:10C4B000101010D01010000040404040435C40403D
:10C4C000504C434040404000C1A20000FE92929276
:10C4D00092FE0000FE020202FE0000003F20100A51
:10C4E00004180000FF000408070000BCB400003E70
:10C4F00022E2223E0010885724548C000000407E27
:10C50000403F22220001FE424242FE010100C2B72A
:10C5100000001088C43380824222121A26224080F2
:10C5200000020100FF00404242427E42424242403D
:10C5300000BEB6000484E45C44C400F29292FE9211
:10C5400092F2020002017F10103F808F54245F445A
:10C5500084878000D3B20000FE02FA02FE0080FF52
:10C5600080A090888680008047300F10670000FF11
:10C5700040230C10204000D5CB00808080BEA2A2BA
:10C58000A2A2A2A2A2BE8080800000000006050434
:10C5900004044484443C00000000BAC500108C44EC
:10C5A00004E40495A64424148444940C0002027A02
:10C5B000414143427E42424243F8000000C3DC0056
:10C5C0000484E45C44C40002F2828282FE80800023
:10C5D00002017F10103F00080808084888403F000B
:10C5E000C2EB00C808090EE808405E5050DF50500A
:10C5F0005E4000206F201C131000FE027F027E822E
:10C60000FE0000B6CB000000FC0404040404040493
:10C610000404FC00000000007F20202020202020B7
:10C6200020207F000000BFDA00404424A4948C84C2
:10C63000FF848C94A4244440004040405F4A4A4A0E
:10C640004A4A4A4A5F40404000B2E900404042CC7A
:10C650000020D04C4B48C80808F800000000007FBC
:10C6600020101F1212125F80403F0000D1AF004027
:10C670004042CC00202222A262222222200000007E
:10C6800040201F20444E4544444445464C4000D47D
:10C69000CB00001088C4330040424242C2424242B2
:10C6A0004000020100FF0000000040807F00000009
:10C6B0000000D0D0002030AC6320188082422212CB
:10C6C0001A26428000226722121212404242427E03
:10C6D0004242424000BEAD002030AC63201800084A
:10C6E0004848FF48484808002267221212120002F8
:10C6F0000202FF0212221E00CEB3000000FC24241E
:10C7000024FC252624FC242424040040308F80842B
:10C710004C55252525554C80808000B6C80020103A
:10C72000E824272424E424342C20E0000000806046
:10C730001F090909097F090949897F000000BDC750
:10C74000000808080808F8898E888888880808087A
:10C750000000804020180700004080403F0000009B
:10C7600000B7BD0000F808080CCA494848C80808C6
:10C7700008F8000000FF0000001F0808081F004024
:10C78000807F0000CFF200404042CC0004F494943B
:10C79000FF9494F40400000040201F2048444241CC
:10C7A0005F414244484000CBD900008060F8070454
:10C7B000E4A4A4BFA4A4E4040000010000FF4040DE
:10C7C0007F4A4A4A4A4A7F404000D6B50004444462
:10C7D000445F44C44444445F44C404040000000073
:10C7E000000000FF000008100807000000BDDA008C
:10C7F00000F2929292929E00F2929292929E000089
:10C800000010114A88443F0010114A88443F00003C
:10C81000C8F5000000000000000000002F0000002C
:10C82000000700070000147F147F1400242A7F2AC9
:10C830001200626408132300364955225000000597
:10C8400003000000001C224100000041221C0000E7
:10C8500014083E08140008083E0808000000A06004
:10C8600000000808080808000060600000002010B0
:10C87000080402003E5149453E0000427F4000004E
:10C880004261514946002141454B31001814127F45
:10C8900010002745454539003C4A4949300001719F
:10C8A00009050300364949493600064949291E0051
:10C8B0000036360000000056360000000814224101
:10C8C0000000141414141400004122140800020182
:10C8D00051090600324959513E007C1211127C0068
:10C8E0007F49494936003E41414122007F41412272
:10C8F0001C007F49494941007F09090901003E4167
:10C9000049497A007F0808087F0000417F41000004
:10C910002040413F01007F08142241007F404040F9
:10C9200040007F020C027F007F0408107F003E4120
:10C9300041413E007F09090906003E4151215E0048
:10C940007F091929460046494949310001017F0103
:10C9500001003F4040403F001F2040201F003F405B
:10C9600038403F006314081463000708700807008C
:10C97000615149454300007F41410000552A552A35
:10C9800055000041417F00000402010204004040C4
:10C99000404040000001020400002054545478003C
:10C9A0007F484444380038444444200038444448D4
:10C9B0007F00385454541800087E0901020018A45E
:10C9C000A4A47C007F080404780000447D4000009B
:10C9D0004080847D00007F102844000000417F409B
:10C9E00000007C04180478007C08040478003844B3
:10C9F00044443800FC242424180018242418FC0083
:10CA00007C0804040800485454542000043F444067
:10CA100020003C4040207C001C2040201C003C406A
:10CA200030403C004428102844001CA0A0A07C00FA
:10CA30004464544C441414141414140000000000F2
:10CA40000000000000000000000000000000F800EE
:10CA5000000000000000333000000000100C061041
:10CA60000C0600000000000000000040C07840C03C
:10CA7000784000043F04043F040400007088FC0870
:10CA8000300000001820FF211E0000F008F000E038
:10CA900018000000211C031E211E0000F0088870F1
:10CAA0000000001E2123241927211010160E00005B
:10CAB0000000000000000000000000000000E0187E
:10CAC000040200000000071820400000020418E0E3
:10CAD0000000000040201807000000404080F08067
:10CAE0004040000202010F01020200000000F000BD
:10CAF0000000000101011F01010100000000000011
:10CB000000000080B0700000000000000000000085
:10CB1000000000000101010101010100000000000E
:10CB20000000000030300000000000000000008025
:10CB3000601804006018060100000000E0100808FA
:10CB400010E000000F102020100F00001010F8005F
:10CB50000000000020203F2020000000700808088E
:10CB60008870000030282422213000003008888896
:10CB70004830000018202020110E000000C02010B6
:10CB8000F8000000070424243F240000F8088888E7
:10CB90000808000019212020110E0000E0108888EC
:10CBA000180000000F112020110E0000380808C8DE
:10CBB0003808000000003F000000000070880808EE
:10CBC000887000001C222121221C0000E0100808AF
:10CBD00010E0000000312222110F00000000C0C050
:10CBE0000000000000003030000000000000800065
:10CBF0000000000000806000000000000080402075
:10CC0000100800000102040810200040404040408D
:10CC10004040000404040404040400000810204000
:10CC2000800000002010080402010000704808087D
:10CC300008F0000000003036010000C030C828E8CD
:10CC400010E0000718272423140B000000C038E070
:10CC5000000000203C23020227382008F88888883A
:10CC6000700000203F202020110E00C0300808086E
:10CC7000083800071820202010080008F8080808C5
:10CC800010E000203F202020100F0008F88888E8DE
:10CC9000081000203F20202320180008F88888E88A
:10CCA000081000203F200003000000C030080808E2
:10CCB00038000007182020221E020008F808000093
:10CCC00008F808203F210101213F20000808F8084A
:10CCD0000800000020203F2020000000000808F885
:10CCE000080800C08080807F00000008F888C02805
:10CCF000180800203F20012638200008F80800000E
:10CD0000000000203F20202020300008F8F800F824
:10CD1000F80800203F003F003F200008F830C00026
:10CD200008F808203F200007183F00E01008080816
:10CD300010E0000F10202020100F0008F80808084D
:10CD400008F000203F210101010000E01008080860
:10CD500010E0000F18242438504F0008F888888805
:10CD6000887000203F2000030C30200070880808E5
:10CD70000838000038202121221C00180808F80873
:10CD80000818000000203F2000000008F8080000FC
:10CD900008F808001F202020201F000878880000C5
:10CDA000C83808000007380E010000F80800F80035
:10CDB00008F800033C0700073C030008186880805F
:10CDC00068180820302C03032C30200838C800C80D
:10CDD0003808000000203F2000000010080808C8A4
:10CDE0003808002038262120201800000000FE020C
:10CDF0000202000000007F40404000000C30C000F4
:10CE0000000000000000010638C00000020202FE1F
:10CE1000000000004040407F0000000000040202CB
:10CE200002040000000000000000000000000000FC
:10CE300000000080808080808080800002020400EA
:10CE40000000000000000000000000000080808062
:10CE50008000000019242222223F2008F800808050
:10CE6000000000003F112020110E00000000808013
:10CE7000800000000E1120202011000000008080A2
:10CE800088F800000E112020103F200000808080D4
:10CE9000800000001F222222221300008080F088E0
:10CEA0008888180020203F2020000000008080801B
:10CEB000808000006B94949493600008F800808058
:10CEC000800000203F210000203F20008098980033
:10CED0000000000020203F2020000000000080987B
:10CEE00098000000C08080807F000008F80000806B
:10CEF000808000203F24022D302000000808F80028
:10CF00000000000020203F202000008080808080E2
:10CF1000808000203F20003F20003F8080008080F4
:10CF2000800000203F210000203F20000080808002
:10CF3000800000001F202020201F008080008080B3
:10CF400000000080FFA12020110E00000000808062
:10CF5000808000000E112020A0FF80808080008053
:10CF600080800020203F2120000100000080808080
:10CF70008080000033242424241900008080E08075
:10CF80008000000000001F202000008080000000C2
:10CF9000808000001F202020103F20808080000023
:10CFA00080808000010E3008060100808000800033
:10CFB0008080800F300C030C300F000080800080D8
:10CFC0008080000020312E0E312000808080000003
:10CFD00080808080818E70180601000080808080B3
:10CFE0008080000021302C222130000000000080D1
:10CFF0007C020200000000003F404000000000FFF3
:10D0000000000000000000FF0000000002027C8021
:10D010000000000040403F00000000000601010247
:10D020000204040000000000000000006001000095
:10D03000010000002000000020000000002C000083
:10D04000200000000306010B0405020925262734F1
:10D050003500000100010001000100000040000057
:10D0600000000200000004000000080000001000A2
:10D07000845700208458002084590020845A0020BE
:10D080000B0000000C0000000D0000000E0000006E
:10D090000F00000010000000110000003800000028
:10D0A000390000003A0000003B0000003B00000097
:10D0B000000102030405060004000000080000004F
:10D0C0001000000020000000400000008000000070
:10D0D0000001000001000200040008001000200010
:10D0E0004000800000010002000400080010002041
:10D0F00000400080000102030405060708090A0B2E
:10D100000C0D0E0F010000000200000004000000E2
:10D110000800000010000000200000004000000097
:10D120008000000000010000000200000004000078
:10D130000008000000100000002000000040000077
:10D1400000800000060708090A1717171717282874
:10D150002828282800030306010406020500030509
:10D160001F1C1F1E1F1E1F1F1E1F1E1F1C1D1E32C9
:10D17000363700000100000002000000040000003B
:10D180000800000010000000200000000000000067
:10D1900000000000303132333435363738394142FF
:10D1A0004344454640305800303132333435363709
:10D1B00038396162636465664030780004000008B5
:10D1C000000000000000000200010000100000004C
:10D1D00004FA97999999D93FAF788E1DC571CC3FC4
:10D1E0009FC678D0099AC33F935555555555E53F8D
:10D1F000599322942449D23FDE03CB966446C73F1D
:10D2000044523EDF12F1C23F000000000000F03F38
:10D21000000000000000F83F0000000000000000D7
:10D220000000004003B8E23F0000000000000000E2
:10D2300006D0CF43EBFD4C3E033333333333E33F70
:10D24000FFAB6FDBB66DDB3F4D268F515555D53F9C
:10D2500001411DA96074D13F65DBC9934A86CD3F6A
:10D26000EF4E454A287ECA3F3E5555555555C53F58
:10D2700093BDBE166CC166BF2CDE25AF6A56113F4A
:10D28000F16BD2C541BDBBBED0A4BE726937663E4C
:10D2900000000000000000003031323334353637F2
:10D2A00038396162636465667870003031323334D6
:10D2B000353637383941424344454658500000001E
:10D2C00002400000000000A0000000000540000037
:10D2D000000000C8000000000C4000000000409C5E
:10D2E00000000000194000000020BCBE000000004B
:10D2F00034400000BFC91B8E00000004B540000090
:10D30000504BCFD06607E2CF010000006C41000017
:10D310003E8251AADFEEA73401000000D94200008E
:10D32000DCB5A0E23A301F97FFFFFFFFB4450000D5
:10D33000FD25A0C8E9A3C14FFFFFFFFFFF3F00008D
:10D340000000008000000000FF3F0000000000809F
:10D35000000000000D0A2A2A2A2A2A2A2A2A2A2A12
:10D360002A2A2A2A2A2A2A2A2A2A2A2A2A2A2A2A1D
:10D370002A2A2A2A2A2A2A2A2A2A2A2A2A2A2A2A0D
:10D380002A2A2A2A2A2A2A2A2A2A2A2A2A2A2A2AFD
:10D390002A2A2A2A000000000D0AB0E6C8A8B9E926
:10D3A000CAF4203A20EACCB3CFBFC6BCBC2032308E
:10D3B00031372F382D323032372F38202E090909D6
:10D3C0000909090D0ABCBCCAF5D6A7B3D6203A2074
:10D3D0004D722E2057616E6720203133363335353C
:10D3E0003133363138202E002A4745542A204961EE
:10D3F00070466C61673A5B25635D21202052756E33
:10D400004170704E756D3A5B41505025635D21202F
:10D41000204A756D70526573756C743A5B25635D57
:10D42000212020426F6F74566572733A5B25735DDD
:10D43000212020417070566572733A5B25735D211F
:10D4400020204373713A5B25735D212020456332B0
:10D4500030566F6C3A5B25735D21202053696D490E
:10D46000636369643A5B25735D21202046747055BF
:10D470007365726E616D653A5B25735D2120204690
:10D48000747050617373776F72643A5B25735D21BA
:10D490002020467470466F6C6465723A5B25735D3C
:10D4A00021202046747049503A5B25735D2120206D
:10D4B00054637049503A5B25735D2120205463709A
:10D4C000506F72743A5B25735D210000B2CECAFDC5
:10D4D000B2BBBACFB7A82100C3FCC1EEB8F1CABD38
:10D4E000B4EDCEF321000000C3FCC1EEB2BBD6A761
:10D4F000B3D600007175616E2E73756E696E672EFE
:10D50000636F6D002F67657453797354696D652E71
:10D51000646F0000504F535420687474703A2F2F7A
:10D520002573257320485454502F312E310D0A4352
:10D530006F6E74656E742D547970653A6170706C9D
:10D5400069636174696F6E2F6A736F6E3B636861A4
:10D55000727365743D5554462D380D0A486F7374C7
:10D560003A25730D0A636F6E74656E742D6C656E6B
:10D570006774683A25640D0A0D0A257300000000DF
:10D580007B226D6163223A222573227D0000000018
:10D59000415445300D0A000041542B4342430D0ACB
:10D5A0000000000041542B51504F57440D0A000019
:10D5B00041542B474D520D0A0000000041540D0A02
:10D5C00000000000415426560D0A00004154265721
:10D5D0000D0A0000453A203000000000453A203195
:10D5E000000000002B434243000000004F4B0000AE
:10D5F000504F574552454420444F574E00000000BD
:10D600004552524F5200000041542B514943534759
:10D61000503D25642C312C222573222C22222C22D1
:10D62000222C310D0A00000041542B435245473D46
:10D63000320D0A0041542B43475245473D320D0AF3
:10D640000000000041542B435245473F0D0A0000A3
:10D6500041542B43475245473F0D0A0041542B513B
:10D66000494143543F0D0A0041542B51434349441F
:10D670000D0A000041542B514E57494E464F0D0A9A
:10D680000000000041542B4353510D0A00000000DC
:10D6900041542B514944454143543D25640D0A00F2
:10D6A00041542B51494143543D25640D0A0000006B
:10D6B0002B435245473A00002B43475245473A0017
:10D6C0002B514E57494E464F3A0000002B435351C1
:10D6D0003A0000002B51494143543A002B51434337
:10D6E0004944000041542B5149434C4F53453D257B
:10D6F000642C31300D0A000041542B51494F5045E4
:10D700004E3D312C25642C22544350222C2225736B
:10D71000222C25642C25642C310D0A0041542B51F8
:10D720004953544154453D312C25640D0A000000F5
:10D7300041542B514953454E443D25642C25640DDD
:10D740000A0000002B514953544154453A0000004F
:10D750002B51494F50454E3A000000003E0000005A
:10D7600053454E44204F4B002573000041542B512C
:10D77000485454504346473D22636C6F736577614C
:10D78000697474696D65222C3130300D0A00000017
:10D7900041542B514854545055524C3D25642C361D
:10D7A000300D0A0041542B51485454504346473DD4
:10D7B00022636F6E74656E7474797065222C310DFE
:10D7C0000A00000041542B51485454504346473DF1
:10D7D0002272657175657374686561646572222C67
:10D7E000310D0A0041542B51485454504346473D93
:10D7F00022636F6E746578746964222C320D0A009E
:10D8000041542B5148545450504F53543D25642C8F
:10D81000362C360D0A00000041542B514854545008
:10D82000524541443D360D0A000000002B5148543A
:10D830005450504F53543A20302C323030000000B6
:10D840002B5148545450524541440000434F4E4ED2
:10D850004543540041542B51475053474E4D454189
:10D860003D22524D43220D0A0000000041542B512D
:10D870004750534346473D226E6D65617372632284
:10D880002C310D0A0000000041542B5147505343E6
:10D8900046473D226175746F677073222C310D0A03
:10D8A0000000000041542B514750533D310D0A00F8
:10D8B00041542B51475053454E440D0A000000007F
:10D8C0002B51475053474E4D45413A202447505223
:10D8D0004D43000020DA020800000020EC070000A1
:10D8E0006CC10108C4DD0208EC070020C4860000FA
:10D8F000C8C101081001000043000000F8FFFFFF4D
:10D900000040404040404040404041414141414052
:10D910004040404040404040404040404040404007
:10D920004005020202020202020202020202020296
:10D93000022020202020202020202002020202029B
:10D9400002029090909090901010101010101010F3
:10D9500010101010101010101010101002020202FF
:10D960000202888888888888080808080808080843
:10D97000080808080808080808080808020202023F
:10D980004000000000000000000000000000000057
:10D990000000000000000000000000000000000087
:10D9A0000000000000000000000000000000000077
:10D9B0000000000000000000000000000000000067
:10D9C0000000000000000000000000000000000057
:10D9D0000000000000000000000000000000000047
:10D9E0000000000000000000000000000000000037
:10D9F0000000000000000000000000000000000027
:10DA0000000000001C00000043000000F8FFFFFFC2
:10DA10000C0000000E0000000F0000002E000000AF
:10DA20000134320432301EE8D40208CC041AD8047F
:10DA300051320C6201177BE0010801011F05020150
:10DA40000106870C1302011F010302020ABB0C131B
:10DA500003011F020403030CEF0C130401100C0359
:10DA60000504040E23E1010805011F040105051149
:10DA7000570C180A06010109070606148B0C1A0731
:10DA8000441E08060615BF0C19551F070906061681
:10DA9000F30C1B090128181109091727E201080ACC
:10DAA00001020B0B0A0A185B0C180A0B01020A0A86
:10DAB0000B0B198F0C180A0C01030D0D0B0C1AC35C
:10DAC0000C180A0D01030C0C0D0C1BF70C18160E8C
:10DAD0000104100F0E0E1C2BE301080F01040E10A1
:10DAE0000F0F1D5F0C180A1001040F0E10101E936B
:10DAF0000C180A110105131211111FC70C281D1251
:10DB000001051113121220FDE40108130105121181
:10DB100013132137E5010814010614011A710C2DA5
:10DB200015010715011AA70C1A16031E1612161650
:10DB3000FF0C2D1701091701280957E601081801E4
:10DB40000A18011AAD0C2D19010B1901280905E756
:10DB500001081A010C1A011A5D0C2D1B010D1B0185
:10DB60001AB10C2D1C010E1C011AD70C2D1D010F12
:10DB70001D01280923E801081E01101E01290C2D92
:10DB80001F01111F011AA50C2D20011220012809C7
:10DB90001DE901082101132101852DEA0108223028
:10DBA000400E3132312E352E3231372E3235321889
:10DBB0000E581B701714D50208F4D4020804081A72
:10DBC0008004C11AA410238A021AF0081AFF011156
:10DBD0001AD628191032011ABC14320AAAEC1C22D7
:10DBE00003191F111AC414190B115AD41C1ADC087A
:10DBF0001A043529145A901CB938193532040A15FB
